:020000040800F2
:100000000000022049F50008218800082388000824
:1000100025880008278800082988000800000000BB
:100020000000000000000000000000002B88000815
:100030002D880008000000002F8800083188000883
:100040008DF500088DF500088DF500088DF5000888
:100050008DF500088DF500088DF50008358800083D
:100060008DF500088DF500088DF500082D5C000861
:100070008DF500088DF500088DF500088DF5000858
:100080008DF500088DF500088DF500088DF5000848
:100090008DF500088DF500088DF50008058A00082B
:1000A0008DF500088DF500088DF500088DF5000828
:1000B00059880008698800088DF500088DF500084A
:1000C0008DF500088DF500088DF500088DF5000808
:1000D0008DF500088DF50008198B00088DF50008D6
:1000E0008DF500088DF500088DF500088DF50008E8
:1000F0008DF500088DF500088DF500088DF50008D8
:100100008DF500088DF500088DF500088DF50008C7
:100110008DF500088DF500088DF500088DF50008B7
:100120008DF500088DF500088DF500088DF50008A7
:100130008DF500088DF500088DF500088DF5000897
:100140008DF500088DF500088DF500085D88000824
:100150008DF500088DF500088DF500088DF5000877
:100160008DF500088DF500088DF500088DF5000867
:100170008DF500088DF500088DF500088DF5000857
:080180008DF500088DF5000863
:10018800ACA60508000000200C0B0020100B002076
:10019800EC610020064B07481A68074B1A60074BAA
:1001A80000221A70064B01221A7001F070B800BFC5
:1001B80080400020180D0020944000206C40002052
:1001C800943A002008B5034801F061F8024B002278
:1001D8001A7008BDA80F0020943A002008B5054BF6
:1001E800012200201A7004F04DF80348BDE80840C9
:1001F80001F04DB82C4100204C1000202DE9F041B1
:10020800144C204602F083FB00201349134A02F0E5
:1002180035F91349134A0746002002F02FF912490D
:10022800124A0646002002F029F9D22105463A462C
:1002380023460A2002F03AFAD22132462346FA200F
:1002480002F034FA5A20D2212A462346BDE8F0416A
:1002580002F02CBA600E0020D2960508CD010008E5
:10026800DB960508E5010008E39605089D010008EE
:1002780008B5054B012200201A7004F003F8034862
:10028800BDE8084001F003B82C4100204C100020C4
:10029800044B054800221A70044B02221A7000F021
:1002A800F6BF00BF6C400020600E0020943A00208A
:1002B80008B5034800F0EBFF024B00221A7008BD96
:1002C800A80F0020943A00202DE9F041144C204654
:1002D80002F01DFB00201349134A02F0CFF813491E
:1002E800134A0746002002F0C9F81249124A064686
:1002F800002002F0C3F8D22105463A4623460A20D8
:1003080002F0D4F9D221324623465A2002F0CEF91F
:10031800AA20D2212A462346BDE8F04102F0C6B9F8
:10032800180D0020D2960508B9020008EC960508B9
:1003380099020008F596050879020008002008B51A
:1003480003F0A0FF064B00221A70064B1B78022B05
:100358000CBF05480548BDE8084000F098BF00BF3D
:100368002C410020943A0020600E0020180D002037
:1003780010B5084C204602F0CAFA00200649074A80
:1003880002F07CF8D22102462346E620BDE8104060
:1003980002F08CB994110020FE9605084503000868
:1003A80010B5074C4FF6E071206801F0BBFB2068E0
:1003B800044901F065FBBDE8104002F0E1BC00BF54
:1003C800100B00200797050810B5074C4FF6E07191
:1003D800206801F0A7FB2068044901F051FBBDE843
:1003E800104002F0CDBC00BF100B00201C97050880
:1003F80070B5514C2DED028B20684FF6E07101F07D
:1004080091FB20684D4901F03BFB02F0B9FC00204C
:1004180003F038FF23790BB9FFF7C2FF6379464D24
:1004280053B928684FF6E07101F07CFB286844490D
:1004380001F026FB02F0A4FCA3790BB9FFF7C4FF77
:100448003D4C6379002B69D02379002B66D094ED5D
:10045800038AD4ED048A78EE687A88EE288AA2683E
:10046800384B394D1A6017EE900A0EF0F1F9002258
:10047800364B0EF041FA02460B46002034490EF086
:1004880065FB0EF01BFD334B0646186018EE100A8C
:100498000EF0DEF90022304B0EF07AF802460B46D9
:1004A80000202B490EF052FB21A3D3E900230EF0C4
:1004B8006FF80EF003FDA2792860002323716371A1
:1004C80002B1A371254A1F4C137031464FF4967040
:1004D80005F01DFC29684FF4987005F018FC216898
:1004E8004FF49A7005F013FC1A4B94ED001A124C55
:1004F80093ED000AD5ED000A07F096F820684FF64C
:10050800E07101F00FFB2068154901F0B9FA07F016
:10051800BEF802F035FC134802F076FC1248BDEC38
:10052800028BBDE8704000F0B2BE00BFAFF30080A0
:100538000000000000805140100B00203197050892
:10054800469705080C0D0020100D002000005E40A5
:1005580000004940140D00200000F03F943A0020AC
:100568005B97050880969800A80F0020014800F0C6
:100578008EBE00BFA80F00202DE9F047384C394D3A
:10058800A3686068AB600EF063F9064620680F4602
:100598000EF05EF90022344B0EF0AEF900228046D0
:1005A800894630463946304B0DF0F4FF42464B46FB
:1005B8000EF0CCFA0EF082FC25A3D3E90023686183
:1005C800394630460DF0E6FF42464B460EF0BEFA7D
:1005D8000EF074FCA8614FF6E07003F027FE68691E
:1005E800224E0EF035F905F11C0402460B46204652
:1005F800314612F0FBFD224600236E203A2103F01B
:1006080043FFA8690EF024F902460B4620463146FE
:1006180012F0ECFD224600236E206C2103F034FF1B
:10062800A8680EF015F90CA3D3E900230EF064F9BD
:1006380002460B4620460E4912F0D8FD6E209E2138
:1006480022460023BDE8F04703F01EBFAFF3008049
:100658000000000000805140000000A2941A6D4282
:10066800DC5E0020100B002000005E406F9705083C
:100678007597050870B506F0D1FF10EE104A06F020
:10068800E3FF064620460EF0E3F807EE106AF8EEA0
:10069800C77A044617EE900A0D460EF0D9F81AA349
:1006A800D3E900230EF028F902460B4620462946D6
:1006B8000EF04CFA0EF002FC114CA0600EF0C8F8D7
:1006C8000DA3D3E900230EF017F904F11C05024627
:1006D8000B4628460B4912F089FD4FF6E07003F0EF
:1006E800A5FD00236E209E212A4603F0CDFE01239E
:1006F800A37170BDAFF30080000000A2941A6D4290
:10070800100B0020759705081F85EB51B81E19407E
:1007180038B506F077FF0F4C10EE100A84ED030A87
:100728000EF096F804F11C0502460B4628460A49C5
:1007380012F05CFD4FF6E07003F078FD00236E20A8
:100748003A212A4603F0A0FE01236371BDE8384030
:1007580026E600BF100B00206F97050838B506F095
:1007680051FF0F4C10EE100A84ED040A0EF070F8D9
:1007780004F11C0502460B4628460A4912F036FDCC
:100788004FF6E07003F052FD00236E206C212A46DC
:1007980003F07AFE01232371BDE8384014E600BF58
:1007A800100B00206F9705082DE9F04F4F4D504E64
:1007B80085B000244FF6FF78284602F0A8F8414695
:1007C800224623464B480094019401F06FF9042710
:1007D8007062224623464FF6E0714748009701941D
:1007E80001F064F9414630602246234643480097A9
:1007F800019401F05BF94146B06222462346404825
:100808000097019401F052F92346F06241462246CE
:100818003C480097019401F049F93B4930633B4A51
:10082800204601F02BFE3A493A4A0746204601F095
:1008380025FE3949394A8046204601F01FFE3849CD
:10084800384A8146204601F019FE3749374A824620
:10085800204601F013FE3649364A84462046CDF834
:100868000CC001F00BFE21468346726A2B462046D7
:1008780001F01CFF214632682B467D2001F016FF4F
:100888006E21F26A2B460A2001F010FF3C21326BE0
:100898002B460A2001F00AFF69213A462B46E6203A
:1008A80001F004FF372142462B46E62001F0FEFE08
:1008B8004A462B46E6209B2101F0F8FE52462B467D
:1008C8006E20C82101F0F2FEC8215A462B46AA2004
:1008D80001F0ECFEDDF80CC0E620C82162462B468C
:1008E80005B0BDE8F04F01F0E1BE00BF040F0020E5
:1008F800100B00207E9705084697050832970508D3
:10090800869705089F970508B997050865070008A1
:10091800C097050819070008C89705087D0600084C
:10092800D097050881050008D697050875050008C1
:10093800DD970508F9030008014B93ED000A70479D
:10094800140D0020014B93ED000A7047100D002094
:10095800014B93ED000A70470C0D0020AFF30080A7
:10096800294B2A48062210B51A704FF6E07400F099
:100978008EFC0020214607F059F83120214607F067
:1009880055F86320214607F051F89520214607F0D5
:100998004DF81F34C7204FF4FC6107F047F8204694
:1009A80003F044FC052001210023194A03F06CFDE3
:1009B800052020210023174A03F066FD0520522157
:1009C8000023154A03F060FD84210520134A002303
:1009D80003F05AFD4FF4FC6003F028FCB621052013
:1009E8000F4A002303F050FD204603F01FFC0D4A78
:1009F80000238720DC2103F047FD0B4B00221A60FF
:100A08000A4B01221A7010BD2C410020DC12002074
:100A1800E49705081998050811980508C99F05085D
:100A2800269D0508E8970508844000206C400020B2
:100A38003B4B3C48072270B51A704FF6E07400F043
:100A480026FC0020214606F0F1FF3120214606F061
:100A5800EDFF6320214606F0E9FF9520214606F0C8
:100A6800E5FF4FF6FF752146C72006F0DFFF284651
:100A780003F0DCFB0520012100232B4A2B4E03F059
:100A880003FD052020210023294A03F0FDFC052051
:100A980052210023274A03F0F7FC05208421002374
:100AA800254A03F0F1FC0520B6213246002303F065
:100AB800EBFC40F213144FF4FC6003F0B7FB204644
:100AC80001211E4A002303F0DFFC204620211C4A96
:100AD800002303F0D9FC204652213246002303F0BC
:100AE800D3FC20468421174A002303F0CDFCB6210D
:100AF800154A0023204603F0C7FC284603F096FB5E
:100B0800124A00237D20DC2103F0BEFC104B00229A
:100B18001A60104A012313700F4A137070BD00BF8A
:100B28002C410020DC120020ED9705080F9C0508D9
:100B3800F1970508F5970508F8970508019805083D
:100B4800FD970508FC97050800980508059805080D
:100B5800844000206C400020684D002038B52D4BA3
:100B68002D4805241C704FF6E07500F090FB00201E
:100B7800294606F05BFF2720294606F057FF4F203D
:100B8800294606F053FF7720294606F04FFF9F209D
:100B9800294606F04BFF2946C7201F3506F046FFB9
:100BA800284603F043FB0121002320461B4A03F09B
:100BB8006BFC162100232046194A03F065FC3E21F0
:100BC80000232046174A03F05FFC662100232046D5
:100BD800154A03F059FC8E2100232046134A03F0DE
:100BE80053FCB621124A0023204603F04DFC284648
:100BF80003F01CFB0F4A00237D20DC2103F044FC9A
:100C08000D4B00221A600D4A012313700C4A137011
:100C180038BD00BF2C410020DC1200200F9C0508C5
:100C28001098050814980508189805081C980508D0
:100C38002098050824980508844000206C4000206E
:100C4800684D0020F8B53B4B3B483C4F3C4E0422D6
:100C58001A704FF6E07400F01AFB0020214606F0E7
:100C6800E5FE3120214606F0E1FE6320214606F02C
:100C7800DDFE9520214606F0D9FE4FF6FF75214688
:100C8800C72006F0D3FE284603F0D0FA052001213C
:100C980000233A4603F0F8FB052020210023294AC7
:100CA80003F0F2FB052052210023274A03F0ECFB56
:100CB800052084210023254A03F0E6FB0520B62100
:100CC8003246002303F0E0FB40F213144FF4FC60BB
:100CD80003F0ACFA204601213A46002303F0D4FB86
:100CE800204620211A4A002303F0CEFB2046522139
:100CF8003246002303F0C8FB20468421154A00230E
:100D080003F0C2FBB621144A0023204603F0BCFBC3
:100D1800284603F08BFA114A00237D20DC2103F0DA
:100D2800B3FB0F4B00221A600E4A012313700E4AC0
:100D38001370F8BD2C410020DC12002045980508EE
:100D48000F9C05083098050840980508359805084F
:100D58003A9805083F9805084498050848980508F2
:100D6800844000206C400020684D0020F8B5324BCC
:100D78003248334F334E03221A704FF6E07400F0B6
:100D880086FA0020214606F051FE6320214606F02F
:100D98004DFEB3204FF4FC6106F048FE2146C72003
:100DA8001F3406F043FE204603F040FADC210023FE
:100DB8007D20254A03F068FB204603F037FA05201A
:100DC800012100233A4603F05FFB0520522100234E
:100DD8001E4A03F059FBB62100230520324603F0D2
:100DE80053FB40F213154FF4FC6003F01FFA002385
:100DF800284601213A4603F047FB5221284632464D
:100E0800002303F041FBB621114A0023284603F0D2
:100E18003BFB204603F00AFA0E4A00230520A221D4
:100E280003F032FB0C4B00221A600C4A01231370AA
:100E38000B4A1370F8BD00BF2C410020DC120020C3
:100E4800629805080F9C0508539805085D980508E1
:100E58006198050821980508844000206C4000200E
:100E6800684D002008B5074B074802221A7000F0A9
:100E78000EFA06F0D5FC054B00221A60044B01223D
:100E88001A7008BD2C410020DC120020844000208C
:100E98006C400020002008B503F0F4F9064B00224E
:100EA8001A70064B1B78022B0CBF05480548BDE895
:100EB800084000F0ECB900BF2C410020943A002013
:100EC800600E0020180D00202DE9F14F2D4C204612
:100ED80001F01DFD00202C492C4A01F0CFFA2C49C5
:100EE8002C4A8146002001F0C9FA2B492B4A0746B3
:100EF800002001F0C3FA2A492A4A0646002001F0D8
:100F0800BDFA2949294A0546002001F0B7FA2849BF
:100F1800284A8046002001F0B1FA2749274A82462C
:100F2800002001F0ABFAD22183464A462346E62048
:100F380001F0BCFB28203A462346014601F0B6FBE7
:100F4800462132462346282001F0B0FB64212A4678
:100F58002346282001F0AAFB822142462346282066
:100F680001F0A4FB524623462820A02101F09EFB55
:100F780028205A46BE21234601B0BDE8F04F01F0B3
:100F880095BB00BF4C100020FE9605089D0E00087A
:100F9800669805086D0E000853980508750D000839
:100FA800489805084D0C000871980508650B00085D
:100FB8007C980508390A0008E897050869090008B7
:100FC80008B5002003F05EF906F0EEFA06F06AF8BC
:100FD800064B00221A70064B01221A7006F084FD97
:100FE8000448BDE8084000F052B900BF2C41002079
:100FF800943A0020180D002008B5002003F042F9AB
:1010080006F0D2FA064B00221A70064B02221A701A
:1010180006F06AFD0448BDE8084000F038B900BF92
:101028002C410020943A0020600E002008B50020D2
:1010380003F028F9034B044803221A70BDE808405E
:1010480000F025B9943A0020040F002010B50B4C8D
:1010580006F0AAFA04F0A4F806F01FFB06F044FD17
:1010680020684FF6E07100F05DFD2068044900F04B
:1010780007FDBDE8104001F083BE00BF440B00200F
:10108800869805080088C83880B2042810B505D9A4
:101098000A480B4A0B4B7F2102F09AF80A4CC0B25F
:1010A80004F008F920684FF6E07100F03BFD206875
:1010B8000649BDE8104000F0E3BC00BF9A98050857
:1010C800BCD00308BA980508440B0020EB98050823
:1010D8002DE9F04F5248534D85B0002401F017FC1C
:1010E8004FF6FF71224623464F480094019400F0C2
:1010F800DDFC042607464FF6E071224623464B489E
:101108000096019400F0D2FC4FF6E071804622462A
:10111800234647480096019400F0C8FC4FF6FF713B
:1011280081462246234643480096019400F0BEFCBF
:10113800234628604FF6FF7122463F4800960194E7
:1011480000F0B4FC3D4968603D4A204601F096F93C
:101158003C493D4A8246204601F090F93B493C4AC9
:101168008346204601F08AF93A4902903A4A2046D5
:1011780001F084F93A4603902146294B204601F0B4
:1011880095FA21464246264BC82001F08FFA0A21DB
:101198004A46234BC82001F089FA2A68204B64216B
:1011A800782001F083FA78206A681D4B014601F027
:1011B8007DFAC82505262827E0B203F0ABFF274AA9
:1011C8000146284601F05AF994FBF6F106FB114155
:1011D80079431E31024689B20020114B0134013592
:1011E80001F064FA042CADB2E6D1D22152460520B2
:1011F8000B4B01F05BFAD2215A464C20084B01F008
:1012080055FAD221029A064B9C2001F04FFA039A14
:10121800034BEC20D22105B0BDE8F04F01F046BAEF
:10122800A80F0020440B0020FB9805080599050825
:10123800129905081D99050832970508319905087E
:101248005510000839990508351000084299050815
:10125800011000084B990508C90F00088D100008F7
:1012680008B500F005FAFEF7C9FFFFF79DFAFFF78A
:101278002BF8FFF729FEFFF72BFFFFF779F800F0AF
:101288008BFA00F0D9F8BDE8084000F0A1B910B514
:10129800044628B90F48104A104B452101F098FF21
:1012A8000F4B1868844213D010B1C36900219847C6
:1012B800002002F0E7FF002002F0CEFF4FF6FF709B
:1012C80002F0B4FFE369204601219847044B1C60F3
:1012D80010BD00BF54990508CBD0030870990508C4
:1012E8004C0B00200048D2E7A80F00204FF6FF70F3
:1012F80070474FF6FF70704713B5002944D04FF27E
:10130800DE7002F0BFFF002003F086F80F2002F025
:101318008DFF1E4C1E4A412101230A2003F0B4F818
:10132800042003F079F8236828209621042B21DC77
:101338000123184A03F0A8F801A90DF10602206854
:1013480003F02AFB0F2002F071FFBDF80400BDF87E
:10135800061014382822002380B202F097FFBDF847
:101368000610BDF80400143989B22822012302F0BE
:101378008DFF09E0084A012303F086F81E20A52105
:10138800064A012303F080F81CBD00BF500B002063
:101398008099050893990508AF990508C599050826
:1013A80037B51E4C2368042B05462BDC01A80DF12C
:1013B800060103F0EFFABDF80630BDF8042018491D
:1013C800042007F06BFD2368002B04DA1548164A41
:1013D800164B592105E0042B05DD1248124A144B1F
:1013E8005A2101F0F5FE04EB8302BDF80410013325
:1013F8009180BDF806102360052BD18008D1201DEF
:1014080003F04AFB00230B482360FFF740FF03E08B
:1014180028460121FFF770FF3EBD00BF500B00209A
:10142800DC990508219A0508DDD00308439A0508C8
:101438005A9A0508F010002037B50B4C204601F0E9
:1014480066FA0A4B0A49009300250120094A0A4B0B
:10145800019501F004F9294602462346284603B0BF
:10146800BDE8304001F022B9BC0D0020011300088E
:10147800F5120008FB120008A91300084FF6FF70C8
:1014880070474FF6FF7070471FB54FF6E07002F0D7
:10149800F9FE002002F0C0FF0F2002F0C7FE002175
:1014A800294A2A4C01230A2002F0EEFF002002F00C
:1014B800BDFE042002F0B0FF0A201921244A0123AE
:1014C80002F0E2FF2521234A01230A2002F0DCFF73
:1014D8001F2002F0ABFE01230A2037211E4A02F02A
:1014E800D3FF237873B301231E2096211B4A02F0F1
:1014F800CBFF62881A49684611F078FE01231E2046
:10150800A2216A4602F0C0FFA2881649684611F077
:101518006DFEAE216A4601231E2002F0B5FF0F20A2
:1015280002F084FE6088A188143880B22822002343
:1015380002F0ACFEA1886088143989B22822012300
:1015480002F0A4FE1FBD00BF889A0508680B0020A2
:101558009A9A0508BA9A0508DA9A0508FD9A0508BC
:101568000F9B05081C9B050801B18DE7704713B553
:101578000DF1060101A803F0C1F9144B01221A70FC
:101588005988BDF80420891A0E311C2919460AD831
:101598009C88BDF80600201A0E301C2803D89968CC
:1015A8000131996001E000238B60084B996801299B
:1015B80005DD00229A601A70FFF794FE05E05A8054
:1015C800BDF806209A80FFF75FFF1CBD680B00205E
:1015D80037B50B4C204601F09AF90A4B0A4900939B
:1015E80000250120094A0A4B019501F038F82946DF
:1015F80002462346284603B0BDE8304001F056B8FD
:10160800F010002071150008851400088B140008DC
:101618007715000838B50D4B0D4D00241C700D4B87
:101628001C700D4B4FF0FF321A600C4B1A680C4BB4
:1016380020461A6002F026FE0A4B1B78022B0CBFCC
:1016480009480A48FFF723FE2C7038BD2C410020BA
:10165800684D00206C40002084400020804000201D
:1016680094400020943A0020600E0020180D0020BD
:1016780010B50B4C204601F04AF9002001462246DD
:1016880000F074FA00200749074A00F0F7FED2215B
:10169800024623464FF48270BDE8104001F006B8B8
:1016A800DC120020D69705081D16000810B5064C58
:1016B8004FF6FF71206800F035FA044B206819686E
:1016C800BDE8104000F0DCB9740B00209801002040
:1016D80008B5002002F0D6FD054B1868054B1968BF
:1016E80000F0CEF90448BDE80840FFF7D0BD00BFC0
:1016F800740B002094010020A80F002008B5FFF704
:10170800D5FF0020014605F043FEBDE8084001F082
:1017180037BB0088A0F5C87080B2092808B505D97C
:101728000748084A084B8F2101F052FD074B1880E3
:10173800074BFF21197005F02BFEBDE80840B5E7FF
:10174800299B0508EFD003084C9B0508801300204F
:10175800821300200088A0F5967080B2092808B589
:1017680005D90848084A094B832101F031FD084B87
:101778001880084B0121197005F00AFEBDE80840E1
:1017880094E700BF299B050804D103084C9B050872
:1017980080130020821300202DE9F34100243A48E9
:1017A8003A4D01F0B4F8224623464FF6FF71384807
:1017B8000094019400F07AF904262246234607464D
:1017C8004FF6FF7133480096019400F06FF92346F5
:1017D800286022464FF6FF712E480096019400F0CB
:1017E80065F92D4968602D4A204600F047FE2C49CE
:1017F8002C4A0646204600F041FE214680463A46DD
:101808002046214B00F052FF2A681F4B2046282112
:1018180000F04CFF3246D2211B4B5A2000F046FF05
:10182800AA20D2214246184B00F040FF0F254FF462
:10183800967440F2351620461B491C4A00F01EFEDD
:1018480001340246782128460F4BA4B2233500F014
:101858002DFFB442ADB2EED10F254FF4C87440F25B
:10186800991620461249134A00F008FE0134024630
:101878009B212846044BA4B2233500F017FFB4423D
:10188800ADB2EED1BDE8FC8138120020740B002007
:101898007D9B050843970508899B050805170008DF
:1018A800929B0508D91600089B9B05085D17000840
:1018B8009D9B05081B17000808B508B143682BB99C
:1018C8000348044A044B9B2101F082FC586908BD77
:1018D8009F9B050818D10308C19B050808B5FFF7A9
:1018E800EBFF8068123080B208BD08B5FFF7E4FF4F
:1018F8004068063080B208BD2DE9F84F0446884696
:10190800FFF7DAFF6689E589074606F1030905F15D
:101918000F0AB8F1000F1FD01F2002F087FC2046E5
:10192800FFF7DCFF83462046FFF7DFFF2946034623
:101938005FFA8BF2F0B202F0ADFC042002F06CFD0D
:101948000B364FF6FF70033502F070FCB0B2A9B247
:101958003A68012302F098FD3D69204641464A460F
:101968005346A847BDE8F88F13B504460DF10601A4
:1019780001A802F0C3FF2046FFF79EFF6389BDF868
:101988000410BDF80620C91AE389D21A0339C368BE
:101998000F3A204698471CBDF7B5044614200D465B
:1019A80016461F4611F0B0F8089BC7600361064B46
:1019B8000649074A80E8700000930190054B002013
:1019C80000F04DFEFEBD00BF01190008F318000825
:1019D800E518000871190008704708B508B1436890
:1019E8002BB90448044A054BAD2101F0F1FB5869B5
:1019F80008BD00BFE09B050830D10308C19B05085E
:101A0800F8B505460E46FFF7E8FF836B04461BB1A1
:101A180028463146984700E018466F8994F83C30CC
:101A2800ED890EB9034310D0208E02F0FFFB608EC3
:101A380002F012FC94F8350002F0EEFC94F8343011
:101A480038462946224602F01FFD002384F83C3020
:101A5800F8BD08B5FFF7C1FF90F83500BDE80840AC
:101A680002F0EFBC38B5FFF7B8FF044611F044FCAC
:101A7800054694F8350002F0DFFC684380B238BDB3
:101A880038B50D46FFF7A9FF29462E22044611F066
:101A980063FC50B1204629462E2211F0AFFC0023EA
:101AA80084F82E30012384F83C3038BD2DE9F74303
:101AB800074640200E461546984611F025F804467C
:101AC80028B91148114A124B4E2101F081FB114BE4
:101AD800114A12498DE818000020114B00F0BFFD93
:101AE80039468146FFF7CCFF9DF82830268684F8D2
:101AF80035300B9B6586A363002384F8348084F813
:101B08003C304846BDE8FE83E09B050848D1030801
:101B1800FE9B0508091A00085B1A00086D1A0008E0
:101B2800E119000810B50C46FFF757FF012304869A
:101B380080F83C3010BD00BF4FF4A0707047C8203B
:101B480070477047074B1B78022B07B508D1064B27
:101B58001B78022B04D001A80DF1060102F0CEFE7D
:101B68000EBD00BF684D00202C41002073B50A4B04
:101B780006460D461446009300200849084A094BBA
:101B8800019000F06CFD294602462346304602B01B
:101B9800BDE8704000F08ABD4B1B0008411B0008DF
:101BA800471B00084D1B000813B502AB03E90600EC
:101BB800436843B1027C0124082A9C7004D11B6944
:101BC8002146984700E01C4620461CBD30B5002839
:101BD8002BD0058B002425E0036A1A7C012A05D145
:101BE8005B681A888A421BD1187F30BD052A06D146
:101BF8005B681A888A4213D193F82C0030BD032AF7
:101C080006D15B681A888A420AD193F8250030BD4C
:101C1800062A05D15B681A888A4201D1D87A30BD74
:101C280001340430AC42D7D3002030BD08B18175EF
:101C380001207047F8B504460D46D0B1E175D0F8DB
:101C480098309847012D0DD12746002606E0F869FF
:101C580000F10802436906CA98470136238B043706
:101C68009E42F4D3D4F8983020462946984701205C
:101C7800F8BDF8BDF8B50546084617460E4611F0FA
:101C88003BFB013FB84234BF04463C463CB12846C2
:101C98003146224611F0B2FB00232B55F8BD2C70BB
:101CA800F8BDF7B5044600200090019000296CD0DB
:101CB8000E8B68E000F1080351F823301D7C042DD9
:101CC80004D15D682D88954247D0013000F10803A2
:101CD80051F823301D7C012D04D15D682D88954273
:101CE8003BD0013000F1080351F823301D7C052D4D
:101CF80004D15D682D8895422FD0013000F108038A
:101D080051F823301D7C032D04D15D682D88954240
:101D180023D0013000F1080351F823301D7C022D37
:101D280004D15D682D88954217D0013000F1080371
:101D380051F823301D7C072D04D15D682D8A95420A
:101D48000BD0013000F1080351F823301D7C062D1B
:101D580008D15D682D88954203D103F1080120461A
:101D680015E0013000F1080351F823502B7C082BB3
:101D780009D16F683F88974204D105F108012046D0
:101D88001A4605E00130B04294D32046694608223D
:101D980011F06AF92046FEBDF8B505460F4616460D
:101DA800002830D04388032B2FD0202010F0ACFE21
:101DB800044600282BD040F80C5B39460C22FFF76C
:101DC80059FF1820E66110F09FFE0646B8B10223BD
:101DD8000374012363760F4B446063600E4BA3606A
:101DE800002323766B8805EB830201339BB2012B1A
:101DF80050606B800CD16A685268137608E0204600
:101E080010F08AFE04E0064602E0002600E00646DE
:101E18003046F8BDB8500408564D040837B5456833
:101E280002AB03E906003DB3037C0124042B85F8CB
:101E3800314022D1688E02F0F9F995F8300002F0AD
:101E4800EBFA95F8343043B9BDF80200BDF8061036
:101E5800AA1C234602F018FB0FE0012B03D1084807
:101E680040F2395104E0022B07D1054840F24151B4
:101E7800044A054B01F0ACF92C4620463EBD00BF94
:101E8800119C0508081C04080F9C0508F8B50446B1
:101E98000F46164610B3838A0A2B20D0202010F054
:101EA80033FE0546E8B14460102200F108003946C7
:101EB800FFF7E0FE4FF6FF73A08A2B801F236B808D
:101EC80000232B76831D013080B20128EE6144F88F
:101ED8002350A08207D1A3691876F8BDF8BD002069
:101EE800F8BD0120F8BD0120F8BD2DE9F0411D46DF
:101EF8004B1C984280460C4617460CDD95420ADC7E
:101F0800013208F101035B1A521BC8B2D2B29BB26C
:101F1800294602F0BDF9A8F10208BDF81800C4EB83
:101F2800080802F083F901261FFA88F808E0A919C1
:101F3800601C80B289B24246002302F0A7F901363C
:101F48007B1B9E42F3D3BDE8F081F8B5C7B21446B7
:101F580038461E460D4602F09FF9621E92B2384678
:101F6800294602F099F9304602F060F9022606E0A7
:101F7800A21B92B23846294602F08EF90136A642D3
:101F8800F6D3F8BD70B5044600F11E003C220023CC
:101F980080B20D4602F07AF91E3DA9B220463C22D5
:101FA8000123BDE8704002F071B970B504460138EC
:101FB8000322002380B20D4602F068F9013DA9B260
:101FC800204603220123BDE8704002F05FB9F7B54F
:101FD800089D2E7BEF7A1C463604AB7A06EB072663
:101FE800F618431A687B06EB00602D180020019054
:101FF800121B08462146009501F098FEFEBD30B53B
:10200800456885B004AB03E906007DB101242C7353
:102018006D68BDF80800BDF80A109DF80C209DF801
:102028000E300095FFF7D3FF204600E0284605B0A4
:1020380030BD2DE9F04385B004AB03E906004468E0
:10204800BDF80860BDF80C70002C41D0012384F85D
:10205800263094F825300BB9A26800E06268FFB218
:10206800BDF80A109DF80E30009230463A46FFF748
:10207800AEFF04F10C08022002F0CEF9404611F040
:102088003BF9054600B1451E0F3F0024153E1FFAD7
:1020980087F90DE002F0CAF902F0CEF904FB1061ED
:1020A80089B248462022002302F008FA0134E4B23B
:1020B800AC42EFD3002002F0B9F8B8B2B1B2424650
:1020C800012302F0FBF9002002F0A6F9012000E04C
:1020D800204605B0BDE8F0832DE9F04385B004AB98
:1020E80003E906004568BDF80860BDF80C70002DCE
:1020F8003CD001236B762B7EBDF80A10012B0CBF58
:102108006A68AA689DF80E300092FFB23A463046D7
:10211800FFF75DFF0C35022002F07EF9284611F02A
:10212800EBF80E3F81460024163E1FFA87F80DE0B3
:1021380002F07CF902F080F904FB106189B2404694
:102148002022002302F0BAF90134E4B24C45EFD959
:10215800002002F06BF8B8B2B1B22A46012302F0AF
:10216800ADF9002002F058F9012000E0284605B03A
:10217800BDE8F0832DE9F04F85B00546DDF84090C5
:10218800029148469046039311F0B6F8DDF838A05E
:10219800DDF83CB00646294600242F4611E024B15C
:1021A800B4420CBF5B46534600E0039B01F10805AF
:1021B800ADB200932846029A4346FFF708FF013460
:1021C8002946B442EBDD002002F030F8022002F08C
:1021D80023F97D1D08F10508A8B21FFA88F14A46BF
:1021E800012305B0BDE8F04F02F04EB970B5406864
:1021F80086B006AB03E9060000282ED0012380F83C
:102208002D308668164BF21A534243EB020390F8BE
:102218002C205AB1002B134D134B144A08BF1D46EE
:10222800134B00F11C0418BF13460AE0002B0D4D98
:102238000D4B0E4A18BF1D460D4B00F10C0408BF8C
:102248001346BDF81200BDF81410BDF8162000960C
:1022580001950294FFF78EFF012006B070BD00BF04
:1022680078250408B42104085A270408962304088A
:102278003C29040870B5446886B006AB03E906003B
:1022880004B301236377A668104B227FF11A4B42EF
:1022980043EB01030AB10BB904E01BB966680C4DA6
:1022A8000C4B01E00C4D0D4BBDF81200BDF814109D
:1022B800BDF8162000960C3401950294FFF75AFFDA
:1022C800012000E0204606B070BD00BFC4300408FD
:1022D800002D0408E22E0408A632040888340408F5
:1022E8002DE9F04385B004AB03E906004468BDF866
:1022F8000860BDF80A90BDF80C50BDF80E80002C9F
:1023080000F08C800123A3740220676802F084F82F
:102318004FF6FF7001F0A0FF002001F087FFEDB23B
:102328005FFA88F8A6F1160189B230462A46434674
:102338000097FFF74CFE277A002F2ED1A28A23465A
:1023480000E00137974204D29969097E04330029D5
:10235800F7D002F06BF802F06FF8A9F116091FFA2E
:1023680089F90E2101FB10914FF6FF7208F101085F
:102378005FFA88F389B2009248462A46FFF7B5FD0E
:10238800022002F049F81F2001F050FFA38A002B19
:1023980038D0103DE8B2303E2CE0E3685C68A28A91
:1023A8002346013A002700E00137974204D2996991
:1023B800097E04330029F7D002F038F802F03CF81F
:1023C8000E2101FB10914FF6FF7208F101085FFA28
:1023D80088F389B2009248462A46FFF786FD022014
:1023E80002F01AF81F2001F021FFA38A53B1103D13
:1023F800E8B21A3E0637B1B254F827200123083252
:1024080002F05CF8002002F007F84FF6FF7001F0C8
:1024180023FF1F2001F00AFF012000E0204605B03D
:10242800BDE8F0832DE9F04105463620884614467C
:102438001F4610F069FB0646E0B120F8025B4146F2
:102448002E22FFF717FCBDF8183086F83440738643
:102458001820012386F8307086F8313010F054FBCC
:10246800044618B104234660037404E0304610F0B3
:1024780053FB00E004462046BDE8F081F8B5064667
:1024880024200F46154610F03FFB0446D8B10F4BE9
:10249800068083600E4B39464360102200F10C0021
:1024A800FFF7E8FB012600231820256223776677CB
:1024B80010F02AFB054610B14460067404E020467B
:1024C80010F02AFB00E005462846F8BDC430040891
:1024D8001E2B0408F8B506462C200F46154610F0AA
:1024E80013FB0446E8B120F80C6B39461922FFF7B4
:1024F800C1FB0D4BA562A3600C4B6360002384F8FD
:1025080025301820012384F8263010F0FDFA0546FE
:1025180018B103234460037404E0204610F0FCFA69
:1025280000E005462846F8BDF44904089246040828
:1025380010B50446142010F0E7FA20B100234380B8
:10254800014B0480036110BDA11D000838B5054684
:10255800442010F0D9FA0446C0B10E4B05824360FE
:102568000D4B0360012383740023037283820B4B9A
:102578000364182010F0C8FA054618B10723446010
:10258800037404E0204610F0C7FA00E00546284628
:1025980038BD00BF884204087E3E0408951E000826
:1025A8002DE9F04105463420884614461F4610F0B0
:1025B800ABFA064620B3144B05808360134B4146A3
:1025C8004360102200F10C00FFF754FB214606F18E
:1025D8001C001022FFF74EFB002386F82C30182031
:1025E8000123376386F82D3010F08EFA044618B1AF
:1025F80005234660037404E0304610F08DFA00E0CD
:1026080004462046BDE8F08178250408D21F040856
:102618002DE9F041044614200D461646984610F060
:1026280073FA0746B8B1069B048003610023C3729E
:1026380001234560068180F80A800373182010F092
:1026480063FA044618B106234760037404E0384669
:1026580010F062FA00E004462046BDE8F0812DE95A
:10266800F041044618200D461646984610F04CFADC
:102678000746B8B101238370069B04800361079B5A
:1026880045608660C0F80C804361182010F03CFA61
:10269800044618B108234760037404E0384610F074
:1026A8003BFA00E004462046BDE8F0812DE9F341FD
:1026B80098461B8B1D2B05460C4617464FF000000D
:1026C80000F2B480B5F5A07F0090019000F2AE80D2
:1026D800F02900F2AB80127CADF80610511EADF85F
:1026E8000250072900F28A80DFE801F045595E04AC
:1026F800456A14767B684E4A7A611A8893F83430B2
:102708003A80013BDBB2012B7FD8ADF80240ADF82F
:1027180006507AE005F11602ADF8002004F1160221
:10272800ADF8042002AE434A16E903007A6107F1C6
:10273800080282E8030003F10802013348F8227016
:10274800A8F818307B681A8A187A3A8000286CD161
:10275800FFF7FCFE3849436859603849DF600126B5
:10276800163D196002461E72A8B2E1B24346FFF751
:102778009DFF30465AE0012A0CBF314B314B786837
:102788007B6130F80C3B3B8010F0B6FD431CDB004E
:102798001A34ED18ADF80440ADF8005035E07B6808
:1027A800294A1B687A6102E0284A7B687A611B889B
:1027B80014353B80ADF800501434ADF8044024E0E3
:1027C8007B68234A7A611A883A801A899B7AAD18FD
:1027D800ADF80050E418F0E77E681E4B7B61338843
:1027E80038463B8073689847013D4519ADF800505D
:1027F800B36838469847013C0419DEE71648174A7B
:10280800174B40F21A3100F0E3FC02AA12E9030068
:1028180007F1080383E80300B8F8183003F1080249
:10282800013348F82270A8F818300120BDE8FC816F
:10283800251E0008E9220008743A04086A360408CC
:102848007D220008F5210008E12000083B2000084F
:1028580007200008B11B0008119C0508181C040873
:102868000F9C0508F8B51646002834D01378002BBD
:102878002ED0028B002327E0046A257C042D21D169
:1028880065682F888F421DD195F8313053B16F8E0E
:1028980001F0F2FC04F1080268866369204606CA62
:1028A80098476F86A81C31462E22FFF7E3F995F862
:1028B80031307BB104F108026369204606CA9847A3
:1028C8000120F8BD013304309342D5D30020F8BD70
:1028D8001846F8BD0120F8BD70B5B8B1068B04469E
:1028E800002310E0256A287C04280AD16D6828880E
:1028F800884206D11046A91C2E22FFF7BBF90120F9
:1029080070BD01330434B342ECD3002070BD38B538
:10291800044620B3134BC361134BC0F89830134BD4
:10292800C0F89C30124B00257822C0F8A03085757D
:10293800C5750583294600F1200010F0D7FBD4F8AF
:1029480098302046294698470A4A1388312B07D8D9
:10295800094941F8234001331380012038BD38BDAF
:10296800284638BD3D1C0008351C0008D51B00084A
:10297800AB1C00087C0B0020841300202DE9F041DB
:102988000446002800F0B380078B02460025A8E023
:10299800136A1E7C042E00F08780012E23D158680C
:1029A80003888B4240F09B8005F1080710F0B4F8CB
:1029B80054F827004FF00008C0F8048010F0ACF875
:1029C800228B531E9D4208D00732238354F82210CD
:1029D80044F8271044F8228002E044F82780258331
:1029E8003046BDE8F081052E5ED0032E5CD0022E65
:1029F80013D15B68186803888B4270D14388013B08
:102A08009BB243800BB910F087F805F1080654F81B
:102A18002630586810F080F84EE0072E21D15E6805
:102A2800338A8B425BD1002706E0BB1D013756F87D
:102A3800230010F071F8FFB2B38ABB42F5D8002723
:102A4800B78205F1080654F82630586810F064F883
:102A580054F8260033E044F8267025830120BDE8A9
:102A6800F081062E1ED1586803888B4237D105F1B4
:102A7800080610F051F854F826000027476010F0B7
:102A88004BF8228B531E9D4209D00833013A54F863
:102A98002310228344F8261044F82370DEE744F814
:102AA80026701AE0082E1AD1586803888B4216D16E
:102AB80010F032F805F1080654F8260000274760A0
:102AC80010F02AF8228B531E9D42C4D0073254F8C6
:102AD800221044F8261044F822702383BEE70135FB
:102AE8000432BD42FFF454AF0020BDE8F081BDE8D8
:102AF800F08170B5044600282AD0068B751E08366A
:102B080000EB86061EE056F8043D1A7C042A13D012
:102B1800012A11D0052A0FD0032A0DD0022A02D18A
:102B28005B681B6809E0072A02D15B68198A05E01F
:102B3800062A01D0082A04D15B6819882046FFF7C5
:102B48001DFF013D681CDED100232383012070BDD9
:102B580070BDF0B528B30023068B1A461EE0046A40
:102B6800257C072D18D16468258A8D4214D1A78A3F
:102B7800002504EB83040DE004EB050C0435DCF8B8
:102B880018C09CF818C0BCF1010F03F1010301D172
:102B9800D8B2F0BDBB42EFD301320430B242DED32B
:102BA8000020F0BD70B508B3048B00231BE0026A57
:102BB800157C072D15D15268158A8D4211D1002335
:102BC800958A11461C46012007E013B996693076AC
:102BD80001E08E69347601330431AB42F5D301202C
:102BE80070BD01330430A342E1D3002070BD2DE94C
:102BF800F04128B30023078B1A461EE0046A257C9F
:102C0800072D18D16468258A8D4214D1B4F814C0F0
:102C1800002504EB83040CE066190435B66996F8C0
:102C28001880B8F1010F03D106F10800BDE8F08162
:102C380001336345F0D301320430BA42DED30020B9
:102C4800BDE8F0812DE9F04700282FD00023B0F827
:102C580018C01D4627E0046A267C072E21D1646827
:102C6800268A8E421DD1B4F81480002604EB83090D
:102C780015E009EB0604A7693C7E012C0DD192F8FA
:102C880000A0BAF1000F08D007F108001146102281
:102C9800FEF7F0FF2046BDE8F087013304364345D0
:102CA800E7D3013504306545D5D30020BDE8F0876A
:102CB800F0B5B0B1068B002510E0046A277C062F1A
:102CC8000AD1646827888F4206D123819DF8143081
:102CD8006260A3720120F0BD01350430B542ECD327
:102CE8000020F0BD10B500210446FEF7A3FF2046E2
:102CF8000121BDE81040FEF79DBF38B598B1048B9F
:102D0800024600230CE0106A058804328D4206D181
:102D180000F10802436906CA9847012038BD01330B
:102D2800A342F0D3002038BD10B50C460021FEF7B1
:102D380081FF20460121BDE81040FEF77BBF13B597
:102D480002AC04E90C00BDF80230834206D8BDF895
:102D58000030834234BF0020012000E00020BDF88D
:102D680006308B4206D8BDF804308B4234BF0021B0
:102D7800012100E00021002818BF0846C0B21CBD90
:102D880038B5114B114A1988002319E052F8045F2D
:102D9800A87D012812D100240CE004F1080355F89D
:102DA8002300037C082B03D1436800211B69984743
:102DB8000134A4B22B8BA342EFD838BD01339BB2A8
:102DC8008B42E3D138BD00BF7C0B0020801300206C
:102DD800704770B5094CA5787DB9094B1E78012E4E
:102DE8000BD16368013363606268064B9A4204D969
:102DF800284601F0D3FAA670656070BD7C0B0020F0
:102E08003000002040420F00054A9060134602E05F
:102E180099680139996091680029F9D1704700BF14
:102E28007C0B0020F0B585B001F066FD002800F0AD
:102E38004981002502A80DF10A01ADF80850ADF846
:102E48000A5001F05BFD03A80DF10E01ADF80C501E
:102E5800ADF80E5001F09EFDBDF80C10BDF808202D
:102E68000091BDF80E10BDF80A3001912C46964D20
:102E78009649082006F012F8A878012803D101F035
:102E88008DFAAC7019E1924B5B78012B40F01581FB
:102E9800AB78002B40F011816B6029888D4A09E1DD
:102EA80052F8046FB07D012840F002810025FAE055
:102EB80005F10803BDF8080056F82340BDF80A10CC
:102EC80004F108030CCBFFF73AFF002800F0E98073
:102ED800237C013B062B00F29F80DFE803F00429E6
:102EE800159D1F9D4C006668012304F10805337782
:102EF80095E8060063692046984700233377204603
:102F0800636995E8060086E0636893F8252012F166
:102F1800FF3218BF012283F8252077E0636893F811
:102F28002C2012F1FF3218BF012283F82C206DE00B
:102F38006268137E1568002B6ED16E882F4629466D
:102F4800184606E051F804EFDEF804E001338EF885
:102F58001800B342F6D301231376002607E057F88A
:102F6800040F00F10802436906CA984701366B88C6
:102F78009E42F4D350E0656820892E68A37B227BAB
:102F88000096A0F1160189B2FFF721F81420FFF787
:102F98003BFF2B7AC3B9AF8A29461A461E4609E079
:102FA800886990F818E00676BEF1010F08BF13464D
:102FB80004310132BA42F3D301220BB9AB6924E0E0
:102FC800053355F8233020E06368DB685A6800232E
:102FD800908A154619461F4609E0AE6996F818E02A
:102FE8003776BEF1010F08BF0B4604350131814227
:102FF800F3D3411E8B4203D1053052F8203003E051
:1030080004D2073352F8233001221A7604F1080259
:1030180006CA636920469847237C013B072B4CD896
:10302800DFE803F00410074B0A0D123A63681B6AC5
:1030380034E063689B6A2DE063681B6B2AE0636871
:103048001B6927E0636824E063681A7A7AB9988A6A
:103058001946013800E00132824204D28C69247E8C
:103068000431002CF7D0063253F8223011E0DB6827
:103078005A68908A11460138002300E001338342E0
:1030880004D28C69247E0431002CF7D0063352F820
:103098002330DB69984710E06368DB68204698476F
:1030A8000BE00135ADB2338BAB423FF601AF04E024
:1030B80001339BB28B427FF4F3AE01F063FC0F2027
:1030C800FFF7A2FE05B0F0BD7C0B0020379C050879
:1030D8003000002080130020034B9A6812B19A68D0
:1030E800013A9A60704700BF7C0B00202DE9F34736
:1030F8000120DFF8D080DFF8D090014609F0F6FF14
:103108000025012403234FF48076022740466946B0
:103118008DF8053000968DF804708DF806508DF8FE
:10312800074009F03BFC40460821224609F0B6FC5E
:10313800234BDFF898801A6844F2A243B2FBF3FAF3
:103148000AF1FF3A204621461FFA8AFA09F0FEFFE3
:10315800C8F804A048464146A8F80050A8F802500C
:10316800A8F8085088F80A500AF08CFB7023A8F8D1
:103178000C300423A8F810300AF1FF3A63236422C4
:1031880003FB0AF3B3FBF2F39BB2C8F8143008F15F
:103198000C014846A8F80E40A8F81870A8F81A506C
:1031A800A8F81C60A8F81E500AF08AFC4846214678
:1031B8000AF0FDFB484621460AF003FFBDE8FC87FC
:1031C800A401002000000240000001408C0B0020F8
:1031D80083B50E460746154910201C46154605F0CE
:1031E8005DFE1020124905F059FE1020114905F026
:1031F80055FE10200E4905F051FE002310200E49FF
:10320800019305F04BFE334610200C493A4605F071
:1032180045FE10200A492A4605F040FE10200949BB
:10322800224605F03BFE019B0133E7E7719C050848
:10323800769C0508969C0508A69C0508B69C05087A
:10324800CB9C0508DC9C050808B5164B1A6A0132A8
:103258001A621A6A012A1A4603D013484FF4A07159
:103268000FE05862194602E04B6A013B4B62506A14
:103278000C4B0028F8D11A6A012A06D00A4840F2F5
:103288004B110A4A0A4BFFF7A3FF1A6A013A1A625E
:103298001B6A2BB10448054A064B40F24D11F2E770
:1032A80008BD00BF8C0B0020ED9C05081A540408CB
:1032B800179D0508289D05080C4B0D491A6844F20E
:1032C800A2436428B2FBF3F3D4BF20EAE070642081
:1032D800013B9BB24B60013B58436422B0FBF2F0C8
:1032E80080B2486103480C310AF06DBBA40100208C
:1032F8008C0B00200000014010B5134B93F82820D8
:103308002AB11248124A134B4FF40A710EE00122F7
:1033180083F8282066234FF0C042013BDBB21080BF
:1033280033B90A480A4A0C4B40F23221FFF750FFE2
:103338001488A4B28442F0D1084B1980024B0022B1
:1033480083F8282010BD00BF8C0B0020ED9C0508D9
:1033580024540408399D05080F9C050800000260E4
:1033680010B5FFF7C3FE6420FFF7A6FFE5204FF472
:103378000041FFF7C1FF00200121FFF7BDFF012039
:103388004FF48071FFF7B8FF02204FF4E061FFF7B8
:10339800B3FF032041F23001FFF7AEFF0420002104
:1033A800FFF7AAFF082040F20221FFF7A5FF092036
:1033B8000021FFF7A1FF0A200021FFF79DFF0C2045
:1033C8000021FFF799FF0D200021FFF795FF0F203F
:1033D8000021FFF791FF10200021FFF78DFF11203A
:1033E8000021FFF789FF12200021FFF785FF132036
:1033F8000021FFF781FF102041F2B071FFF77CFF39
:1034080037211120FFF778FF3220FFF71DFF122028
:1034180040F23B11FFF770FF3220FFF715FF132032
:103428004FF4C051FFF768FF0F212920FFF764FF11
:103438003220FFF709FF20200021FFF75DFF212040
:103448000021FFF759FF30200021FFF755FF3120F9
:103458000721FFF751FF322040F20311FFF74CFF1D
:10346800352040F20741FFF747FF40F20444362079
:1034780040F60F11FFF740FF37202146FFF73CFFCA
:1034880038204FF48061FFF737FF39202146FFF7D6
:1034980033FF3C200021FFF72FFF3D204FF48061D0
:1034A800FFF72AFF50200021FFF726FFEF215120C8
:1034B800FFF722FF52200021FFF71EFF532040F2A2
:1034C8003F11FFF719FF60204FF41C51FFF714FF5D
:1034D80061200121FFF710FF6A200021FFF70CFF90
:1034E80080200021FFF708FF81200021FFF704FF5B
:1034F80082200021FFF700FF83200021FFF7FCFE58
:1035080084200021FFF7F8FE85200021FFF7F4FE54
:1035180090201021FFF7F0FE92200021FFF7ECFE2B
:1035280093200321FFF7E8FE95204FF48871FFF7F9
:10353800E3FE97200021FFF7DFFE98200021FFF728
:10354800DBFE072040F27311BDE81040D4E610B549
:10355800FFF7CCFD6420FFF7AFFE21210720FFF71E
:10356800CBFE3220FFF770FE01210020FFF7C4FEDA
:103578003220FFF769FE23210720FFF7BDFE322026
:10358800FFF762FE00211020FFF7B6FE40F6B830C4
:10359800FFF75AFE33210720FFF7AEFE3220FFF770
:1035A80053FE112046F63001FFF7A6FE3220FFF742
:1035B8004BFE4FF4C0610220FFF79EFE3220FFF75A
:1035C80043FE122046F6EB41FFF796FE3220FFF746
:1035D8003BFE03204AF6A401FFF78EFE3220FFF7D8
:1035E80033FE00210C20FFF787FE3220FFF72CFE68
:1035F8000D2040F60C01FFF77FFE3220FFF724FE76
:103608000E204FF42C51FFF777FE3220FFF71CFEF7
:10361800B0211E20FFF770FE3220FFF715FE0120B3
:1036280042F63F31FFF768FE3220FFF70DFE052016
:103638000021FFF761FE3220FFF706FE0021062079
:10364800FFF75AFE3220FFF7FFFD16204EF61C71D9
:10365800FFF752FE3220FFF7F7FD172040F2031163
:10366800FFF74AFE3220FFF7EFFD00210B20FFF79E
:1036780043FE3220FFF7E8FD00210F20FFF73CFE54
:103688003220FFF7E1FD41200021FFF735FE32200F
:10369800FFF7DAFD42200021FFF72EFE3220FFF768
:1036A800D3FD00214820FFF727FE40F23F143220C7
:1036B800FFF7CAFD21464920FFF71EFE3220FFF71B
:1036C800C3FD00214A20FFF717FE3220FFF7BCFD9B
:1036D80000214B20FFF710FE3220FFF7B5FD4420F4
:1036E8004FF46F41FFF708FE3220FFF7ADFD0021D0
:1036F8004520FFF701FE3220FFF7A6FD21464620B0
:10370800FFF7FAFD3220FFF79FFD302040F20771E6
:10371800FFF7F2FD3220FFF797FD31204FF40171DA
:10372800FFF7EAFD3220FFF78FFD32204FF40171D9
:10373800FFF7E2FD40F202543220FFF785FD2146F3
:103748003320FFF7D9FD3220FFF77EFD342040F209
:103758000751FFF7D1FD3220FFF776FD35204FF4F2
:103768000171FFF7C9FD3220FFF76EFD36204FF4D7
:103778000171FFF7C1FD3220FFF766FD21463720B2
:10378800FFF7BAFDA4F500743220FFF75DFD21466E
:103798003A20FFF7B1FD3220FFF756FD2F2041F206
:1037A800BE21FFF7A9FD3220FFF74EFD21463B2041
:1037B800FFF7A2FD3220FFF747FD00212320FFF786
:1037C8009BFD3220FFF740FD00212420FFF794FDE8
:1037D8003220FFF739FD25204FF40041FFF78CFD1B
:1037E8003220FFF731FD00214F20FFF785FD322001
:1037F800FFF72AFD4E200021FFF77EFD3220BDE8AD
:10380800104021E508B5124B93F829202AB1114838
:10381800114A124B40F242210FE0012283F829207D
:10382800222166234FF0C042013BDBB2118033B93D
:103838000848094A0A4B40F25B21FFF7C9FC108887
:1038480080B22228F0D1024B002283F8292008BD3B
:103858008C0B0020ED9C050831540408399D05089F
:103868000F9C050810B5224B49F22032032823D8B3
:10387800DFE800F0021A0B111C8846F6280041F216
:103888002801944218BF01461AE01C8841F208003A
:1038980046F6080104E01C8841F2300046F6300183
:1038A800944208BF01460BE0188846F62001904272
:1038B80008BF4FF4815103E00E4840F2792113E02C
:1038C8001B8848F68912934205D049F22032934268
:1038D80007D1032000E01120FFF70EFDBDE81040DE
:1038E80090E7044840F28521034A044BFFF770FC37
:1038F80032000020ED9C0508465404080F9C05087A
:10390800014B18800A209FE4000002604FF0C0437A
:10391800188003F500331A881A88188880B270470F
:103928002DE9F041022098B00121002409F0DEFBC6
:10393800012502268C488DF85C5016A98DF85E404A
:103948008DF85F4016968DF85D6009F027F818200D
:10395800294609F0CBFB2846294609F0DFFB21461A
:103968000C22824809F09AF829460C227F4809F06F
:1039780095F804210C227D4809F090F805210C22C5
:103988007A4809F08BF807210C22784809F086F864
:1039980008210C22754809F081F809210C22734886
:1039A80009F07CF80A2171480C2209F077F80B21FC
:1039B8006E480C2209F072F80E210C226B4809F0AF
:1039C8006DF80F210C22694809F068F807210C22CC
:1039D800674809F063F808210C22654809F05EF889
:1039E80009210C22624809F059F80A210C22604882
:1039F80009F054F80B210C225D4809F04FF80C210E
:103A08000A465B4809F04AF80D210C22584809F08B
:103A180045F80E210C22564809F040F80C2254486B
:103A28000F2109F03BF803274CF6B3734F48169360
:103A380016A98DF85D708DF85E408DF85F408DF8A1
:103A48005C6008F0ABFF4FF6807316A948481693E0
:103A58008DF85D708DF85E408DF85F408DF85C6084
:103A680008F09CFF40F6B830FFF7EEFB22463146DF
:103A78003D4809F008F844F6FF70FFF7E5FB2A46D1
:103A88003146394808F0FFFF40F6B830FFF7DCFB55
:103A98004FF48053102709930DF13C084FF400238D
:103AA80068460F94109412941395149415940094E6
:103AB8000194029404940694079408940A94059433
:103AC8000B940C9311960397CDF8348008F0DFFC23
:103AD8000423684611931094129413951494159422
:103AE8000F96CDF8388008F0D2FC2946204608F019
:103AF8004EFD40F6B830FFF7A7FB2046FFF706FF5C
:103B080004461C491C4D3846224605F0C7F948F6BC
:103B180089139C421AD049F220339C420DD041F2BD
:103B280089239C4212D03846144905F0B7F9144845
:103B3800144A154BA621FFF74BFB3846134922467A
:103B480005F0ACF92C80FFF70BFC0AE0FFF7FFFC4F
:103B580048F689122A8010200D4941F2892305F080
:103B68009DF918B0BDE8F08100040240000C024045
:103B7800001002404E9D050832000020659D050892
:103B8800ED9C05085E5404080F9C05089C9D0508DB
:103B9800D19D05084FF0C04322221A8003F5003357
:103BA80082B01A8892B2ADF806201B889BB2ADF895
:103BB8000630BDF8060080B202B07047134B1B8870
:103BC80048F68912934210B504460BD049F22032C8
:103BD800934213D1C1F1EF01202089B2FFF78CFB8A
:103BE800212006E0C1F1EF014E2089B2FFF784FBE6
:103BF8004F202146BDE81040FFF77EBB0448054A28
:103C0800054B40F2F321FFF7E3FA00BF3200002032
:103C1800ED9C0508675404080F9C05082DE9F04140
:103C28000D46C5F1F008411E5E18C2EB0802C5F149
:103C3800EF039BB292B2B6B29A422CBF9046984616
:103C48009A4234BF11461946864234BF3746074662
:103C580040F23F13864238BF06469E4228BF1E46A2
:103C68001B4B1B8848F68912B8F1EF0F28BF4FF09D
:103C7800EF089342044610D049F2203293421FD1F4
:103C88005020FFF739FB51204146FFF735FB522002
:103C98003946FFF731FB53200AE041EA082189B28F
:103CA8004420FFF729FB45203946FFF725FB46202E
:103CB8003146FFF721FB20462946BDE8F0417DE764
:103CC8000448054A054B40F2DD21FFF781FA00BFA1
:103CD80032000020ED9C0508755404080F9C050867
:103CE80000200146F0224FF4A07397E7072040F226
:103CF8007311FFF701BB07200021FFF7FDBA10B5CC
:103D08001446FFF75BFFFFF77DFD2046BDE8104036
:103D1800F6E508B5FFF752FF4FF0C04322221A809C
:103D280003F500331A88188880B208BDF8B580B248
:103D380002FB03F589B292B29BB2069C9DF81C6007
:103D4800FFF76CFF0020FFF78DFD002709E034F82E
:103D5800020B1EB1030A43EA002080B2FFF7D0FD30
:103D68000137AF42F3DBBDE8F840B9E72DE9F74F7B
:103D780016469DF834200C9F01920546B2B280B2D7
:103D88000C46984689B29BB2FFF748FF4FF0000BEC
:103D98000020FFF767FDDA463DE0002D30DB09EB38
:103DA800050340F23F1293422ADC002C28DB0BEB80
:103DB8000403EF2B24DC19F00F0F04D1B9F1000F25
:103DC800C8BF0AF1010A174B09EA0303002B03DAFB
:103DD800013B63F00F030133019A0AB1C3F10F03EA
:103DE800012202FA03F337F81A2013401BB213B169
:103DF8000D4B588D01E00D4A508880B2FFF780FDC9
:103E080009F1010901E04FF00009C145C5DB0AF1DC
:103E1800010A0BF1010BB345F5DB03B0BDE8F04F28
:103E28005EE700BF0F0000808C0B002032000020EE
:103E38002DE9F04F85B004469DF83C00029200271A
:103E48008A46039088463E4640F23F1C9B463AE02D
:103E5800002C2FDBE1452DDCBAF1000F2ADBB8F18D
:103E6800EF0F27DC2A0702D1002DC8BF01361B49F6
:103E78002940002903DA013961F00F010131039A61
:103E88000AB1C1F10F010E9830F8162003FA01F1BA
:103E98000A4012B272B112494A8D019392B21FFAC6
:103EA80089F01FFA88F1CDF800C0FFF728FFDDF888
:103EB80000C0019B013509F101095D45C8DB0136E8
:103EC800013708F10108029A974203DAA146002552
:103ED8000123F2E705B0BDE8F08F00BF0F000080B6
:103EE8008C0B002082B0044BADF80600BDF806200C
:103EF80092B25A8502B070478C0B002082B0044BF6
:103F0800ADF80600BDF8062092B25A8002B070479C
:103F18003200002070B50646FFF7E2FE0020FFF7EA
:103F2800A1FCF02409E0013D3046ADB2FFF7E8FC02
:103F3800002DF8D1013CA4B214B14FF4A075F2E7FA
:103F480070BD70B51D461446FFF738FE2846FFF7CA
:103F580089FC0025054E05E0708D80B2FFF7D0FC86
:103F68000135ADB2A542F7D170BD00BF8C0B002062
:103F78002DE9F0410C4616461F461A460023054611
:103F8800FFF7DFFF611E711828463A46002389B201
:103F9800FFF7D7FF2846214632460123FFF7D1FF16
:103FA800013D7F19B8B2214632460123BDE8F041F0
:103FB800C7E770B580B202FB03F489B292B29BB234
:103FC800FFF72CFE0020FFF74DFC0025054E04E00E
:103FD800708D80B2FFF794FC0135A542F8DBBDE88F
:103FE80070407DE68C0B0020F8B5561A0C4601315E
:103FF80089B21F460546FFF7E1FD0120FFF732FCB5
:104008004FF0C04322221A800E4A0F491388B6B2D5
:10401800002304E01088013321F8020B9BB2B3425D
:10402800F8D121462846FFF7C9FD0120FFF71AFC01
:10403800002404E03846FFF763FC0134A4B2B4421C
:10404800F8D1F8BD000002606A4D002070B5194B28
:10405800194AD98D92F9004064180025A4B2AC42DF
:1040680008BF0124C62C28BFC6240F2615704FF69A
:10407800FF7288B09E85DC855A8519200A222B4656
:104088002146FFF75EFF21463046FFF742FE2246F3
:1040980003460A4968460FF0A9F86A4604A8084981
:1040A8000FF0A4F83220D22104AA2B4600F0ECF934
:1040B80008B070BD8C0B0020302A0020109E050827
:1040C800189E05082DE9F0431F2093B0FFF722FF43
:1040D8004FF47840FFF71EFF4FF6E0754FF4FC6091
:1040E800FFF718FF2846FFF715FF0020494CFFF798
:1040F80011FF00200146642203464FF6FF79A4F819
:104108002A90FFF71EFF00200A2164220346FFF7CA
:1041180018FF00200146642201234FF47847658583
:10412800FFF70FFF7720EF21C82200234FF4FC662A
:104138006785FFF706FFBD213222012340F23F10B9
:104148006685FFF7FEFEA0203222002378216785CE
:10415800FFF7F7FEA0207821322201234FF01F0835
:104168006685FFF7EEFEA020782132220223A4F80C
:104178002A80FFF7E6FEA0207821322203236585F6
:10418800FFF7DFFE244B2549A3F8028002AD3C224D
:1041980028460EF069FFEB20C32105223023009545
:1041A8000025A4F82A900195FFF7E0FD32210A20A6
:1041B80096220B466785FFF7DBFE32213C209622CC
:1041C8000B466685FFF7D4FE32210B4696226E20F9
:1041D800A4F82A80FFF7CCFEFFF78DFDFFF786FDD8
:1041E8003220FFF769F82846FFF766F86420FFF7E2
:1041F80063F80B4B03F110028DE8240028465A6837
:104208001B682946FFF792FD1195119B0133119305
:10421800FBE700BF8C0B0020320000208A54040802
:10422800A8780108004870475014002082B0064B57
:10423800ADF80600BDF8062092B21A80188880B240
:1042480002B0FFF74FBE00BF4C140020014B188886
:1042580080B270474C14002082B0064BADF80600BF
:10426800BDF8062092B21A80188880B202B0FFF713
:1042780045BE00BF4E140020014B188880B270471D
:104288004E140020FFF746BEFFF7C8BCFFF759BE23
:10429800FFF76EBEFFF78DBE2DE9F04F4FEA4208DB
:1042A80000253D4C85B082468B46C8F10308174669
:1042B8002E461FFA87F909EB0B0C228805EB0A0337
:1042C8001FFA8CFC9BB26146184692B2CDF804C026
:1042D8000293FFF714FDC9EB0B0292B20392029B03
:1042E80022880399184692B2FFF709FDDDF804C049
:1042F8002288C5EB0A039BB26146184692B2029324
:10430800FFF7FDFC029B22880399184692B2FFF73B
:10431800F6FC05EB0B0292B2039209EB0A03228822
:1043280003999BB2184692B20293FFF7E8FC029BEE
:104338002288C5EB0B0C1FFA8CFC1846614692B21A
:10434800CDF804C0C9EB0A09FFF7D9FC2288039904
:104358001FFA89F992B24846FFF7D1FC2288DDF8A6
:1043680004C092B248466146FFF7C9FCB8F1000F95
:1043780004DA08EB860808F1060805E0F31B08F1E3
:104388000A0808EB8308013F01360135BE42ADB289
:104398008FD905B0BDE8F08F4C14002008B9FFF79D
:1043A800AABC012801D1FFF7A1BC704770470020C3
:1043B8000146F0224FF4A073FFF730BC704708B5F0
:1043C80005280CD8DFE800F012140305070909488E
:1043D80008BD094808BD094808BD094808BD09487D
:1043E800094A0A4B40F24111FEF7F2FE084808BD9F
:1043F800084808BD20000020100000200800002008
:10440800000000201D9E0508C65404080F9C0508DE
:10441800280000201800002010B50446FFF7CFFF41
:10442800014B18601C7110BD38000020014B187931
:10443800704700BF3800002008B5FFF7C0FF80882C
:1044480008BD08B5FFF7BBFFC08808BDF7B51F4614
:104458000B4B0C4E1D681446EA882B68203C5443CD
:10446800A4B2AE1B03EB440418BF0126AB888DE849
:10447800500017B1FFF7DCFC01E0FFF777FCFEBD49
:1044880038000020280000202DE9F0410F4698460A
:1044980015460446084E08E0204643463946FFF7CD
:1044A800D5FF33689B88E418A4B215F8012B002ABD
:1044B800F2D1BDE8F08100BF3800002010B50446F5
:1044C80008462146BDE81040DEE7094B70B50446B2
:1044D80018790E461546FFF7B4FFC6F1F001091A20
:1044E80089B220462A460023BDE87040CCE700BFC9
:1044F80038000020704700BF044B1A680AB9044A04
:104508001A601A681018186010467047BC0B002013
:10451800EC6100204FF0FF30704708B50248034AAD
:10452800034B3721FEF754FE3C9E0508DC54040873
:104538000F9C05080120704710B504460A4802215F
:1045480009F05AF80028F9D00748214609F01DF863
:104558000548012109F050F80028F9D00248BDE8C3
:10456800104009F00FB800BF0038004010B51948D6
:10457800022109F041F80028F9D01648002109F075
:1045880004F81448012109F037F80028F9D0114837
:1045980008F0F8FF0402A4B2002301E001339BB243
:1045A800002BFBD00B48022109F026F80028F9D08F
:1045B8000848002108F0E9FF0648012109F01CF825
:1045C8000028F9D0034808F0DDFF2043C0F3CB00F2
:1045D80010BD00BF003800402DE9F0478AB00AAF8F
:1045E8000A20012108F082FD4FF4604347F8143D8A
:1045F800474EDFF824A1012400254FF00208304679
:1046080039468DF81A508DF818808DF819808DF874
:104618001B4008F0C3F930460D21052208F03EFA88
:1046280030460E21052208F039FA052230460F21BE
:1046380008F034FA21464FF4804008F07BFD5046DC
:1046480008F056FE4FF48273ADF802304FF4007351
:10465800ADF80A303823ADF80C30504607236946C8
:10466800ADF81030ADF80050ADF80450ADF8065074
:10467800ADF80850ADF80E5008F06CFE50462146D3
:1046880008F003FFA9468DF81A5030464FF48055BC
:10469800394605958DF818408DF819808DF81B401E
:1046A80008F07CF93046294608F0E9F940253946F2
:1046B80018488DF818908DF819808DF81A908DF893
:1046C8001B40059508F06AF921464FF4804008F030
:1046D8003DFD0621032008F0C7FF0C2307A88DF82D
:1046E800213007958DF820908DF8224007F04AFE7A
:1046F80017238DF8243009A80F238DF825308DF85D
:1047080026308DF8274004F057FD0AB0BDE8F08741
:1047180000040240000C024000380040014B1878A9
:10472800704700BFC00B0020024B5A889B8802804C
:104738000B807047C00B0020014B00221A70704795
:10474800C00B0020F0B593B06846002148220EF057
:10475800CDFC6D46002464484FF4805108F091F96F
:10476800002301E001339BB2002BFBD09020FFF720
:10477800E3FE002301E001339BB2002BFBD0FFF7DF
:10478800F5FE4FF480510746574808F078F90023A2
:1047980001E001339BB2002BFBD053484FF480510A
:1047A80008F06FF9002301E001339BB2002BFBD026
:1047B800D020FFF7C1FE002301E001339BB2002B9C
:1047C800FBD0FFF7D3FE4FF480510646464808F069
:1047D80056F945F8047B01342E6244484021E4B27E
:1047E80008F03BF910B9092CB5D101E0092C78D1B2
:1047F8009DE80C00D218029B03980699D218049BD6
:10480800C018059BC018079BCB180899032490FB78
:10481800F4F092FBF4F25B1893FBF4F3151AC11A47
:104828009C1A002DB8BF6D420029B8BF4942002C20
:10483800B8BF6442502D03DD502909DD502C50DCEF
:104848008D4205DAAC424FF0020405DB111806E090
:104858008C424FF0020401DAD11800E0C1180A9B1B
:10486800099A0C980F9DD2180B9BD2180D9BC01853
:104878000E9BC018109BEB18119D91FBF4F10324BB
:1048880092FBF4F290FBF4F05B1993FBF4F3161A25
:10489800C41A9D1A002EB8BF7642002CB8BF6442D5
:1048A800002DB8BF6D42502E89B203DD502C09DDB2
:1048B800502D16DCA64205DAB5424FF0020405DB9E
:1048C800131806E0A5424FF0020401DAD31800E0FD
:1048D800C318074A93FBF4F39BB2938001235180DA
:1048E800137013B0F0BD00BF00040240000C02407A
:1048F800C00B002000000000FFF710BFF7B5054609
:104908000C4601A80DF10601FFF70EFF1B4BBDF881
:104918000660BDF8040093E80600724301FB00221C
:1049280099685218164992FBF1F207EE102AF8EE30
:10493800C77A40F23F17FCEEE77A17EE902A92B258
:10494800B2F5207F28BF3A462A801D69DA685B697C
:104958006E4302FB0060C01890FBF1F107EE101ADD
:10496800F8EEC77AFCEEE77A17EE903A9BB2B3F509
:10497800F07F28BFEF232380FEBD00BFC80B0020B7
:1049880040420F00FFF7D8BE014B187E704700BFAA
:10499800C80B0020FFF7C8BE042808B505D907488A
:1049A800074A084B7D21FEF713FC054B03EB8000FB
:1049B800038B0B80438B138008BD00BF5D9E0508E9
:1049C800E25404087B9E050808B5082001F090F918
:1049D80042F69643C31A584240EB030008BD10B58F
:1049E8000A2001F0ADF90C4C20600E2001F0A8F966
:1049F8006060122001F0A4F9A060162001F0A0F96F
:104A0800E0601A2001F09CF920611E2001F098F95D
:104A180001236061237610BDC80B002010B5FFF795
:104A2800DBFD01F02FFA044601F038FA0749034686
:104A38002246202004F032FAFFF7C6FF28B101F021
:104A48003BFA10B9BDE81040C9E710BDB79E05088C
:104A580010B5104C0A20216801F059F961680E2040
:104A680001F055F9A168122001F051F9E16816200A
:104A780001F04DF921691A2001F049F961691E20F8
:104A880001F045F9082042F69641BDE8104001F0D2
:104A980021B900BFC80B00202DE9F04F0346A7B08D
:104AA800B0F800C01C898688DF885D89CDF810C001
:104AB800B249B0F802C0B3F80C90B3F80E80CDF844
:104AC80024C00FFA84FB30B201220FFA87FE0BEBE9
:104AD800000C0A7629B20FFA89FACDF888C001EBE2
:104AE8000E0C0FFA88F2CDF890C00AEB0B0CCDF83B
:104AF80030C002EB010CCDF858C0B3F810C05B8A87
:104B0800CDF800C00FFA8CFC06910CEB00010A915D
:104B180002930CEB0A011BB2239103EB0E010E91D9
:104B280099182591049900FA81F05844504460443A
:104B3800DDF824C006990EFA8CFEDDF810C01FFAC5
:104B480080FB1CFB0CF08E4416FB0600964414FBFD
:104B58000400009A19FB09009E4412FB02001FFA88
:104B68008EFA09F053FEDDF824C0029ACDE912014D
:104B78001CFB0CF017FB070015FB050018FB0800D1
:104B880012FB020009F042FEDDF824C0029ACDE9CA
:104B9800140104991CFB01F317FB063615FB046688
:104BA800009B18FB096612FB036009F02FFEDDE984
:104BB8001423CDE90001DDE9120109F09DFE044648
:104BC8000D46DDE9000102460B4609F095FE024656
:104BD8000B462046294609F0DBFCCDE9180158466A
:104BE80009F024FECDE91001DDE91023DDE900011B
:104BF80009F082FECDE90601504609F017FE80460D
:104C080089464246DDE912014B4609F075FEDDE9A9
:104C18001023CDE91C01DDE9140109F06DFE002225
:104C280006460F46564BDDE9180109F065FE424677
:104C380004460D464B46DDE9060109F05DFE0246D5
:104C48000B4609F0A7FC02460B462046294609F008
:104C5800A1FC424604460D464B46DDE91C0109F01D
:104C68004BFE02460B462046294609F091FCDDE939
:104C7800102304460D463046394609F03DFE0246EB
:104C88000B462046294609F083FCDDF828C0CDE90B
:104C980002014FEA8C10DDF830C000EB0C20DDF883
:104CA80010C0A0241CFB040009F0B0FDDDF838C0DA
:104CB800CDE90A014FEA8C10DDF858C000EB0C2052
:104CC800DDF824C01CFB040009F0A0FDCDE90C01AF
:104CD800504609F09BFDDDE91023CDE91601DDE919
:104CE8000C0109F009FE4246CDE91E014B46DDE9FB
:104CF8000A0109F001FE4246CDE920014B46DDE9F3
:104D0800000109F0F9FD32463B4609F041FCCDE9C6
:104D18000E01584609F07AFDDDE91C23CDE91A0198
:104D2800DDE9060109F034FCDDF88CC0C024CDE9CA
:104D3800060104FB0CF0DDF888C0302505FB0C00EB
:104D4800DDF810C078261CFB060009F05FFDDDF8D1
:104D580094C0824604FB0CF0DDF890C005FB0C0003
:104D6800DDF824C01CFB06008B4609F04FFDDDE989
:104D7800102306460F4609F0BFFD03E0C80B0020CC
:104D8800000014404246CDE904014B4650465946BE
:104D980009F0B2FDDDE9142380468946DDE90A0100
:104DA80009F0AAFDDDE9002304460D46DDE90C0102
:104DB80009F0A2FD02460B462046294609F0E8FB09
:104DC8000022A14B09F098FDDDE9202304460D4699
:104DD800DDE91E0109F0DCFB02460B46DDE91601A0
:104DE80009F08AFD02460B462046294609F0D2FB07
:104DF800002204460D46954BDDE90E0109F07CFDC5
:104E080002460B462046294609F0C4FBDDE9022389
:104E180009F09CFE88A3D3E9002309F06DFD0AF090
:104E280005F88B490860DDE91223DDE90C0109F07A
:104E380063FDDDE9002304460D46DDE90A0109F0BA
:104E48005BFD02460B462046294609F0A1FB0022DD
:104E58007D4B09F051FDDDE91E2304460D46DDE9D1
:104E6800200109F095FB02460B46DDE91A0109F01D
:104E780043FD02460B462046294609F08BFB0022DB
:104E880004460D46714BDDE9060109F035FD024681
:104E98000B462046294609F07DFBDDE9022309F08F
:104EA80055FE65A3D3E9002309F026FD09F0BEFFEE
:104EB800674A5060DDE90E23DDE90A0109F01CFDAF
:104EC800DDE9062304460D46DDE90C0109F014FD71
:104ED80002460B462046294609F05CFB00220446A0
:104EE8000D465A4BDDE9180109F006FD02460B464E
:104EF8002046294609F04EFBDDE9022309F026FE8B
:104F08004DA3D3E9002309F0F7FC09F08FFF504BBC
:104F180059469860DDE91423504609F0EDFCDDE9B7
:104F2800002304460D463046394609F0E5FC0246A2
:104F38000B462046294609F02BFB0022424B09F07C
:104F4800DBFC424604460D464B46DDE9040109F008
:104F58001FFB02460B46DDE9160109F0CDFC0246AF
:104F68000B462046294609F015FB35A3D3E9002353
:104F780004460D46DDE90E0109F0BEFC02460B466B
:104F88002046294609F006FBDDE9022309F0DEFD8B
:104F980029A3D3E9002309F0AFFC09F047FFDFF8A4
:104FA800B0C0DDE91223CCF80C003946304609F0D0
:104FB800A3FCDDE9002304460D465046594609F096
:104FC8009BFC02460B462046294609F0E1FA0022DE
:104FD8001D4B09F091FCDDE9042304460D464046CB
:104FE800494609F0D5FA02460B46DDE91A0109F0EF
:104FF80083FC02460B462046294609F0CBFA10A34B
:10500800D3E9002304460D46DDE9060109F074FCE6
:1050180002460B462046294609F0BCFADDE9022380
:1050280009F094FD04A3D3E9002309F065FC09F015
:10503800FDFE074908610DE00000000080842E4154
:105048000000000000C082400000144000008940B9
:10505800C80B0020DDE90E235046594609F04CFCE8
:10506800DDE9062304460D463046394609F044FC7E
:1050780002460B462046294609F08CFA11A3D3E9CB
:10508800002304460D46DDE9180109F035FC024607
:105098000B462046294609F07DFADDE9022309F08E
:1050A80055FD0AA3D3E9002309F026FC09F0BEFE4A
:1050B800034A506127B0BDE8F04FC9E4AFF3008060
:1050C800C80B00200000000000C082400000000063
:1050D80080842E41AFF30080064B074A596811605F
:1050E8001969064A1160D969054A11609A6A054B1F
:1050F8001A60704740000020884000203841002096
:105108008C4000204C400020014B1878704700BFAD
:10511800E40B0020032808B505D90548054A064BC5
:105128007121FEF755F80C235843044B185808BD55
:10513800F29E05080E5504080C9F05084000002043
:10514800032808B505D90648064A074B7621FEF715
:105158003FF8064B0C2202FB0030406808BD00BF38
:10516800F29E05081E5504080C9F05084000002003
:10517800034B044A1B780C2101FB032398687047F2
:10518800E40B002040000020034B044A1B780C204D
:1051980000FB032399607047E40B002040000020C7
:1051A800144B1B78012B10B5134B144C0ED11968F6
:1051B800C82000F0ACFD2168CC2000F0A8FD104B01
:1051C800D020196800F0A3FDD4200DE01968D8207C
:1051D80000F09DFD2168DC2000F099FD084BE020DF
:1051E800196800F094FDE420064B1968BDE81040EA
:1051F80000F08DBD080D00208840002038410020B7
:105208008C4000204C400020144B1B78012B10B51B
:10521800134C0FD1C82000F093FD2060CC2000F083
:105228008FFD104B1860D02000F08AFD0E4B1860DF
:10523800D4200EE0D82000F083FD2060DC2000F0B0
:105248007FFD084B1860E02000F07AFD064B1860DF
:10525800E42000F075FD054B186010BD080D002016
:1052680088400020384100208C4000204C4000201D
:1052780008B502F001FA10B1BDE80840C4E7BDE87E
:10528800084029E70148FCF702B800BF381200209F
:105298000148FBF7FCBF00BF381200200148FBF7AC
:1052A800F6BF00BF381200200148FBF7F0BF00BF6F
:1052B80038120020032808B505D91448144A154B9C
:1052C8004E21FDF785FF144B1870144B02281870F7
:1052D800134B0FD0032813D0012805D0114A1268A8
:1052E8001A60BDE80840CDE70F4A12681A60BDE8A9
:1052F8000840CDE70D4A12681A60BDE80840CDE7BE
:105308000B4A12681A60BDE80840CDE7F29E05080E
:105318002F550408369F0508E40B00207E40002026
:1053280098010020900100208C01002088010020B5
:1053380084010020064B07495960C02100221972D8
:105348001E211A70D9601A745A611A76DA61704788
:105358007814002040787D0110B50321FF22C02079
:1053680001F076F81F4C102120608022C02001F047
:105378006FF8112120608022C02001F069F8122105
:1053880020608022C02001F063F813212060802271
:10539800C02001F05DF8142120608022C02001F0B7
:1053A80057F8152120608022C02001F051F8802292
:1053B80020601621C02001F04BF82060C020172182
:1053C800802201F045F82060074CC020227AB721DE
:1053D80001F03EF80023237463612376E36101231F
:1053E800237010BD684000207814002038B5C02014
:1053F8000321FF2201F02CF80B4D00242B19615DCD
:105408005A78C020023401F023F8C82CF6D1B12113
:10541800AC22C02001F01CF8C0200321002201F0BA
:1054280017F8002038BD00BF435504082DE9F3479D
:1054380006460F4692461D461AB90C1FE4019146CE
:1054480035E005EE902A06EE903AB8EE657AF8EE69
:10545800667AFC01C7EE277AA4F500749FED5C7AA2
:1054680067EE877A17EE900A09F0F2F941EC100B13
:105478000BF0DEF959EC108B4946404609F0FEFC6A
:1054880024184FEACA1009F0C1F9CDE900012846ED
:1054980009F0BCF94B46424609F02EFA02460B4683
:1054A800DDE9000109F074F809F0E8FC8146002EF6
:1054B80014BF4FF022084FF01A08C5F307224146DF
:1054C800C02000F0C5FF08F10101EAB2C02000F0D9
:1054D800BFFFC4F3014208F10201C02000F0B8FF89
:1054E800C4F3072208F10301C02000F0B1FFE2B2C3
:1054F80008F10401C02000F0ABFFC9F3034305F431
:10550800702243EA123208F10501C02000F0A0FF22
:1055180008F10601C9F30722C02000F099FF08F13D
:1055280007015FFA89F2C02000F092FFC020B12184
:10553800A02200F08DFF07EE107A264CF8EEC77A0D
:105548000EBBD4ED015A06EE90AAB8EE657A05EEC8
:10555800905AB8EE666AF8EE656A0123C6EE266AC6
:10556800237477EEA67A67EE277A17EE900A09F089
:105578006FF941EC100B0BF05BF951EC100B09F0D3
:105588007DFC606120E005EE90AAD4ED016AB8EEDA
:10559800656A05EE905AB8EE667AF8EE656A0123F8
:1055A800C6EE266A237677EEA67A67EE277A17EE96
:1055B800900A09F04DF941EC100B0BF039F951EC58
:1055C800100B09F05BFCE0610020BDE8FC8700BF20
:1055D80000000043781400200022012326E7012858
:1055E80038B50D4604D002280CBF3C242C2400E01A
:1055F80034242146C02001F027F805F0070200F006
:105608000F0040EA02122146C020BDE8384000F0F1
:105618001FBF2DE9F3470A9C1D4607468A461646D2
:10562800524B01E06D0864089C42FBD82DB906F185
:105638000076043EF601A94634E006EE905AB8EE2C
:10564800667A06EE904AF8EE667AF601C7EE277A91
:10565800A6F500769FED467A67EE877A17EE900AF0
:1056680009F0F6F841EC100B0BF0E2F859EC108B4E
:105678004946404609F002FC3618E80109F0C6F828
:10568800CDE90001204609F0C1F84B46424609F031
:1056980033F902460B46DDE9000108F079FF09F00D
:1056A800EDFB8146022F9BBF324BDB194FF0000800
:1056B80093F8C880C4F307224146C02000F0C8FE12
:1056C80008F10101E2B2C9B2C02000F0C1FE08F140
:1056D8000201C9B2C6F30142C02000F0B9FE08F1C8
:1056E8000301C9B2C6F30722C02000F0B1FE08F1D9
:1056F8000401C9B2F2B2C02000F0AAFE04F470247A
:10570800C9F3034308F1050143EA1432C9B2C020C2
:1057180000F09EFE08F10601C9B2C9F30722C020B5
:1057280008F1070800F094FE5FFA89F25FFA88F141
:10573800C02000F08DFEBAF1010F0CBF2F220F22FE
:105748000DB942F04002012F06D002D3022F0AD130
:1057580005E0C020102104E0C020112101E0C02094
:10576800122100F075FE0020BDE8FC87FFFF0F0046
:10577800000000434355040807B5012300930023A4
:10578800FFF747FF0EBD00280CBFFF22002208B517
:10579800C020032100F05CFE002008BD08B5C02031
:1057A800B121AC2200F054FE002008BD704708B5B6
:1057B80000F050F900F050F9014B00221A7008BDB2
:1057C800E80B0020024B187880F00100704700BFFA
:1057D800E80B0020014B1878704700BFE80B002049
:1057E80008B54FF400710F4807F037F90E4BD0F1A8
:1057F80001005A7838BF0020824201460ED05A680C
:105808001D2A0DDC01321E2A5A6009D1587007483A
:1058180000225A60BDE8084003F04ABC00225A60E2
:1058280008BD00BF00080240E80B0020929F050851
:10583800014B5878704700BFE80B002010B50021D5
:1058480004460122302000F003FEC0B9012001F017
:10585800A1F8002CB8BF4034E4B210212246302011
:1058680000F0F6FD012001F095F8302011212246C4
:1058780000F0EEFD0120BDE8104001F08BB810BD2E
:1058880010B5002104460122302000F0E1FDC0B926
:10589800012001F07FF8002CB8BF4034E4B2122197
:1058A8002246302000F0D4FD012001F073F83020AA
:1058B8001321224600F0CCFD0120BDE8104001F084
:1058C80069B810BD002810B5044603DB5F2CA8BFDB
:1058D8005F2400E0002430200021012200F0B8FD00
:1058E800A8B90120E4B201F055F83B212246302046
:1058F80000F0AEFD012001F04DF830203C21224699
:1059080000F0A6FD0120BDE8104001F043B810BD2D
:10591800302810B504460ADC10F17F0F02DB00289E
:1059280002DB05E06FF07E0404F5807400E03024AB
:10593800002130200A4600F08BFDA8B90120E4B20E
:1059480001F028F841212246302000F081FD012095
:1059580001F020F830204221224600F079FD012094
:10596800BDE8104001F016B810BD282810B504464F
:1059780009DC10F1180F02DB002802DB04E06FF0ED
:1059880017047F3400E02824002130200A4600F064
:105998005FFDA8B90120E4B200F0FCFF53212246C4
:1059A800302000F055FD012000F0F4FF3020542194
:1059B800224600F04DFD0120BDE8104000F0EABF8E
:1059C80010BD08B530200021012200F041FD60B96A
:1059D800012000F0DFFF30203321402200F038FDA5
:1059E8000120BDE8084000F0D5BF08BD10B5302043
:1059F8000021012200F02CFD044660B9012000F0CE
:105A0800C9FF30203321224600F022FD0120BDE8E5
:105A1800104000F0BFBF10BD10B53020002101229A
:105A280000F016FD0446A0B9012000F0B3FF3421B0
:105A38002246302000F00CFD012000F0ABFF3020A2
:105A48003721224600F004FD0120BDE8104000F097
:105A5800A1BF10BD4020F1E6402011E708B50021A4
:105A68000122302000F0F4FC012000F093FF3020E8
:105A78003421024600F0ECFC012000F08BFF3020BE
:105A88003721024600F0E4FC0120BDE8084000F0A0
:105A980081BF08B500210122302000F0D9FC012087
:105AA80000F078FF302034210C2200F0D1FC0120D6
:105AB800BDE8084000F06EBF704770477047194B4B
:105AC8001949D3ED006A93ED017A00231A469FED38
:105AD800176A03E0F0EE476AB0EE677A505E05EEAB
:105AE800900AF8EEE57A0133C7EE867A9BB218B2CF
:105AF80004327F2877EEE67AECDD27EE077A07EEA8
:105B0800A77A0B49074A0B80BDEEC77A00231360BA
:105B18005360C2ED027A17EE102A064B92001A6003
:105B2800704700BFF00B0020302600200000FA4527
:105B3800603A0020041700202DE9F84F2E4B2F4A19
:105B480019682F4B19B92F4911602F4A02E02F49C4
:105B580011602F4A1A602F4BDFF8BCA0DFF8BC9009
:105B6800DFF8BCB000221A80244A9846176830E053
:105B780007EB84036500B3F9023007EE103AF8EE3C
:105B8800C77A013617EE900A08F062FE18A3D3E927
:105B9800002308F0B1FE09F049F929F815002AF8A0
:105BA800140037F9243007EE103AF8EEC77A0135B9
:105BB80017EE900A08F04CFE0DA3D3E9002308F075
:105BC8009BFE09F033F92BF8140029F81500A8F802
:105BD8000060B8F8006034B2FF2CC9DD00F05EF850
:105BE80000F06AF801F0C0F8BDE8F84F67E700BFB9
:105BF8009A9999999999E93FF8160020EC1600208E
:105C080028150020322E0020322A002032360020AB
:105C180032320020603A0020302200203026002056
:105C28003024002010B50B4C204606F004FB0A4B2C
:105C380018600A4806F0FFFA094B1860FFF77CFF66
:105C4800084B0949012220469A81BDE8104006F018
:105C580073BB00BF10600240F81600208860024045
:105C68000C170020F00B002020800010014B186852
:105C7800704700BF0417002008B5054B0548198870
:105C88000022012309F0C6FD034B187008BD00BFB0
:105C98007000002018220020341D00200348044909
:105CA800044A4FF4807309F02DBE00BF7400002031
:105CB800302200201620002003480449044A4FF4EB
:105CC800807309F01FBE00BF800000203024002030
:105CD8005018002038B505460C460135C1F3072198
:105CE80000F066FEA8B2E1B200F062FE00B238BD74
:105CF80038B5044600F070FD01340546A0B200F046
:105D08006BFDEDB2C0B240EA052000B238BD37B530
:105D18000B0E8DF804300B0C8DF805300B0A8DF83E
:105D280006308DF80710002400E0284601AB451C1A
:105D3800E15C013400F03CFE042CADB2F5D13EBD6F
:105D480037B5002400E02846451C00F045FD01ABAE
:105D5800ADB2E0540134042CF5D19DF805009DF84E
:105D68000430000440EA03609DF8073018439DF8AA
:105D7800063040EA03203EBD38B50446642000F0F2
:105D880009FE25786068AD00EDB2257006F06BFE5F
:105D9800237A40FA03F000F003000543104B257006
:105DA80005F00F055A5D6378D218D2B2D3B201322A
:105DB800D2B2022A637001D80022A2705BB2012B12
:105DC80003DD0123A3700023637094F901300133CC
:105DD80003DAFF23A3700023637094F9020038BD2F
:105DE80014560408F7B504200121234F07F07EF963
:105DF80002AD01214FF48040012407F0A7F90026E5
:105E08004FF4B0733846694645F8083D8DF804608C
:105E18008DF8074006F0C2FD1020214607F066F90C
:105E280078236946154800938DF804608DF807407B
:105E380006F0B4FD0420214607F058F921464FF436
:105E4800804007F083F91E233846694600938DF891
:105E580004608DF8074006F0A1FD0220214607F0F6
:105E680045F9B02306488DF8046069468DF8074067
:105E7800009306F093FDFEBD0008024000100240AA
:105E880000040240802108B5034806F0E6FDD0F181
:105E9800010038BF002008BD0004024008B54FF4D7
:105EA8008071044806F0D9FDD0F1010038BF002008
:105EB80008BD00BF0008024008B5FFF7E3FF08B1BE
:105EC800FFF7ECFFC0B208BD10B5642000F062FD1A
:105ED8000F48FFF751FF044610B90E4B187009E040
:105EE800FFF7DCFF30B9002C0A4B01DD012200E08E
:105EF800FF221A700848FFF73FFF0028074B01D11F
:105F0800187010BD01DD012200E0FF221A7010BDDB
:105F1800C000002090400020CC000020302A002043
:105F280007B50220012107F0E1F8012300938DF85D
:105F3800043002238DF805300448002369468DF8A3
:105F480006308DF8073006F029FD0EBD000402402A
:105F580010B5084C01210022204606F094FD40F2BD
:105F6800FF4000F017FD012120460A46BDE8104019
:105F780006F089BD0004024008B5FFF7E9FF0021DB
:105F88000A46302000F064FA012000F003FD0121E8
:105F98000A46302000F05CFA012000F0FBFC0021EA
:105FA8000122302000F054FA012000F0F3FC012116
:105FB8000822302000F04CFA012000F0EBFC02210E
:105FC8000122302000F044FA012000F0E3FC002117
:105FD8000A46302000F03CFA012000F0DBFC1B21CF
:105FE800CD22302000F034FA012000F0D3FC042147
:105FF8000322302000F02CFA012000F0CBFC06210F
:106008000822302000F024FA012000F0C3FC072108
:106018000A46302000F01CFA012000F0BBFC0821E1
:106028008022302000F014FA012000F0B3FC1E2179
:10603800B022302000F00CFA012000F0ABFC052162
:106048009122302000F004FA012000F0A3FC0D2179
:106058000322302000F0FCF9012000F09BFC0E2107
:106068000022302000F0F4F9012000F093FC142104
:106078008022302000F0ECF9012000F08BFC0B218D
:106088008822302000F0E4F9012000F083FC302061
:106098000C21822200F0DCF9012000F07BFC1221A7
:1060A8008822302000F0D4F9012000F073FC13217D
:1060B8008C22302000F0CCF9012000F06BFC00218C
:1060C8000122302000F0C4F9012000F063FC0C210B
:1060D8000822302000F0BCF9012000F05BFC0D2103
:1060E8000822302000F0B4F9012000F053FC0E2102
:1060F8000822302000F0ACF9012000F04BFC0F2101
:106108000822302000F0A4F9012000F043FC00210F
:106118000A46302000F09CF9012000F03BFC4021A9
:106128000222302000F094F9012000F033FC002214
:106138004121302000F08CF9012000F02BFC3020A8
:106148003F21D42200F084F9012000F023FC002133
:106158000122302000F07CF9012000F01BFC102106
:106168000F22302000F074F9012000F013FC1121F7
:106178000F22302000F06CF9012000F00BFC1221F6
:106188000022302000F064F9012000F003FC132104
:106198000022302000F05CF9012000F0FBFB09210F
:1061A8003C22302000F054F9012000F0F3FB0021DC
:1061B8000122302000F04CF9012000F0EBFB3020E8
:1061C8003421024600F044F9012000F0E3FB3020BE
:1061D8003721024600F03CF9012000F0DBFB3621B4
:1061E8000322302000F034F9012000F0D3FB3921DC
:1061F8000322302000F02CF9012000F0CBFB3B21DA
:106208003C22302000F024F9012000F0C3FB3C219F
:106218000A46302000F01CF9012000F0BBFB0021E9
:106228000A46302000F014F9012000F0B3FB512198
:10623800C022302000F00CF9012000F0ABFB302028
:106248005221002200F004F90120BDE8084000F0C6
:10625800A1BB00BF2DE9F04F454E464D93B001213B
:106268004FF4001006F042FF304605F0E5FE4FF00F
:10627800C0630293404B0393404B002404934FF4B4
:1062880000794FF400334FF480684FF400674FF4FF
:10629800005A4FF4807B304602A90C93019309976A
:1062A800CDF8189005940794CDF82080CDF828A053
:1062B800CDF82CB00D9405F04BFF224630463049FE
:1062C80005F0A1FF3046012105F0A7FF01210A468C
:1062D8004FF0402007F078F9284605F0ADFE294A2E
:1062E800019B0392284A0C9304922846402202A953
:1062F800059209970294CDF818900794CDF820805C
:10630800CDF828A0CDF82CB00D9405F021FF224639
:1063180028461E4905F077FF2846012105F07DFF34
:1063280042F2107701220221194807F04DF9384648
:1063380000F030FB3046012105F045FF01212846D9
:1063480005F041FF384600F025FB0B238DF844305B
:1063580011A801238DF845408DF846408DF8473047
:1063680002F02AFF384600F015FB13B0BDE8F08FA5
:1063780010600240886002400C4000403236002025
:10638800322E00200C3C004032320020322A0020FD
:10639800003C004002481021012205F08BBF00BFDD
:1063A8001060024013B50220012106F09FFE4FF451
:1063B80010730E4C009302238DF804308DF80530CD
:1063C80001238DF806302046002369468DF80730F2
:1063D80006F0E4FA20460621042206F05FFB204678
:1063E8000921042206F05AFB1CBD00BF000402402C
:1063F80030B5154D85B001214FF4001006F09AFE16
:10640800284606F061FB0023ADF804304BF6FF7315
:10641800ADF806303323ADF808304FF48063ADF89B
:106428000A304FF48043ADF80C3004AC074B2846D3
:10643800012144F8103D06F0E9FB2846694606F0BC
:1064480071FB05B030BD00BF00540040801A060043
:1064580073B54FF4961306460D461446019304E0AF
:10646800019B5A1E0192002B57D031484FF400313E
:1064780006F0E4FC0028F3D12D48012106F0D2FBF8
:106488004FF48053019304E0019B5A1E0192002BA4
:1064980045D02748274906F0BCFC0028F4D02448FA
:1064A8003146002206F0D6FB4FF48053019304E0F6
:1064B800019B5A1E0192002B33D01D481E4906F03D
:1064C800A8FC0028F4D01A48294606F046FC4FF4E8
:1064D8008053019303E0019B5A1E01921BB3144899
:1064E800164906F096FC0028F5D01148214606F01A
:1064F80034FC4FF49613019303E0019B5A1E01925A
:106508009BB10B480E4906F099FC0028F5D00848C5
:10651800012106F093FB002008E0012006E002209C
:1065280004E0032002E0042000E005207CBD00BF59
:1065380000540040010003008200070080000700AB
:1065480004000010F7B51F464FF4961306460D4693
:106558001446019304E0019B5A1E0192002B5ED061
:1065680034484FF4003106F069FC0028F3D1314873
:10657800012106F057FB4FF48053019304E0019B7F
:106588005A1E0192002B4CD02A482B4906F041FC98
:106598000028F4D027483146002206F05BFB4FF470
:1065A8008053019304E0019B5A1E0192002B3AD0BC
:1065B8002048224906F02DFC0028F4D01D48294621
:1065C80006F0CBFB4FF48053019304E0019B5A1E65
:1065D8000192002B29D01748194906F01AFC002807
:1065E800F4D000254FF4961610E0615D114806F0CE
:1065F800B4FB019603E0019B5A1E0192BBB10D4802
:10660800104906F01BFC0028F5D00135EBB2BB425F
:10661800EBD30848012106F011FB002008E0012017
:1066280006E0022004E0032002E0042000E0052048
:10663800FEBD00BF005400400100030082000700B7
:10664800800007000400001037B54FF49613044685
:106658000D46019305E0019B5A1E0192002B00F0A4
:106668009B8056484FF4003106F0E8FB0028F2D131
:106678005248012106F0D6FA4FF48053019305E001
:10668800019B5A1E0192002B00F088804B484C4910
:1066980006F0BFFB0028F3D048482146002206F048
:1066A800D9FA4FF48053019304E0019B5A1E0192DA
:1066B800002B75D04148434906F0ABFB0028F4D0C5
:1066C8003E48294606F049FB4FF48053019304E005
:1066D800019B5A1E0192002B64D038483A4906F0B3
:1066E800ADFB0028F4D03548012106F09BFA4FF4A1
:1066F8008053019304E0019B5A1E0192002B53D052
:106708002E482F4906F085FB0028F4D02B48214657
:10671800012206F09FFA4FF48053019304E0019B95
:106728005A1E0192002B41D0244C2849204606F0DD
:1067380085FB0028F3D02046002106F093FA204676
:106748000121238B06F07AFA4FF48053019304E079
:10675800019B5A1E0192002B2AD018481C4906F0AA
:106768006DFB0028F4D0154806F0F9FA4FF4805371
:106778000193124A03E0019B591E0191D3B113887A
:106788009B05F8D4012104460C4806F06BFA0B4827
:10679800104906F06DFB0EE001240CE002240AE02B
:1067A800032408E0042406E0052404E0062402E0AB
:1067B800072400E0082420463EBD00BF00540040E6
:1067C800010003008200070004000010020000100E
:1067D800400000100004001013B54FF4961304464F
:1067E800019305E0019B5A1E0192002B00F0B08036
:1067F80061484FF4003106F021FB0028F2D15E48D1
:10680800012106F00FFA4FF48053019305E0019B34
:106818005A1E0192002B00F09D805748574906F0F8
:10682800F8FA0028F3D05448A021002206F012FA02
:106838004FF48053019305E0019B5A1E0192002BEF
:1068480000F08A804C484E4906F0E3FA0028F3D05D
:10685800C4F30521484806F080FA4FF480530193A9
:1068680004E0019B5A1E0192002B77D0424845490B
:1068780006F0E4FA0028F4D0E1B23F4806F06DFAD9
:106888004FF48053019304E0019B5A1E0192002BA0
:1068980066D039483B4906F0D1FA0028F4D036488A
:1068A800012106F0BFF94FF48053019304E0019BE6
:1068B8005A1E0192002B55D02F48304906F0A9FAEC
:1068C8000028F4D02C48A121012206F0C3F94FF486
:1068D8008053019304E0019B5A1E0192002B43D080
:1068E800254C2949204606F0A9FA0028F3D020466D
:1068F800002106F0B7F920460121238B06F09EF906
:106908004FF48053019304E0019B5A1E0192002B1F
:106918002CD019481D4906F091FA0028F4D01648E1
:1069280006F01DFA4FF480530193134A03E0019BCC
:10693800591E0191E3B113889905F8D40121044641
:106948000D4806F08FF90C48114906F091FA10E04D
:1069580001240EE002240CE003240AE0042408E0E9
:10696800052406E0062404E0072402E0082400E0E9
:10697800092420461CBD00BF00540040010003004C
:106988008200070004000010020000104000001000
:106998000004001082B0002304E0019B013301933E
:1069A800009B01330093009B8342F6D302B07047EB
:1069B80037B54FF4805304460D46019304E0019B1C
:1069C8005A1E0192002B6ED03D484FF4003106F05C
:1069D80035FA0028F3D13A48012106F023F94FF49B
:1069E8008053019304E0019B5A1E0192002B5CD056
:1069F8003348344906F00DFA0028F4D03048A02175
:106A0800002206F027F94FF48053019304E0019B1C
:106A18005A1E0192002B4AD029482B4906F0F9F951
:106A28000028F4D0C4F30521254806F096F94FF460
:106A38008053019304E0019B5A1E0192002B38D029
:106A48001F48224906F0E5F90028F4D0E1B21C48B5
:106A580006F083F94FF48053019303E0019B5A1E1B
:106A6800019243B31648194906F0D3F90028F5D026
:106A78001348294606F071F94FF49613019303E081
:106A8800019B5A1E0192C3B10D48114906F0D6F96F
:106A98000028F5D00A48012106F0D0F80D48FFF784
:106AA80079FF00200AE0012008E0022006E0032028
:106AB80004E0042002E0052000E006203EBD00BFFF
:106AC8000054004001000300820007008000070016
:106AD80004000010A086010013B50520012106F06E
:106AE80005FB184C4FF4E053009302238DF8043053
:106AF8008DF805302046002369468DF806308DF85C
:106B0800073005F04BFF20460A21062205F0C6FF94
:106B180020460C21062205F0C1FF062220460B2143
:106B2800A4F5006405F0BAFF4FF400432046694617
:106B3800009305F033FF20460F21062205F0AEFF33
:106B48001CBD00BF000802401FB50446FFF7E8F966
:106B5800FFF74EFCFFF710FAFFF7BEFF01214FF4D5
:106B6800004006F0E7FA02940F4C1023ADF802300B
:106B7800204600236946ADF80430ADF80C30ADF876
:106B88000030ADF8063006F004FC69464FF04020AE
:106B980006F0D3FC2046012106F083FC4FF040208C
:106BA800012106F07EFC1FBD003C0040014B18602F
:106BB800704700BF0C0C0020704710B50A4A1379C3
:106BC800262B04D80949C8540133137110BD074A4C
:106BD8000123591ED45C0133272B5454F9D1034B9C
:106BE80083F8260010BD00BF0C0C0020343A0020AA
:106BF800704710B504462078FFF7DFFF14F8013F0F
:106C0800002BF8D110BD38B504460D46013D14F8E7
:106C1800010BEDB2FFF7D1FF002DF7D138BD00BF52
:106C2800014B1878704700BF140C0020014B5878AE
:106C3800704700BF140C0020024B187880F0010048
:106C4800704700BF140C0020024B00221A705A70C3
:106C5800704700BF140C0020014B01221A707047C6
:106C6800140C0020014B01225A707047140C0020AC
:106C780082B0002304E0019B01330193009B0133A0
:106C88000093009B8342F6D302B070470148024943
:106C980004F0ACBA983A00209840002007B50420C8
:106CA800012106F023FA01214FF4804006F04EFA44
:106CB8004FF40073009300238DF804300348012338
:106CC80069468DF8073005F069FE0EBD00080240E0
:106CD800034A044B1A60044A044B1A60704700BF09
:106CE8000000FA45B84A0020DB0FC93F904A00204F
:106CF800034B00221A60034A034B1A60E8E700BFFF
:106D0800444100200000FA450816002007EE100A4A
:106D1800024BF8EEC77AC3ED007A704708160020D8
:106D280038B510EE100A07F093FD0DA3D3E9002340
:106D380007F0E2FD084B044618680D4607F088FD89
:106D48000B4602462946204607F000FF08F0B6F831
:106D5800024B186038BD00BFB84A0020904A002096
:106D6800182D4454FB2119402DE9F04F2DED068BC9
:106D7800734CDFF800A289B00027A34637F80A5001
:106D8800704B2580FE5A704B6680186807F060FDCE
:106D980069A3D3E9002307F0AFFD08F047F863685B
:106DA8006A4AC018011101F580610905090D606082
:106DB800C0F30B100DF1200C32F8203032F82120EE
:106DC800616A238115FB02F0628115FB03F516FB4E
:106DD80002F216FB03F60CEB4103E0602561C0F3F9
:106DE800CF30C5F3CF356261A661C2F3CF32C6F3A7
:106DF800CF3623F8200C23F8105C23F8182C23F83E
:106E0800086C534BA08301310B40002BE58322848F
:106E1800668403DA013B63F003030133CBF82430C3
:106E2800002B7CD14B484C4A6946042309F02AF8C8
:106E38004A484B4A04A9042309F024F849484A4A15
:106E480002A9042309F01EF8484A494806A9042360
:106E580009F018F8B4F9283007EE903AB4F92A3056
:106E6800B8EEE79A07EE903AB4F92C30B8EEE78A14
:106E780007EE903AB4F92E30F8EEE79A07EE903A1A
:106E8800F8EEE78A68EE087A49EE097A17EE900A72
:106E980007F0DEFC41EC100B09F056FE51EC100B2C
:106EA80008F00CF868EEA87A49EEA97A0AEE100AFA
:106EB800206317EE900A07F0CBFC41EC100B09F0A9
:106EC80043FE51EC100B07F0F9FF68EE897A58EE93
:106ED800297A28EE288A0AEE900A606309EE298A40
:106EE80017EE900A07F0B4FC804618EE100A89469F
:106EF80007F0AEFC49EC108B41EC110B09F09CFD3E
:106F080051EC100B07F0DAFF8AEE2A0AA06384ED31
:106F18000F0A01F007FC94ED0E0A01F013FC02378A
:106F2800B7F5007F7FF42AAF09B0BDEC068BBDE84A
:106F3800F08F00BFAFF3008039D6C56D305FC44015
:106F4800180C002050180020904A002030560408E1
:106F580003000080B4000020400C0020A80000209E
:106F6800420C00209C000020440C0020460C00200D
:106F78009000002016200020014B93ED0F0A704767
:106F8800180C0020014B93ED0E0A7047180C0020D6
:106F9800014B93ED0C0A7047180C0020014B93ED40
:106FA8000D0A7047180C002010B5FEF7D5F900201F
:106FB800012324210246FEF739FA114B1C780020E0
:106FC800012C05D10146FEF70AFB2046002104E00A
:106FD8000721FEF704FB01200721FEF700FB6322CF
:106FE8001221C020FFF734FA02200121FEF7F7FA38
:106FF800FEF7D4FB0120BDE81040FEF7C4BB00BF7C
:10700800080D00200D4B1B78012B05D10C4B0D4AA8
:10701800196812688A181A600B4B1B78012B084BE9
:10702800196805D1094A914207DD01321A60704793
:10703800074A914201DD01321A607047943A0020F4
:1070480094400020903A0020080D00207FD1F008DD
:10705800FF1FA1070E4B1B78012B05D10D4B0E4AC4
:10706800196812688A1A1A600C4B1B78012B094B95
:1070780005D10B4A1968914208DC1A6070471A68F2
:10708800B2F57A2FDCBF4FF47A221A60704700BF3E
:10709800943A002094400020903A0020080D0020E7
:1070A80040420F00024B1A68024B1A60704700BF3B
:1070B80080400020944000202DE9F04F8246584837
:1070C8008BB0B0FBF1F00C4607F0A0FB41EC100BC5
:1070D80009F0AEFB51EC100B07F0D0FEC3070746D2
:1070E80048BF471E04FB07F007F090FB46A3D3E90F
:1070F800002307F02BFD04460D4645EC104B09F024
:1071080097FB59EC108B204642464B46294607F020
:107118003FFACDE904014946404607F0AFFE3CA3DB
:10712800D3E900230990DDE9040107F061FE002896
:107138003DD1002401234FF01509224698462046E8
:10714800DFF8E4B003E0234642462C46B04600FB95
:1071580004355D452ED800FB0826DDE904012EA381
:10716800D3E9002307F044FE30BBDDE90423002007
:107178002C4907F0EBFC41EC100B0390029109F04D
:1071880057FB0398029953EC102B8DED060B07F073
:10719800FFF909F1FF39CDE904015FFA89F9DDE961
:1071A800060107F06BFEB9F1000FCCD104E0012510
:1071B800002601E025464646099BD9B2BAF1000FE0
:1071C8000BD132462B465046FEF730F90123009387
:1071D800504651463A46534609E032462B4601206E
:1071E800FEF724F90120009001463A460023FEF7F5
:1071F80010FAFEF7D3FA01200BB0BDE8F04FFEF706
:10720800C2BA00BFAFF300800000000084D7774106
:10721800956479E17FFDA53DBBBDD7D9DF7CDB3D1A
:1072280000E9A4350000F03FFFFF0F001F4B1B785B
:10723800022B10B539D01E4B1E4A19681E4B1F4C25
:107248001B68CB189342236018DC0020FFF734FF3B
:1072580001202168FFF730FF194B1C780020012C12
:1072680005D10146FEF7BBF92046002104E00721BD
:10727800FEF7B5F901200721FEF7B1F9114B1B788C
:10728800022B12D10A4C104B22681B689A420CDA66
:107298000E4B1B78012B08D10D4B186800F070F8C5
:1072A8000C4B22681B68D318236010BD684D002062
:1072B8009440002080D1F008304100203441002063
:1072C800080D0020943A0020704000206C400020F7
:1072D8004C400020903A002008B5FEF7D3FD094B3A
:1072E8005A78187002435A701AB19A7801329A7013
:1072F80030B99B78034A012B02D90023537093704D
:1073080008BD00BF580C002007B50420012105F076
:10731800EDFE4FF46043009301238DF804300223FF
:107328008DF805300448002369468DF806308DF83D
:10733800073005F033FB0EBD00080240084B1A6801
:107348004FF47A73B2FBF3F2064B013A5A60064ADD
:10735800F02182F8231000229A6007221A607047F1
:10736800A401002010E000E000ED00E0034B5A68A3
:1073780012B15A68013A5A60704700BF580C002091
:10738800024B58605A68002AFCD17047580C0020FC
:1073980030B585B004460D4601A85C490A220BF0B9
:1073A80063FE5B4B1B78032B10D8DFE803F0020564
:1073B800080B01A8574907E001A8574904E001A8AC
:1073C800564901E0564901A80BF038FF04AA1319E1
:1073D80013F80C3C5D19EDB22F2D01D80A3502E0E7
:1073E800392D01D90A3DEDB204AB1C194FF6FF70D7
:1073F80004F80C5CFCF71AFF0020FDF70DF80DF1FE
:1074080003050F24204623345A21002315F8012FA1
:10741800A4B2FDF71BF8B4F5A57FF3D164205A2177
:107428002C220023FDF712F80023CD205A212C220C
:10743800FDF70CF80020FCF7F9FE354B1B78032B01
:1074480062D8DFE803F002284B5601A931480BF057
:10745800F5FE0A2200212F480CF094F8314A324BED
:1074680012781860012A06D1304A904201DC0132B4
:107478001A602F4A06E0B0F5FA5FBCBF4FF4FA5223
:107488001A602C4A1B689342C4BF274B1A602A4BC8
:107498001A682A4B20E001A91F480BF0CFFE0A22E8
:1074A80000211D480CF06EF81E4A254B1278186012
:1074B800012A06D11D4A904201DC01321A601C4A99
:1074C80006E0B0F5FA5FBCBF4FF4FA521A60194AE9
:1074D8001B68934218DD1A4B1A6015E001A90F4882
:1074E8000BF0ACFE0D4800210A220CF04BF8154BAE
:1074F80009E001A90A480BF0A1FE094800210A2267
:107508000CF040F8104B186005B030BD47A00508D6
:107518007E4000205A400020744000201C4100207A
:1075280050400020080D0020884000203F420F00F6
:1075380080D1F00840420F00804000209440002095
:10754800384100208C4000204C40002010B50D4BE5
:107558000D4C1A680D4821460BF048FE0C4B0D489F
:107568001A6821460BF042FE0B4B0C481A6821465C
:107578000BF03CFE0A4B0B481A682146BDE8104048
:107588000BF034BE8840002051A005085A40002066
:1075980038410020744000208C4000201C4100200D
:1075A8004C4000205040002008B500210A220D4818
:1075B8000BF0E8FF0C4B002118600A220B480BF077
:1075C800E1FF0B4B002118600A220A480BF0DAFF92
:1075D800094B002118600A2208480BF0D3FF084B1A
:1075E800186008BD5A4000208840002074400020E0
:1075F800384100201C4100208C40002050400020D1
:107608004C400020014B93ED020A7047580C0020B3
:10761800014B93ED030A7047580C0020014B93ED82
:10762800040A7047580C0020034B83ED000AC3ED91
:10763800010A83ED021A7047DC5E0020014B1860D6
:10764800704700BF94400020014B1868704700BF86
:1076580088400020014B1868704700BF384100205F
:1076680008B54FF49570FEF743FB40F26523C31A43
:10767800584240EB030008BD08B5C620FEF738FBAA
:1076880040F28D13C21A504240EB020008BD4FF47D
:10769800957040F26521FEF71DBBC62040F28D11A2
:1076A800FEF718BB08B5F9F747F9BCEEC00A4FF466
:1076B800967010EE101AFEF72AFBF9F743F9014607
:1076C8004FF49870FEF723FBF9F742F9BCEEC00AB5
:1076D8004FF49A7010EE101ABDE80840FEF717BB79
:1076E80038B5FFF7BDFFC0B14FF49670FEF728FB21
:1076F800124D134C28604FF49870FEF721FB206060
:107708004FF49A70FEF71CFB0E4B2A6818600E4B5C
:107718005A612268D8619A6106E00B4B0B4A5A619C
:107728000B4A9A610B4ADA61074A0B4B9069D16997
:10773800526958601A60996038BD00BF140D002066
:10774800100D00200C0D0020580C0020E17A843F19
:1077580014AE3740CCBC8C2CDC5E002060EEA00A56
:10776800B7EE007AF0EE606A70EE077A40EE006AD3
:1077780047EEA70A36EEC77A08B5C7EE200A10EE1C
:10778800900A07F065F80022084B07F0B5F80022C8
:10779800074B06F0FFFE07F091FB07EE900AFDEE9F
:1077A800E77A17EE900A9F3008BD00BF00005940E5
:1077B8000000E03F38B52DED028BF7EE008AB0EE01
:1077C800608A70EE288A10EE900A28EE088A07F080
:1077D8003FF808EEA88A00220F4B07F08DF8044600
:1077E80018EE100A0D4607F033F802460B462046FD
:1077F800294607F0ABF90022084B06F0CBFE07F04C
:107808005DFB07EE900AFDEEE77A17EE900A7730F7
:10781800BDEC028B38BD00BF000069400000E03FAE
:10782800F0B5694D2DED068B95E80F008DB008AECB
:10783800103586E80F000FCD01AC0FC495E807009E
:107848004FF6FF7384E807009F2077216422FAF738
:107858007CFBA020772164224FF6FF73FAF775FBB3
:107868009E20772164224FF6FF73FAF76EFB9F2064
:10787800762164224FF6FF73FAF767FB4FF6FF7322
:10788800782164229F20FAF760FB0020FCF72AFB8E
:107898009F2077216522FCF7FFFC9F207721642237
:1078A800FCF7FAFC07AD0C36F7EE009A0435F7EE54
:1078B800008A95ED009A4FF49674B0EE68AA18EE17
:1078C800900A06F0C5FF3EA3D3E9002307F014F899
:1078D80007F0F4FA08EE900A38EEE98AB0EE490AA1
:1078E800F0EE480AFFF73AFFB0EE490AF0EE480A10
:1078F8000746FFF75FFFBFB281B20F223846FCF799
:10790800FEF9013CDBD14FF49674F7EE008A18EECD
:10791800900A06F09DFF2AA3D3E9002306F0ECFFA6
:1079280007F0CCFA08EE900A39EEE88AB0EE490A78
:10793800F0EE480AFFF712FFB0EE490AF0EE480AE7
:107948000746FFF737FFBFB281B20F223846FCF770
:10795800D6F9013CDBD1B542A8D16C4607AE043458
:1079680094ED009A4FF4C875F7EE008A18EE900A65
:1079780006F06EFF12A3D3E9002306F0BDFF07F05F
:107988009DFA08EE900A38EECA8AF0EE490AB0EE7F
:10799800480AFFF7E3FEB0EE480AF0EE490A074648
:1079A800FFF708FFBFB281B200223846FCF7A7F9FB
:1079B800013DDBD1B442D2D10DB0BDEC068BF0BD98
:1079C800295C8FC2F528F03F30960408121A06EE9B
:1079D800902A081AB8EEE67A06EE900AF8EEE67AE9
:1079E800C7EE277A9FED047A67EE877AFDEEE77A8D
:1079F80017EE900A704700BF0000A0438A1A06EEEF
:107A0800902A081AB8EEE67A06EE900AF8EEE67AB8
:107A1800C7EE277A9FED047A67EE877AFDEEE77A5C
:107A280017EE900A704700BF0000484370B506463D
:107A38000D460024610704D5A0B231462A46FCF75A
:107A48005EF90134B4F5A07FF4D170BD70B5064677
:107A58000D460024600704D5A1B230462A46FCF73B
:107A68004EF90134C82CF5D170BD114B11481B7863
:107A78001149124A0068012B114B09D1126808609C
:107A88001A60104B1A68104B1A60104B1A680CE0F9
:107A98001268D2011A600B4B1A680B4BD2011A609C
:107AA8000A4B1A68C0010860D201094B1A60704776
:107AB800080D002088400020804000203841002028
:107AC800704000208C400020903A00206440002044
:107AD80030410020024B1A68024B1A60704700BF01
:107AE800804000209440002008B5FFF7BEFFBDE8A5
:107AF8000840EFE70022F0B51346202603254FF093
:107B08002C0C00E02646303EF6B217460132092E0C
:107B180010F8014B0AD897FBF5F605FB16772FB935
:107B2800CE1801F803C07470023301E0CC5401335D
:107B3800092AE7D12022CA54CB1848225A707A223F
:107B48009A700022DA70F0BD70B58CB005460C460C
:107B580008A80E491E460BF049FB08A86946FFF71E
:107B6800C9FF6A460A4904A80BF040FBBDF840006B
:107B7800FCF75CFB3046FCF76FFB2846214604AA5D
:107B88000023FCF781FC0CB070BD00BF57A00508AE
:107B9800189E05082DE9F047084B2DED0A8B1B7838
:107BA800022BC4B000F01085054B1A78054B5AB962
:107BB8001A68802392FBF3FA08E000BF684D0020A2
:107BC800080D002094400020D3F800A0FFF7D4F956
:107BD800CD4C84ED080AFFF7D5F994ED0A8AD4ED67
:107BE800088A38EE088AF0EE087A38EE288A84ED9A
:107BF800090A88EE278AE06A10EE105A84ED028A94
:107C080084ED0A8A06F024FE02460B4606F0C2FC02
:107C1800064628460F4606F01BFE02460B4630462F
:107C2800394606F0B7FC0022B84B06F08FFF07F084
:107C380045F9B74BB74A9D68E060D3ED007A67EE27
:107C4800A88AC2ED007AD3ED017AB34BE062C4EDA5
:107C5800088A1B78DFEDB18AC2ED017A77EEA88A2F
:107C680013B984ED088A6062206A06F0F1FD0646C1
:107C7800606A0F4606F0ECFD41EC100B41EC190B65
:107C880008F07EFD59EC108BB0EE490AF0EE690A57
:107C980008F076FE304653EC102B394606F02CFEE1
:107CA80007F00CF942464B4608EE100A39463046B2
:107CB80006F022FE07F002F99FED997AC8EE878A4E
:107CC80009EE900A79EEE89A68EE087A49EEA97A00
:107CD800B1EE488A67EE877A9FED92BA88EE278AD6
:107CE800C9EEA79A84ED048A18EE100A06F0B0FDD2
:107CF800CDE90601504606F099FD7FA3D3E900239C
:107D080006F0FAFD064628460F4606F0A1FD024693
:107D18000B463046394606F0EFFD02460B46DDE9D4
:107D2800060106F035FC07F0C9F80AEE100A29EE3C
:107D3800A98A6AEE0ACAB1EE4A9A78EE2C7ADFED81
:107D48007ABA89EE279A794BC9EEA7AAB4EE4B9A6C
:107D5800F1EE10FAC8BFB0EE4B9AB4EE6B9AF1EEA2
:107D680010FA48BFB0EE6B9AC3ED00AA83ED019AF2
:107D78001AEE900A06F06CFD00226D4BCDE9020167
:107D880006F006FC69EE097A044617EE900A0D46DD
:107D980006F05EFD224606460F462B46204629463B
:107DA80006F0AAFD32463B4606F0F4FB41EC100B08
:107DB80008F0CAFE0022DDE902015D4B59EC108B88
:107DC80006F0E8FB02460B4606F096FD32463B46B7
:107DD80006F0E0FB41EC100B08F0B6FE40464946C1
:107DE80055EC104B07F06AF8294608EE900A204631
:107DF80007F064F807EE900AC8EEA78A4D4D4E4C7E
:107E0800B7EE00CA18EE900A06F022FD3CA3D3E9AB
:107E1800002306F0E3FFDFED497A002818BFF0EEF3
:107E2800678AF4EE4C8ADFED467AF1EE10FAC8BFA5
:107E3800F0EE678ADFED437A6AEE277AC5ED008AAD
:107E480017EE900A06F004FDDFED3F7A37EEC88A98
:107E5800064678EE6CCA0F46C4E902671CEE900A23
:107E680006F0F6FC47EC106B41EC110BC4E900017D
:107E780008F0E2FD38EE8C8A3CEE68CA51EC100B33
:107E880088EE0C8A07F01AF8304B1B7880F000480F
:107E9800B4EE4B8AF1EE10FAC8BFB0EE4B8AB4EEDE
:107EA8006B8AF1EE10FA48BFB0EE6B8A022BC5F868
:107EB800048067D1264F3E68002E63DB254B264D94
:107EC800C3F800A0B400621C5B6825F814A018EE83
:107ED800900A25F8123006F0BBFC00221F4B06F072
:107EE8000BFD06F0CBFF04F10209013625F8190055
:107EF800404606F0ADFC33E01F85EB51B81E194033
:107F08002D431CEBE2361A3F580C002000000840B5
:107F1800DC5E00209C0100202C41002000008C42E7
:107F28000000F042003C1C46003C1CC6604D00208E
:107F3800000049404C4C0020184F002017B7D1389A
:107F480072F97F3F0AD7233D17B7D139943A0020F9
:107F580084400020544D00202C4F00200000F040A9
:107F680099A3D3E9002306F0C7FC06F05FFF0334AA
:107F7800B6F5FA7FC8BF4FF0FF3325F814003E600E
:107F8800C8BF3B60FFF704F87D4C84ED0C0AFFF78F
:107F980005F884ED0D0AFDF769FE5246A06379499C
:107FA80034A80BF023F9206B06F052FC02460B466E
:107FB80024A875490BF01AF9606B06F049FC0246D3
:107FC8000B4628A871490BF011F919EE900A06F032
:107FD8003FFCCDE90401DDE904236D492CA80BF031
:107FE80005F96C49DDE9062330A80BF0FFF8DDE957
:107FF8000223694910A80BF0F9F819EE100A06F0E7
:1080080027FCCDE90A01DDE90A23644914A80BF02D
:10801800EDF818EE900A06F01BFCCDE90801DDE941
:1080280008235F4918A80BF0E1F8404606F010FC59
:1080380006460F4632463B465A491CA80BF0D6F86E
:1080480018EE100A06F004FC804689464B4656494D
:10805800424620A80BF0CAF80CA85449A26B0BF0B2
:10806800C5F8534B1B78013BDBB2012B00F29E8213
:10807800504B1B78072B00F29982DFE813F00800B9
:108088009702A90030017301CD0167022D02022079
:10809800FCF7C2F94FF6FF70FCF7DEF81F20FCF77B
:1080A800C5F819210023444A2D20FCF7EDF94FF6B5
:1080B800FF70FCF7D1F800200024FCF7B7F80F2078
:1080C800B42152464FF6FF730094FFF73DFD0F2091
:1080D800772124AA2346FCF7D7F9A0200DEB00024C
:1080E80077212346FCF7D0F90F20412118AA23460F
:1080F800FCF7CAF9A02041211CAA2346FCF7C4F9C1
:108108000F2065212CAA2346FCF7BEF930AA234686
:10811800A0206521FCF7B8F90F20532110AA2346A7
:10812800FCF7B2F9A020532114AA2346FCF7ACF9B6
:108138000F209B2120AA2346FCF7A6F9104B9B6B26
:10814800B3F57A7FCCBF4FF4FC604FF47840FCF76E
:1081580083F80CAAA0209B210023FCF795F9174B64
:108168001B780221012B0CBF154A164A4FF48C705C
:108178000023FCF789F91F20FCF76EF816E200BF10
:10818800580C00205CA0050866A0050871A0050829
:108198007CA0050886A0050890A005089BA00508F6
:1081A800A6A00508B1A00508BCA00508C8A0050838
:1081B800943A00202C410020D5A00508080D002085
:1081C800F4A00508F8A00508CDCCCCCC0C5FC440C1
:1081D800DDE904233EA8B2490BF008F8DDE90623DF
:1081E80041A8B0490BF002F8DDE9022338A8AE49EE
:1081F8000AF0FCFFDDE90A233BA8AC490AF0F6FFC8
:10820800E62002213EAA0023FCF73EF9E6201621CB
:1082180041AA0023FCF738F90220C82138AA002314
:10822800FCF732F93BAA00230220DC21FCF72CF9E9
:10823800DFED9F7A68EEA78A4FF6E07518EE900A90
:1082480006F006FB47EC106BCDE9020108F098FA3E
:1082580059EC108B47EC106B08F092FB002057ECA0
:10826800106BFBF7F9FF0A21524600230520009501
:10827800FFF76AFC4FF47840FBF7D8FFDDE902010D
:1082880042464B4606F038FB77A3D3E9002306F0B5
:1082980081F906F0CBFD324684B23B46DDE90201A6
:1082A80006F02AFB02460B4671A1D1E9000106F04F
:1082B8006FF906F0BBFD81B22046F9F776FE9D20E6
:1082C800772105220023FBF7E1FF9F207521052276
:1082D8000123FBF7DBFF2846FBF7A8FF66E1754B98
:1082E8001868754B52461968FFF770FBB0F59F7F09
:1082F800044602DD714B02221A709FED718AF4EE7A
:10830800C8AAF1EE10FA14D5F5EEC0AAF1EE10FAEB
:108318000FDDFDEEEAAA4FF4FA711AEE902A00205A
:10832800FFF76CFBA3B281B24FF6FF721846FBF75A
:10833800E6FCB4EEC89AF1EE10FA40F13781DFEDB1
:10834800617AB4EEE79AF1EE10FA40F32F81BDEEB0
:10835800C99A5D4819EE102A4FF4FA71FFF74EFBDF
:10836800A4B2EEE0534B1868534B52461968FFF716
:108378002DFBB0F59F7F064602DD504B02221A7096
:10838800F5EEC09AF1EE10FA1DDDDDE904013AA31D
:10839800D3E9002306F022FDA8B139A3D3E90023CD
:1083A800DDE9040106F0A8FA02460B460020474919
:1083B80006F0EEF806F03AFDB4B281B24FF6FF725D
:1083C8002046FBF79CFC1AEE100A06F041FA2EA391
:1083D800D3E9002304460D4606F01EFD002800F0F0
:1083E800E5802046294624A3D3E9002306F0F6FCBD
:1083F800002800F0DB8026A3D3E900232046294685
:1084080006F07AFA0022324B06F0C4F806F00EFDA8
:10841800B6B281B2304696E0DDE908011EA3D3E981
:10842800002306F0F9FC002800F0C080214B1868F2
:10843800214B52461968FFF7C9FAB0F59F7F0446E9
:1084480002DD1E4B02221A709DED080B08F0F6FAA9
:1084580053EC102B1046194600221E4BA4B206F00E
:108468004BFA9BE0AFF300800000000000E063409F
:108478000000000000C05D409A9999999999B93F08
:108488000000000000409F409A9999999999B9BFB6
:108498000000000000408F4076711B0DE02DA03FCA
:1084A800FCA0050806A1050810A105081AA10508E1
:1084B8000000C8428840002038410020684D002054
:1084C8000000FA430000FAC30CFEFFFF00006940F9
:1084D80000005940000054C047A3D3E900233046A8
:1084E800394606F009FA46A3D3E9002306F02EFB25
:1084F80006F0E4FC384B08EE100A1868374B524671
:108508001968FFF763FAB0F59F7F02DD344B02224A
:108518001A70DFED347A48EEE77A84B2FDEEE77A36
:10852800204617EE901A4FF6FF7289B2FBF7E7FB69
:10853800BDEEC88A6FF0B30018EE102AB421FFF719
:108548005DFA81B220464FF4FC622DE0DFED267A19
:10855800B4EEE78AF1EE10FA28D51F4B18681F4BC6
:1085680052461968FFF732FAB0F59F7F044602DDDC
:108578001B4B02221A7049EC108B08F05FFA53EC7F
:10858800102B104619460022184B06F0B5F9024682
:108598000B4600201649A4B205F0FAFF06F046FC87
:1085A8004FF6FF7281B22046FBF7A9FB114B1B78EF
:1085B800022B09D043B14FF6FF7300930520DC214D
:1085C80052460023FFF7C0FA44B0BDEC0A8BBDE861
:1085D800F08700BFAFF300808840002038410020BA
:1085E800684D0020000048430000C8420000594080
:1085F800000069402C410020000000000080764007
:108608001F85EB51B81E194073B50646002847D0A0
:10861800244B18888619B6B232B2002A05DB40F21C
:108628003F139A42C8BF1E4600E000260121FBF70F
:10863800C5FA0120FBF716F91B4D0024605B0234D4
:10864800FBF75EF9B4F5C67FF8D14FF6FF75B0B207
:10865800C72201212B46FBF7C7FC124B1E80134B88
:108668001C68134B36B21B6806EE906A1B1BB8EEEB
:10867800E67A06EE903AF8EEE67A67EE277A17EE93
:10868800900A06F0E5F800220A4B06F05FFA06F0B9
:10869800CDFBDC212218002305200095FFF754FAB2
:1086A8007CBD00BF404C00206A4D0020884000205F
:1086B800384100200000744013B50F4CA38FADF86B
:1086C8000630BDF806309BB253B1BDF806004FF630
:1086D800FF7380B20121C722FBF786FC0023A38722
:1086E800064B1B78022B06D1054C94F90000FFF7C6
:1086F8008BFF002323701CBD580C0020684D002000
:10870800302A002038B54FF47A7441F28835204673
:10871800FEF762F80134C0B2A4B200F07DF9AC42B1
:10872800F5D138BD054B06491A6801EB82010132C3
:1087380002F01F0281ED000A1A607047484C0020C1
:10874800D44C0020054B06491A6801EB820101321E
:1087580002F01F0281ED000A1A607047E85E0020EF
:10876800584C0020094A0A4913680968994209D0F7
:10877800084901EB8301013303F01F0391ED000A5F
:10878800136070479FED040A704700BF544C0020E7
:10879800484C0020D44C002000000000094A0A4937
:1087A80013680968994209D0084901EB830101332C
:1087B80003F01F0391ED000A136070479FED040A50
:1087C800704700BF104F0020E85E0020584C002082
:1087D80000000000024A00231360024A1360704739
:1087E800544C0020484C0020024A00231360024ADF
:1087F80013607047104F0020E85E002008B5002184
:10880800C620FDF767FA4FF495700021BDE80840CF
:10881800FDF760BAAFF3008070477047FEE7FEE7E8
:10882800FEE7704770477047FEF7A0BD08B5022005
:1088380003F002FE48B1054BD3F880305B699847D6
:108848000220BDE8084003F005BE08BD984000209E
:1088580000F062BA014802F0DBBA00BF983A002083
:10886800704700BF414BD3F8882042F47002C3F828
:1088780088203F4B1A6842F001021A6000229A6071
:10888800196821F0847121F48031196039495960DF
:10889800196882B021F480211960DA60009201928F
:1088A8001A6842F480321A601A6802F4003201929F
:1088B800009A01320092019A1AB9009AB2F5A06F93
:1088C800F2D12B4B1B6813F4003318BF012301931B
:1088D800019B012B2ED1264B1A6C42F080521A6450
:1088E800254A116841F4804111609A689A609A6833
:1088F80042F400429A609A6842F4A0529A601F4A71
:108908005A601A6842F080721A601968184A890118
:10891800FBD51B4B40F205611960936823F00303F4
:108928009360936843F002039360936803F00C0329
:10893800082BFAD10E4B9A6822F400029A60114A69
:10894800C3F884201A6842F080621A601A6812011B
:10895800FCD5064B4FF000629A60D3F8882042F4A9
:108968007002C3F8882002B0704700BF00ED00E035
:1089780000380240103000240070004008544007BE
:10898800003C024080400030184B194A996801F0B9
:108998000C01042903D0082903D0164B19E0164B03
:1089A80017E059685A6811F4800F596814BF124BC0
:1089B800104B02F03F02B3FBF2F30C4A5268C2F3C9
:1089C8000142C1F38811013252004B43B3FBF2F369
:1089D800074A1360054B9A68054BC2F303129A18AD
:1089E8001968127921FA02F21A60704700380240B9
:1089F800A40100200024F40000127A0008B54020E9
:108A080003F01AFD30B1FBF79DFE4020BDE8084099
:108A180003F020BD08BD0000014608B5044805F074
:108A2800D5FC0348402105F07EFD0028F9D008BD9B
:108A380000440040F0B589B04FF4E13301200193C0
:108A480000232B4CADF808301E460146ADF80A301D
:108A5800ADF80C30ADF810300C23ADF80E3004F042
:108A680045FB4FF40030012104F064FB206802212B
:108A7800072204F013F807226068032104F00EF8B7
:108A88000125022704232068059305A98DF81A609B
:108A98008DF81B508DF818708DF8197003F07EFF53
:108AA80008236068059305A98DF8187003F076FF10
:108AB800A06801A905F0E0FB2A4640F225510D48BF
:108AC80005F018FD262307A88DF81C308DF81D60C9
:108AD8008DF81E608DF81F5000F06EFBA0682946C7
:108AE80005F047FC044A054B1A6009B0F0BD00BF09
:108AF800B801002000440040218A0008345F0020AB
:108B0800024B9868002105F034BC00BFB801002072
:108B180010B5094C40F22551204605F00EFD50B124
:108B2800A288D2B2112A02D1044B01211970044B38
:108B380019884A401A8010BD00440040160C0020D5
:108B4800980C00201FB5214B0C46186000214FF0EF
:108B5800804004F02CFF012100224FF0804005F0F6
:108B680056FA022C01D10B2303E0012C02D142F664
:108B7800DF6302930523ADF804304FF080400023F3
:108B880001A9ADF80C30ADF8063004F07BFE4FF0CB
:108B98008040012105F05BFA4FF08040012104F08C
:108BA800E4FE01210A464FF0804005F030FA4FF00C
:108BB8008040012104F0FBFE044B19680029FCD118
:108BC8004FF0804004F0F3FE1FBD00BF9C0C002056
:108BD8007047F0B5012085B02D4D014604F086FAA6
:108BE8004FF4D0530026019303270223284601A9F6
:108BF8008DF808308DF809708DF80A608DF80B60D3
:108C080003F0CCFE284609210A2203F047FF284634
:108C18000B210A2203F042FF0A2228460C2103F006
:108C28003DFF01244FF48063284601A901938DF884
:108C38000A408DF80B408DF8097003F0AFFE0A2149
:108C48000A46284603F02AFF21464FF4804004F0E4
:108C58007DFA8020214604F055FA31464FF0006035
:108C680000F0DEFA4FF4A06000F09CFA1C2303A881
:108C78008DF80C308DF80D608DF80E408DF80F4092
:108C880000F09AFA2046214604F054FA05B0F0BDE7
:108C98000000024007B54FF4C06000F083FA432398
:108CA8008DF8043001A801238DF805308DF80630C1
:108CB8008DF8073000F080FA0EBD044811B9012183
:108CC80003F0DDBE012103F0DCBE00BF0008024056
:108CD800022137E7012135E737B5042001210D4D81
:108CE80004F004FA022301248DF8053028460023F5
:108CF80069468DF806308DF8073000948DF80440E9
:108D080003F04CFE2846214603F0B9FEC820FFF7C1
:108D1800E1FF3EBD0008024008B54FF08040012148
:108D280005F08AF988B101214FF0804005F08FF9EC
:108D3800064B196819B11A68013A1A6008BD4FF054
:108D48008040BDE8084004F032BE08BD9C0C0020FD
:108D58007047012070470349034A02204FF4B77354
:108D680000F09CB824A10508749604080349044A35
:108D7800022040F2371300F091B800BF24A1050883
:108D8800849604080349044A022040F2011300F0C3
:108D980085B800BF24A10508A19604080249034A22
:108DA8000220F52300F07AB824A10508BA96040831
:108DB8000249034A0220EA2300F070B824A10508FA
:108DC800D49604080249034A0220DF2300F066B85B
:108DD80024A10508EC9604080249034A0220C82386
:108DE80000F05CB824A10508099704080249034A61
:108DF8000220BC2300F052B824A105082E970408CD
:108E08000249034A0220A62300F048B824A1050815
:108E18004D9704080249034A02208B2300F03EB80C
:108E280024A105086B9704080249034A02208023FD
:108E380000F034B824A10508889704080249034AB9
:108E48000220682300F02AB824A105089D97040889
:108E58000249034A0220522300F020B824A1050841
:108E6800B7970408FDF7F0BEFDF7F6BE04490A6897
:108E780001320A6003490346022000F00FB800BF20
:108E8800A00C002045A10508FDF7ECBE80F080008D
:108E9800092801D8FDF7ACBE704700BF0EB403B077
:108EA80070470A2810B5044602D10D20FFF7F9FFD4
:108EB800064A13681BB103F8014B136010BD044B3D
:108EC8001B680BB12046984710BD00BFA40C0020BA
:108ED800345F002010B5044601E0FFF7E2FF14F804
:108EE800010B0028F9D110BD2DE9F04F044685B0DB
:108EF8000D464FF00A0A00E035462078002800F0B9
:108F0800C480252801D0013467E06078302803D177
:108F1800A0780123033407E02D2802D0023400236F
:108F280002E0A078022303344FF0000805E00AFBB2
:108F3800080814F8010BA8F13008A0F13002D2B2E9
:108F4800092AF4D96C2801D04C2803D114F8010B54
:108F580043F00403002800F09880602886BFA0F141
:108F68002002D2B202464F2A3DD006D8432A2DD03D
:108F7800442A09D0422A30D133E0552A04D0582A4D
:108F880029D0532A29D101E00A272DE02E1D2F6868
:108F9800002500E001357A5D002AFBD104E020209D
:108FA800FFF77FFF4D4601E0980704D4454505F1DA
:108FB8000109F4D34D463846FFF78CFF03E0202023
:108FC800FFF76FFF01354545F9D395E728782E1D42
:108FD800FFF767FF90E7102706E0FFF762FF2E46CE
:108FE8008AE7022700E008272E1D442A296804D1B1
:108FF800002902DA494243F00803002200E02A4629
:10900800B1FBF7FE07FB1E11CDB2092D714607D93A
:10901800782814BF4FF0070C4FF0270C6544EDB2C9
:1090280030350DF80250551CBEF1000F02D0102D3E
:10903800E5D10F22190705D504A94D192D2105F8E9
:10904800101C951C13F0010F0CBF4FF0200B4FF0B4
:10905800300B9B072F4604D508E05846FFF721FF41
:109068004F46474507F10109F7D34F46013D1DF823
:109078000500FFF716FF002DF8D103E02020FFF7C9
:1090880010FF01374745F9D336E705B0BDE8F08F43
:1090980070B5064D0C462E68286001E0FFF701FF09
:1090A80014F8010B0028F9D12E6070BD345F002040
:1090B8000FB407B504A951F8040B0191FFF714FF89
:1090C800BDE80E4004B070470EB417B505A9084CAA
:1090D80051F8043B206018460191FFF705FF22680C
:1090E800002313702360BDE81E4003B0704700BF23
:1090F800A40C00200EB433B505A9074C51F8043B65
:109108002568206018460191FFF7EEFE2560BDE84E
:109118003C4003B0704700BF345F002070B51E4666
:1091280004461C481546FFF7C3FF022E1FD0042E25
:1091380025D0012E2AD105E0A15D1748FFF7B8FF19
:10914800013600E00026AE42F6DB2020FFF7A9FE3C
:10915800002609E0A05DA0F12003DBB25E2B88BFEA
:109168002E20FFF79EFE0136AE42F3DB0EE034F808
:10917800021B0A48FFF79CFF013DF8D106E054F8AE
:10918800041B0748FFF794FF013DF8D10A20BDE80A
:10919800704086E668A105086FA1050875A1050855
:1091A8007BA1050840F0BE60024B40F42020D86047
:1091B800704700BF00ED00E0C37810B503B3164B4D
:1091C8004278DB688478DB43C3F30223C3F10401EC
:1091D800C9B202FA01F10F2242FA03F2C9B22240DF
:1091E8000A430E4B01781201CB18D2B283F8002340
:1091F80003780122590903F01F0302FA03F307E079
:1092080003780122590903F01F0302FA03F32031FE
:10921800024A42F8213010BD00ED00E000E100E014
:1092280021F0604121F07F01014B084398607047AD
:1092380000ED00E0044B1A6909B1104301E022EA8D
:1092480000001861704700BF00ED00E0044B1A6889
:1092580004280CBF42F0040222F004021A6070478E
:1092680010E000E037B50023104C019305460320B9
:10927800FFF72EFDEB681A69013C019213D0019AA1
:10928800002AF4DA019A42F001020192019A1A6165
:10929800064A1969013A019102D00199C907F8D41F
:1092A8000320FFF715FD00203EBD00BF410D030060
:1092B80010B5C47874B900EB820003339B10D0F862
:1092C800D000224603E051F8044C01320460043116
:1092D8009A42F8D1002010BD033230B59210D0F870
:1092E800D0400B46002003E02568013043F8045CB9
:1092F80004339042F8D101EB800030BD0122F0B573
:109308000023827040220129C37082800CD1082377
:109318000370042343704FF4A073C38002230372C5
:10932800C1724FF0A04309E041B90C230370062332
:1093380043704FF4A063C3801F4BC17203F50062F2
:109348000261C3604678044601461A46002508E0D3
:1093580002F5106C02F530620A65C1F814C00135D7
:109368003A460431B54202F12007F1D303F5806291
:10937800426103F58862C0F8CC20067803F5A06541
:109388000146002203E0C1F88C5001322035043137
:10939800B242F8D31946002202E0C4F8CC100132D8
:1093A8000434B24201F58051F7D303F56063C0F885
:1093B8000C310020F0BD00BF0000044038B5037A2E
:1093C800C2680025012B04461FD1936B417A65F3CF
:1093D800104309B143F480139363D3686FF3861382
:1093E8006FF396536FF351436FF3D343D360204623
:1093F800FFF738FFE378012B19D1052363F3440500
:10940800E36845F020059D6011E0D36843F0400310
:10941800D360FFF727FF637AE268002B0CBF4FF495
:1094280004134FF4441393631420FFF753FCE378B9
:10943800012B07D1E3689D68052262F3440545F0D6
:1094480020059D60002038BDC3689A6842F001027B
:109458009A6000207047C3689A6822F001029A60F7
:109468000020704707B500230193019B43F02003B8
:109478000193019B61F38A130193019BC2681361F5
:10948800064B1169013B019102D001998806F8D475
:109498000320FFF71DFC00200EBD00BF410D030097
:1094A80007B500230193019B43F010030193019B2F
:1094B800C2681361064B1169013B019102D0019901
:1094C800C906F8D40320FFF703FC00200EBD00BF37
:1094D800410D030008B5C268D36801296FF35D73B5
:1094E8006FF39E7302D143F0005302E009B943F0D1
:1094F80080433220D360FFF7EDFB002008BDC3682E
:10950800586900F001007047C3685B6913F0010FE8
:1095180014BF002001207047C368586900F001009B
:109528007047C3685A69986910407047C36858689B
:10953800704743699B6813F0010F14BF0020012096
:109548007047C36800229A614FF0FF325A615A602F
:109558006FF080425A610B4A9A61C2789969002A71
:109568000CBF1022002242F0487221EA02010A438D
:109578009A619A6922F0005222F008029A6100204A
:10958800704700BF0008008043691A6861F3010250
:109598001A607047D0F8CC3018686FF382006FF308
:1095A80041006FF3C3006FF34510704738B50446A8
:1095B8000D46FFF782FB2046FFF7ECFFC0F30723B9
:1095C80003F01003DBB233B9012D04D1D4F8CC3049
:1095D80040F480501860C0F3072303F01003DBB297
:1095E8002BB125B9D4F8CC3065F30C301860C820FD
:1095F800BDE83840FFF76EBB43695869704738B516
:109608000546FFF7C7FFD5F8CC3040F480741C60DE
:109618006420FFF75FFBD5F8CC306FF308241420E3
:109628001C60FFF757FB012038BD70B50446FFF7F3
:1096380053FBD4F80C3100251D60237A012B08BF99
:109648002946204618BF0121FFF79EFF2046FFF755
:10965800D6FF63691A686FF382021A60E37A012BF6
:109668002E460ED1E36880225A6262F30F05E0228B
:1096780062F30F06C0F26005C0F260069D62C3F88F
:10968800006110212046FFF7EDFE2046FFF708FF96
:10969800002322464FF0FF35184604E0D2F88C101C
:1096A80001338D60C860217804328B42F6D320469E
:1096B8000121FFF77BFF2046FFF743FF002070BD25
:1096C80070B500EB810301F11504D3F8902000EB8D
:1096D80044154FF0FF339360C37895F81551012B6B
:1096E8000CBF04230023032D2BD8DFE805F0021F4D
:1096F800021300EB411404F56C7443F08903A57858
:1097080043F482637DB9247943F04003CCB143F03C
:10971800200316E000EB411443F0990394F8B24398
:1097280043F4C0636CB143F480730AE000EB441463
:1097380043F0010394F8124143F408730CB143F465
:10974800C073D360436901249D6904FA01F42C4372
:109758009C61C3689C69153100EB411044F00074AA
:109768009C6190F81011002361F39C5390F811113B
:1097780061F3CE2390F8121161F3CF3390F81311EF
:10978800A1F1020CDCF1000141EB0C0161F3514342
:1097980090F8151100F58874B0F8160161F3934339
:1097A80060F30A03032908BF43F000531360002045
:1097B80070BD70B501F11E04640186B003590A46F4
:1097C800002583B100EB4111013BB1F8B6135B18DA
:1097D800B3FBF1F39BB2B3F5807F05D909020151C0
:1097E8004FF4807300E0012300EB421191F8B2437B
:1097F80001F56C712CB1C98800EB42145943C4F8C7
:10980800C01300EB4211D1F8C01361F3120563F3E2
:10981800DC4500EB421393F8B84364F35E7500EB44
:109828008204D4F890402561C578012D08BFD3F88B
:10983800BC33456908BF63612368AE6816F0010F41
:1098480014BF0026012666F35D7343F000436FF3EF
:109858009E732360C378002B31D102F1150300EB0E
:10986800431393F8124154BB49B393F81531032BB2
:109878001DD8DFE803F0020F020FC368DC6A03316A
:109888000194C1F38F01A4B28C4210D2996941F0BE
:1098980020010BE02B6903310493C1F38F019BB2C4
:1098A8008B4204D2C368996941F08061996100EBE9
:1098B8004211B1F8C033D1F8BC13FFF7F9FC00200E
:1098C80006B070BD00EB810186B0D1F89020136816
:1098D80043F04043C3F3074111F00C0101D00829BC
:1098E80002D1C168C96A01E041690969C1F3074148
:1098F80009B961F3DF731360002006B070470346AF
:1099080010B503EB81030124D3F890304FF00042E7
:1099180064F3DC421A611A68002042F0004260F3E6
:109928009E721A6010BD43694FF0FF31002210B5D6
:109938009A610446596101460AE0D1F88C0003682F
:109948006FF3DF7343F080436FF3CF33036001326B
:10995800237804319A42F0D32046FFF7A1FD204630
:109968001021BDE810407DE5002310B51A460446D5
:10997800C0F8103303F1C60044F8202003F1D400E6
:1099880004EB80004260E01801330F2B80F890232D
:10999800F0D10823A4F8B6332046FFF7AFFC2046E1
:1099A800FFF759FD2046FFF709FD01212046FFF783
:1099B80091FD2046FFF739FE2046FFF745FD0020C0
:1099C80010BDD0F8CC301868C0F34140704708B5D6
:1099D800FFF715FE002008BDD0F810037047D0F837
:1099E800140370474369986880B27047401890F82C
:1099F8009F037047D43100EB8100406870474018DE
:109A080090F89003704708B5FFF75AFE08BD421852
:109A180008B5002382F89F3301F11E0200EB4212C1
:109A28005360FFF7C6FE08BD80B584B000AF78600C
:109A38004FF00003FB6040F20C23C2F200031B68E6
:109A48001B6878689847FB6843F00803FB607B68ED
:109A5800DB68FA685A614FF00103184607F11007EE
:109A6800BD4680BD80B584B000AF78604FF000037C
:109A7800FB6040F20C23C2F200031B689B68786805
:109A88009847FB6843F00053FB607B68DB68FA6823
:109A98005A614FF00103184607F11007BD4680BD13
:109AA80080B485B000AF78607B68D3F890301B68CD
:109AB800BB60BB6843F00043BB60BB6843F08043B6
:109AC800BB607B68D3F89030BA681A604FF0000327
:109AD800FB60FB6843F40013FB607B68DB68FA6893
:109AE8005A614FF00103184607F11407BD4680BCC0
:109AF800704700BF80B588B000AF78604FF00003B2
:109B0800FB724FF000037B617B6943F010037B61BC
:109B18007B68DB687A68D268926911467A696FEA6D
:109B280002020A409A617B68DB681B6ABB61BB69F9
:109B3800C3F30303DBB2FB72FB7ADBB27A6803F18F
:109B480022034FEA8303D3189B681B68FB60BB6939
:109B5800C3F34343DBB2022B40F09A80BB69C3F3E3
:109B68000A139BB2002B40F39480FB7ADBB27A682D
:109B78004FEA4313D31803F56F731B68002B00F0EB
:109B88008880FB7ADBB27A684FEA4313D31803F56F
:109B98006F731A68BB69C3F30A139BB278681146DE
:109BA8001A46FFF799FBBB69C3F30303DBB2BA6933
:109BB800C2F30302D2B279684FEA42128A1802F558
:109BC8006F721168BA69C2F30A1292B28A18796878
:109BD8004FEA4313CB1803F56F731A60BB69C3F3DD
:109BE8000303DBB2BA69C2F30302D2B2796802F1A5
:109BF8001E024FEA42128A1802F104021168BA6979
:109C0800C2F30A1292B28A18796803F11E034FEA66
:109C18004313CB1803F104031A60FB7ADBB27A68AA
:109C280003F11E034FEA4313D31803F104031B681F
:109C3800FB61FB7ADBB27A6803F1D4034FEA830352
:109C4800D318FA695A60FB7ADBB27A6803F1220307
:109C58004FEA8303D3189B681B693B613B69C3F3D5
:109C6800C9439BB2002B14DDFB6843F00043FB6043
:109C7800FB686FF39E73FB60FB7ADBB27A6803F1D3
:109C880022034FEA8303D3189B68FA681A6000E03E
:109C980000E000BF7B6943F010037B617B68DB68F1
:109CA8007A68D268926911467A690A439A614FF0D4
:109CB8000103184607F12007BD4680BD80B59CB05A
:109CC80000AF786039607A683B6803F122034FEA95
:109CD8008303D3189B68FB66FB6E9B68BB66FB6EB1
:109CE800DB687B66BA6E7B6E1340BB667A683B683E
:109CF80003F122034FEA8303D3189B681B683B6672
:109D08004FF000037B6697F8683003F00403DBB27A
:109D1800002B22D04FF00003BB65BB6D43F004035A
:109D2800BB65BA6DFB6E9A607A683B6803F12203E3
:109D38004FEA8303D3189B68DB687B657B6D43F030
:109D480002037B657A683B6803F122034FEA8303C9
:109D5800D3189B687A6DDA6098E097F8683003F05A
:109D68002003DBB2002B0AD04FF000033B653B6DAC
:109D780043F020033B653A6DFB6E9A6086E097F8E6
:109D8800683003F00803DBB2002B3ED07A683B68EA
:109D980003F122034FEA8303D3189B68DB68FB6453
:109DA800FB6C43F00203FB647A683B6803F122030F
:109DB8004FEA8303D3189B68FA6CDA607A683B68C9
:109DC800D31803F564734FF005021A704FF00003BF
:109DD800BB64BB6C43F01003BB64BA6CFB6E9A6047
:109DE8004FF000037B647B6C43F008037B647A6C60
:109DF800FB6E9A60BB6E6FF30413BB663B68DBB205
:109E080078681946FFF75EFD40E097F8693003F07F
:109E18000403DBB2002B39D07A683B6803F12203D4
:109E28004FEA8303D3189B68DB683B643B6C43F0C1
:109E380002033B647A683B6803F122034FEA830319
:109E4800D3189B683A6CDA603B68DBB278681946CD
:109E5800FFF738FD4FF00003FB63FB6B43F0100383
:109E6800FB63FA6BFB6E9A607A683B68D31803F55C
:109E780064734FF008021A704FF00003BB63BB6BAA
:109E880043F48063BB63BA6BFB6E9A6097F86930E2
:109E980003F00203DBB2002B28D07A683B6803F199
:109EA80022034FEA8303D3189B68DB687B637B6BD1
:109EB80043F002037B637A683B6803F122034FEAAD
:109EC8008303D3189B687A6BDA603B68DBB27868E7
:109ED8001946FFF7F7FC4FF000033B633B6B43F475
:109EE80000733B633A6BFB6E9A60DEE197F868306B
:109EF80003F00103DBB2002B00F0A5807B68DB7860
:109F0800012B1DD17A683B6803F122034FEA8303D2
:109F1800D3189B681B69FB657A683B6803F11E03CD
:109F28004FEA4313D3181A68FB6DC3F31203D21A0E
:109F380079683B6803F1D4034FEA8303CB185A606E
:109F48007A683B68D31803F564734FF001021A70FE
:109F58007B683A6802F1C6024FF0000143F822100C
:109F68004FF00003FB62FB6A43F00103FB62FA6AED
:109F7800FB6E9A6097F8623003F00C03DBB2002B9B
:109F880006D097F8623003F00C03DBB2082B3BD104
:109F98007A683B6803F122034FEA8303D3189B686E
:109FA800DB68BB62BB6A43F00203BB627A683B684A
:109FB80003F122034FEA8303D3189B68BA6ADA6075
:109FC8003B68DBB278681946FFF77CFC4FF000036A
:109FD8007B627B6A43F010037B627A6AFB6E9A604D
:109FE8007A683B684FEA4313D31803F572731B78FA
:109FF80083F00103DAB279683B684FEA4313CB1860
:10A0080003F572731A7050E197F8623003F00C038D
:10A01800DBB20C2B40F048813B6E43F000533B66AB
:10A028007A683B6803F122034FEA8303D3189B68DD
:10A038003A6E1A607A683B68D31803F566734FF076
:10A048000102DA7130E197F8683003F00203DBB2FD
:10A05800002B00F084807A683B6803F122034FEA02
:10A068008303D3189B68DB683B623B6A6FF3410349
:10A078003B627A683B6803F122034FEA8303D318F3
:10A088009B683A6ADA607A683B68D31803F56473A8
:10A098001B78DBB2012B08D17A683B68D31803F52B
:10A0A80066734FF00102DA714EE07A683B68D318A4
:10A0B80003F564731B78DBB2052B08D17A683B681B
:10A0C800D31803F566734FF00402DA713CE07A683E
:10A0D8003B68D31803F564731B78DBB2062B08D0F2
:10A0E8007A683B68D31803F564731B78DBB2082BD6
:10A0F80010D17B683A6802F1C6024FF0000143F8BC
:10A1080022107A683B68D31803F566734FF0030290
:10A11800DA7119E097F8623003F00C03DBB20C2B0C
:10A1280012D17A683B684FEA4313D31803F5727368
:10A138001B7883F00103DAB279683B684FEA43136E
:10A14800CB1803F572731A704FF00003FB61FB69BB
:10A1580043F00203FB61FA69FB6E9A60A5E097F889
:10A16800683023F07F03DBB2002B3ED07A683B686F
:10A1780003F122034FEA8303D3189B68DB68BB61B2
:10A18800BB6943F00203BB617A683B6803F12203B1
:10A198004FEA8303D3189B68BA69DA607B683A6828
:10A1A80002F1C60253F8223003F101017B683A68D4
:10A1B80002F1C60243F822107A683B68D31803F507
:10A1C80064734FF006021A703B68DBB27868194670
:10A1D800FFF778FB4FF000037B617B6943F0800356
:10A1E8007B617A69FB6E9A605FE097F8683003F0EC
:10A1F8001003DBB2002B58D097F8623003F00C0341
:10A20800DBB20C2B1DD17A683B6803F122034FEABD
:10A218008303D3189B68DB683B613B6943F0020307
:10A228003B617A683B6803F122034FEA8303D31842
:10A238009B683A69DA603B68DBB278681946FFF7D1
:10A2480041FB7A683B68D31803F564734FF0030247
:10A258001A704FF00003FB60FB6843F01003FB60CB
:10A26800FA68FB6E9A6097F8623003F00C03DBB271
:10A27800002B06D097F8623003F00C03DBB2082BF2
:10A2880013D13B6E43F000433B663B6E6FF39E7306
:10A298003B667A683B6803F122034FEA8303D318CD
:10A2A8009B683A6E1A6000E000BF4FF00103184641
:10A2B80007F17007BD4680BD80B59AB000AF7860E1
:10A2C80039607A683B6803F122034FEA8303D318A5
:10A2D8009B687B667B6E9B683B667B6EDB68FB6579
:10A2E8003A6EFB6D13403B667A683B6803F12203C4
:10A2F8004FEA8303D3189B681B68BB6597F86030E7
:10A3080003F00403DBB2002B22D04FF000037B657F
:10A318007B6D43F004037B657A6D7B6E9A607A6887
:10A328003B6803F122034FEA8303D3189B68DB6879
:10A338003B653B6D43F002033B657A683B6803F17C
:10A3480022034FEA8303D3189B683A6DDA6080E2F0
:10A3580097F8603003F02003DBB2002B0AD04FF0EF
:10A368000003FB64FB6C43F02003FB64FA6C7B6E18
:10A378009A606EE297F8613003F00203DBB2002BBB
:10A3880028D07A683B6803F122034FEA8303D31885
:10A398009B68DB68BB64BB6C43F00203BB647A68F0
:10A3A8003B6803F122034FEA8303D3189B68BA6C16
:10A3B800DA603B68DBB278681946FFF783FA4FF03A
:10A3C80000037B647B6C43F400737B647A6C7B6E64
:10A3D8009A603EE297F8603003F00103DBB2002B8D
:10A3E80038D07B683A6802F1C6024FF0000143F8A2
:10A3F80022107A683B6803F122034FEA8303D318DB
:10A408009B68DB683B643B6C43F002033B647A68FF
:10A418003B6803F122034FEA8303D3189B683A6C25
:10A42800DA603B68DBB278681946FFF74BFA4FF001
:10A438000003FB63FB6B43F00103FB63FA6B7B6E6A
:10A448009A607A683B68D31803F564734FF0010289
:10A458001A70FEE197F8603003F00803DBB2002BB6
:10A4680030D04FF00003BB63BB6B43F00803BB6302
:10A47800BA6B7B6E9A607A683B6803F122034FEAF5
:10A488008303D3189B68DB687B637B6B43F0020311
:10A498007B637A683B6803F122034FEA8303D3188E
:10A4A8009B687A6BDA603B68DBB278681946FFF71D
:10A4B80009FA7A683B68D31803F564734FF005020C
:10A4C8001A70C6E197F8603003F01003DBB2002B76
:10A4D80038D07B683A6802F1C6024FF0000143F8B1
:10A4E80022107A683B6803F122034FEA8303D318EA
:10A4F8009B68DB683B633B6B43F002033B637A6812
:10A508003B6803F122034FEA8303D3189B683A6B35
:10A51800DA603B68DBB278681946FFF7D3F94FF089
:10A528000003FB62FB6A43F01003FB62FA6A7B6E6E
:10A538009A607A683B68D31803F564734FF0030296
:10A548001A7086E197F8603023F07F03DBB2002BA6
:10A558003ED07A683B6803F122034FEA8303D3189D
:10A568009B68DB68BB62BB6A43F00203BB627A6824
:10A578003B6803F122034FEA8303D3189B68BA6A46
:10A58800DA603B68DBB278681946FFF79BF97B68AD
:10A598003A6802F1C60253F8223003F101017B68E0
:10A5A8003A6802F1C60243F822107A683B68D31869
:10A5B80003F564734FF006021A704FF000037B62D4
:10A5C8007B6A43F080037B627A6A7B6E9A6040E123
:10A5D80097F8603003F04003DBB2002B38D07B687B
:10A5E8003A6802F1C6024FF0000143F822107A6877
:10A5F8003B6803F122034FEA8303D3189B68DB68A7
:10A608003B623B6A43F002033B627A683B6803F1B2
:10A6180022034FEA8303D3189B683A6ADA603B68DF
:10A62800DBB278681946FFF74DF94FF00003FB617C
:10A63800FB6943F04003FB61FA697B6E9A607A68B4
:10A648003B68D31803F564734FF004021A7000E1F5
:10A6580097F8613003F00403DBB2002B3AD07A6834
:10A668003B6803F122034FEA8303D3189B68DB6836
:10A67800BB61BB6943F00203BB617A683B6803F1C5
:10A6880022034FEA8303D3189B68BA69DA603B68F0
:10A69800DBB278681946FFF715F94FF000037B61C4
:10A6A8007B6943F010037B617A697B6E9A607A68F4
:10A6B8003B68D31803F564734FF008021A704FF023
:10A6C80000033B613B6943F480633B613A697B6EFD
:10A6D8009A60BEE097F8603003F00203DBB2002B0B
:10A6E80000F0B7807A683B6803F122034FEA8303DE
:10A6F800D3189B68DB68FB60FB686FF34103FB6062
:10A708007A683B6803F122034FEA8303D3189B68F6
:10A71800FA68DA607A683B68D31803F564731B78C3
:10A72800DBB2012B22D17A683B68D31803F5667334
:10A738004FF00102DA7197F85A3003F00C03DBB2DC
:10A74800082B7CD17A683B684FEA4313D31803F58A
:10A7580072735B7883F00103DAB279683B684FEA79
:10A768004313CB1803F572735A7068E07A683B6834
:10A77800D31803F564731B78DBB2032B08D17A680E
:10A788003B68D31803F566734FF00202DA7156E09E
:10A798007A683B68D31803F564731B78DBB2042B23
:10A7A8001AD17A683B6803F115034FEA4313D318AB
:10A7B80003F588731B79012B05D13B68DBB27868F8
:10A7C8001946FFF79CF87A683B68D31803F5667357
:10A7D8004FF00202DA7132E07A683B68D31803F569
:10A7E80064731B78DBB2052B08D17A683B68D318F1
:10A7F80003F566734FF00402DA7120E07A683B686B
:10A80800D31803F564731B78DBB2062B17D17B686A
:10A818003A6802F1C60253F82230032B0FD17A6846
:10A828003B68D31803F566734FF00302DA717B684F
:10A838003A6802F1C6024FF0000143F822104FF0C7
:10A848000003BB60BB6843F00203BB60BA687B6E61
:10A858009A604FF00103184607F16807BD4680BDAE
:10A8680080B588B000AF78604FF00003FB614FF00F
:10A878000003FB604FF000033B614FF00003BB6136
:10A888004FF000037B617B68D3F8CC301B68BB6159
:10A898007B68D3F8CC301B687B617B696FF38203DC
:10A8A8007B617B696FF341037B617B696FF3C30352
:10A8B8007B617B696FF345137B613B7E03F0020389
:10A8C800DBB2002B0FD07B6943F002037B6140F2BF
:10A8D8000C23C2F200031B685B6878689847FB6921
:10A8E80043F00103FB613B7E03F00803DBB2002B5E
:10A8F80075D07B6943F008037B613B7E03F004035A
:10A90800DBB2002B63D0BB7E03F00603DBB2042B63
:10A9180005D0BB7E03F00603DBB2022B35D17B6882
:10A928005B691B683B61BB7E03F00603DBB2042B4B
:10A9380017D17B685B6941F270725A603B7C03F007
:10A948000303DBB2022B24D07B681B7A022B04D1D1
:10A9580078684FF00201FEF717FE7868FEF74FFEA1
:10A9680017E07B685B694BF680325A603B7C03F0EA
:10A978000303DBB2012B0CD078684FF00101FEF71E
:10A9880003FE7868FEF73BFE03E07868FEF737FEC3
:10A9980000E000BF40F20C23C2F200031B68DB6832
:10A9A800786898474FF00003FB60FB6843F000535A
:10A9B800FB607B68DB687A68D26892691146FA683E
:10A9C8006FEA02021140FA680A439A6107E040F20E
:10A9D8000C23C2F200031B681B69786898473B7E0A
:10A9E80003F02003DBB2002B07D07B6943F0200380
:10A9F8007B61FB6943F00103FB617B68D3F8CC30D2
:10AA08007A691A60FB69184607F12007BD4680BDC0
:10AA180080B586B000AF78607B685B691B69BB60F6
:10AA28003B7BC3F3C303DBB27A6803F11E034FEA2F
:10AA38004313D3181B6803F103034FEA9303FB8204
:10AA4800A3E03B894FEA8303BB82BA8A3B7BC3F30B
:10AA5800C303DBB2796803F11E034FEA4313CB1833
:10AA68001B689A421DD93B7BC3F3C303DBB27A68E8
:10AA780003F11E034FEA4313D3181B68BB824FF040
:10AA880000033B613B6943F080633B617B68DB68A3
:10AA98007A68D268926911463A696FEA02020A40F6
:10AAA8009A613B7BC3F3C303DBB27A6803F11E03ED
:10AAB8004FEA4313D3181B6803F103034FEA9303C8
:10AAC800FB823B7BC3F3C303DBB27A684FEA4313D1
:10AAD800D31803F56F7319683B7BC3F3C303DBB269
:10AAE8001A46BB8A7868FEF7E3FB3B7BC3F3C303D4
:10AAF800DBB23A7BC2F3C302D2B279684FEA4212A0
:10AB08008A1802F56F721168BA8A8A1879684FEA4A
:10AB18004313CB1803F56F731A603B7BC3F3C3036E
:10AB2800DBB23A7BC2F3C302D2B2796802F11E02E9
:10AB38004FEA42128A181168BA8A8A1A796803F1A8
:10AB48001E034FEA4313CB181A603B7BC3F3C303BE
:10AB5800DBB23A7BC2F3C302D2B2796802F11E02B9
:10AB68004FEA42128A1802F104021168BA8A8A1856
:10AB7800796803F11E034FEA4313CB1803F104036A
:10AB88001A607B685B691B69BB603B89FA8A9A42D9
:10AB98000DD23B7BC3F3C303DBB27A6803F11E0318
:10ABA8004FEA4313D3181B68002B7FF44AAF4FF0CA
:10ABB8000103184607F11807BD4680BD80B588B067
:10ABC80000AF78607B68DB68DB6AFB603B7CC3F3C3
:10ABD800C303DBB27A6803F11E034FEA4313D318A9
:10ABE8001B6803F103034FEA9303FB83A3E0BB89CC
:10ABF8004FEA8303BB83BA8B3B7CC3F3C303DBB24B
:10AC0800796803F11E034FEA4313CB181B689A4275
:10AC18001DD93B7CC3F3C303DBB27A6803F11E037F
:10AC28004FEA4313D3181B68BB834FF00003BB6183
:10AC3800BB6943F02003BB617B68DB687A68D26834
:10AC480092691146BA696FEA02020A409A613B7C2E
:10AC5800C3F3C303DBB27A6803F11E034FEA43135D
:10AC6800D3181B6803F103034FEA9303FB833B7C70
:10AC7800C3F3C303DBB27A684FEA4313D31803F56F
:10AC88006F7319683B7CC3F3C303DBB21A46BB8BF3
:10AC98007868FEF70DFB3B7CC3F3C303DBB23A7C59
:10ACA800C2F3C302D2B279684FEA42128A1802F597
:10ACB8006F721168BA8B8A1879684FEA4313CB18F8
:10ACC80003F56F731A603B7CC3F3C303DBB23A7CB2
:10ACD800C2F3C302D2B2796802F11E024FEA4212ED
:10ACE8008A181168BA8B8A1A796803F11E034FEA29
:10ACF8004313CB181A603B7CC3F3C303DBB23A7C23
:10AD0800C2F3C302D2B2796802F11E024FEA4212BC
:10AD18008A1802F104021168BA8B8A18796803F15B
:10AD28001E034FEA4313CB1803F104031A607B6830
:10AD3800DB68DB6AFB60BB89FA8B9A420DD23B7CED
:10AD4800C3F3C303DBB27A6803F11E034FEA43136C
:10AD5800D3181B68002B7FF44AAF4FF00103184645
:10AD680007F12007BD4680BD80B586B000AF78608A
:10AD78004FF000037B614FF000033B617868FEF7FA
:10AD88003BFC0346FB604FF000037B6134E0BB896A
:10AD98001A467B6942FA03F303F00103DBB2002B86
:10ADA80026D07A687B6903F122034FEA8303D3181C
:10ADB8009B681B68BB607B7A23F07F03DBB2002BA8
:10ADC8000BD049F6C543C0F60003786879699847FF
:10ADD80003463A6913433B610AE04AF2C123C0F6CD
:10ADE800000378687969984703463A6913433B61D9
:10ADF8007B6903F101037B617B681B781A467B69D9
:10AE08009A42C4D83B69184607F11807BD4680BD69
:10AE180080B584B000AF78604FF00003FB604FF05E
:10AE28000003BB607868FEF777FB0346002B00F051
:10AE38008B807868FEF775FB0346BB60BB68002B08
:10AE480002D14FF0000380E03B7A03F00803DBB245
:10AE5800002B09D049F63123C0F6000378689847DB
:10AE68000346FA681343FB603B7A03F01003DBB236
:10AE7800002B09D049F6FD23C0F6000378689847EF
:10AE88000346FA681343FB603B7A03F02003DBB206
:10AE9800002B09D04AF6C533C0F6000378689847F6
:10AEA8000346FA681343FB60FB7A03F00403DBB242
:10AEB800002B09D04AF61923C0F600037868984792
:10AEC8000346FA681343FB60FB7A03F00203DBB224
:10AED800002B09D04AF67153C0F6000378689847EA
:10AEE8000346FA681343FB60FB7A03F00103DBB205
:10AEF800002B09D04AF66903C0F600037868984722
:10AF08000346FA681343FB60FB7A03F02003DBB2C5
:10AF1800002B09D049F66D23C0F6000378689847DE
:10AF28000346FA681343FB60BB7A03F02003DBB2E5
:10AF3800002B09D049F6A923C0F600037868984782
:10AF48000346FA681343FB60FB68184607F11007CD
:10AF5800BD4680BD0123C0F810330020704701238F
:10AF6800C0F81433002070470023C0F81433184683
:10AF780070470020704738B504460021FDF79DFE54
:10AF8800E36800254FF0FF329D6120465A61FEF7C5
:10AF980062FAC4F81053284638BD70B5012300255D
:10AFA80040220C46CB700B778A7181F82130064617
:10AFB8000D704D708D7081F82050097900F02BFBD1
:10AFC8006179304600F027FB284670BD2DE9F04135
:10AFD800069F1646984604460D46FDF7FAFD0020E2
:10AFE800FDF77AFE31462046FFF7D7FF2946C6F817
:10AFF8007C80C6F880702046FEF7B6FCD6F8803014
:10B008001B6898472046BDE8F041FDF743BE0B1F7B
:10B01800DBB2012B10B5044606D8D0F880305B6C43
:10B0280098470B23237010BD062905D10B23037005
:10B03800D0F880301B68984710BD002370B58B741A
:10B048000B7F013B05460C460A2B00F2C980DFE85E
:10B0580013F00B0012003900400058006500790019
:10B0680080009900A900B90001F11401627900F08B
:10B078003BFD022343E04979FEF7B8FC012819D1CA
:10B08800237D618B584A03F0800339B141F288313E
:10B0980011800BB1032307E0052305E0322111805D
:10B0A8000BB1092300E0072323772846FEF79AFC13
:10B0B800208295E0032840F093800B232377052313
:10B0C800A3748DE00B798A89896800F044FD042314
:10B0D80015E00979FEF78AFC012802D109232377B4
:10B0E80003E0042823D0032808D02846FEF77AFC7A
:10B0F800238AC01A3C4B1B88984271D90B232377AB
:10B108006EE04B7900EB4313012283F8C9234B7996
:10B118008A89896800F0FDFC0623F0E74979FEF783
:10B1280065FC012801D10723E9E7042803D16378E6
:10B1380023700C23E3E7022801D10523DFE7032866
:10B148004ED1DBE70B7900210A4600F004FD082305
:10B15800D5E70979FEF74AFC0128064627D00328D7
:10B16800CCD02846FEF73EFC238AC01A1E4B1B880B
:10B178009842C3D8042E33D1637823700C232377E5
:10B18800032070BD4B7900EB431393F8C92382F079
:10B19800010283F8C9234B7900210A4600F0B9FC63
:10B1A8000A23ACE74979FEF721FC012803D163782B
:10B1B80023700D23A3E7022801D109239FE7032861
:10B1C80010D19BE78B7B0133DBB2022B8B7301D849
:10B1D800012394E708238B744B7802200B7070BD11
:10B1E800002070BD002070BDA80C002070B594B080
:10B1F800022305460C468DF84F30FEF7EDFB18B1DB
:10B208002846FEF7ECFB28B923781BB1032B01D0A5
:10B218000323237023780B2B00F29181DFE813F0CE
:10B228000C001F0026006D018F01580040014C01E1
:10B23800590131018F015E012846FEF7CDFB002838
:10B2480000F07D8101232370C820FDF743FD2846C7
:10B25800FEF7BDFBD4F88030DB6898476FE1D5F87E
:10B268001433012B40F06B81022367E1D4F880305E
:10B278009B6898470021284600F0B4F98021607146
:10B28800284600F0AFF920712846FEF79AFB0523FF
:10B29800C0B22370D4F8803084F821009B699847A5
:10B2A800A079217994F8202094F821300190002683
:10B2B8002846009600F048F9A0796179019094F841
:10B2C800202094F821300096284600F03DF936E118
:10B2D800A378092B00F23381DFE813F00A00280075
:10B2E800380060006B007F009800B100C9002B0196
:10B2F80028462146082200F01DFD0646002840F099
:10B308001E8194F829306179A3710122A2700090FE
:10B31800019332463346284600F043F9A379217950
:10B328000193009628463246334634E028462146A3
:10B33800122200F0FFFC002840F00181D4F8803090
:10B3480004F12200DB699847022330E028462146B1
:10B35800012200F045FD0646002840F0F08002205A
:10B36800FDF7B8FC012384F82030D4F880301B6A3C
:10B3780098470323A370217994F820200096334638
:10B388002846019600F00DF9617994F8202000967E
:10B3980001962846334600F004F9D0E028462146B5
:10B3A800092200F019FE002840F0C9800423A37088
:10B3B800C5E0E28E2846214600F00EFE002840F047
:10B3C800BE80D4F8803004F134005B6A04F13E0199
:10B3D80004F1500298470523E9E794F8302072B148
:10B3E800FF2300932846214603AB00F07BFC00288E
:10B3F80040F0A580D4F8803003A89B6A03E0D4F815
:10B40800803050489B6A98470623D0E794F831204B
:10B4180072B1FF2300932846214603AB00F062FC7B
:10B42800002840F08C80D4F8803003A8DB6A03E061
:10B43800D4F880304348DB6A98470723B7E794F885
:10B4480032206AB1FF2300932846214603AB00F05F
:10B4580049FC002873D1D4F8803003A81B6B03E0A3
:10B46800D4F8803037481B6B984708239FE794F837
:10B4780039202846214600F0C0FC00285FD1092366
:10B4880095E7D4F880309B6B9847012857D1E36F34
:10B4980028461B6821469847002850D106234DE0CE
:10B4A800E36F28469B68214698478DF84F009DF822
:10B4B8004F3043B9072341E0E36F2846DB68214654
:10B4C80098478DF84F009DF84F102046FFF79FFDD5
:10B4D80035E028462146FFF7B0FD30E021462846F2
:10B4E800FFF75BFDD4F880305B689847E36F04F1A1
:10B4F80020015B682846984721E0D4F880301B6912
:10B50800984721462846FFF748FDD4F880305B6805
:10B518009847E36F04F120015B682846984728465E
:10B5280000F085F80023237028460121FEF71CFA55
:10B5380005E0D4F880305B6B98470923237014B07A
:10B5480070BD00BF82A10508F8B501F5327430F866
:10B55800146001F1150400EB441406F07F0784F829
:10B5680010219DF8182084F8117184F81521BDF870
:10B578001C2084F81331A4F81621C6F3C01600EB7A
:10B58800411204F5887584F81261002482F8C843D2
:10B5980082F8C9430BB901232B71FEF791F80020FB
:10B5A800F8BD70B5BDF814401AB100EB411585F827
:10B5B800B02301F1150200EB4215B5F81661A64259
:10B5C80005F5887501D004B1EC8000EB421292F8C1
:10B5D80013419C4202D00BB182F81331FEF770F888
:10B5E800002070BD10B502460023B2F99045002C2A
:10B5F80008DB03F532726FEA41416FEA514120F8E6
:10B60800121006E00133DBB20232082BEDD14FF6FF
:10B61800FF73D8B210BD072907D801F5327130F889
:10B62800113023F4004320F8113000207047002324
:10B63800A0F89435A0F89635A0F89835A0F89A3572
:10B64800A0F89C35A0F89E3518467047F8B5314DDE
:10B6580095F8423006460F46052B58D8DFE803F028
:10B668000357571309272B6D1B689847042385F840
:10B6780042303046FDF75DFF012848D1254B0322B3
:10B6880083F8422043E095F8462095F84030214958
:10B6980000F0A3FA204B01221A703046052385F8E2
:10B6A8004230FEF79FF980B2A5F84C002FE0FEF774
:10B6B80099F9B5F84C30174C9BB2C01AB5F84A3016
:10B6C800984221D294F840103046FEF78FF90128AD
:10B6D8000AD1114B1A78012A19D100221A70236D48
:10B6E80020465B68984712E094F840103046FEF711
:10B6F8007DF904280BD194F8482094F8403030465E
:10B70800394600F095FB10B9032384F84230002035
:10B71800F8BD00BF805F0020AA0C0020384B93F8CA
:10B72800453073B50446042B66D8DFE803F00332CE
:10B738000340530000F58873009309230193012205
:10B748004FF4045300F0B4FA002855D12D4B94F867
:10B75800102194F813111A7094F811215A7094F862
:10B76800122102EB01225A8094F8142194F818113E
:10B778001A7194F815215A7194F816219A7194F84F
:10B78800172102EB01221A811D4B012083F8450085
:10B7980035E000F5887300931A4B1B890122019349
:10B7A8004FF4085300F084FA30BB03220EE0212343
:10B7B80000220B750A234B75CA820A834A831346F3
:10B7C80000F06CF908B1032816D104220C4B83F859
:10B7D800452011E0212300220B7501250B234B7511
:10B7E800CD820A834A831346164600F057F928B9D2
:10B7F800034B83F8456002E0012000E028467CBD49
:10B80800805F0020D45F002038B5114D95F84010B6
:10B81800044649B1FEF756F895F840102046FFF760
:10B82800FAFE002385F84030094D95F8411051B1D2
:10B838002046FEF747F895F841102046FFF7EBFE43
:10B84800002385F84130034B00221A7038BD00BF31
:10B85800805F0020AA0C00202DE9F347344B062214
:10B8680083F8422091F84420012A07460C4658D113
:10B8780091F84520012A04BF2E4A1A65002283F850
:10B88800422083F8452091F8522083F84820B1F8E7
:10B898005420A3F8462091F85620092AA3F84A20F4
:10B8A80003D8234B0A22A3F84A2094F842A0204D3B
:10B8B800BAF1020F28BF4FF0020A26464FF00008DF
:10B8C8004FF0030927E096F852100B0608D53846C2
:10B8D80085F84410FFF786FE014685F8400009E028
:10B8E80085F8431096F852103846FFF77BFE01465C
:10B8F80085F84100B5F8460094F82020019094F8A6
:10B908002130CDF800903846FFF71EFE08F10108F7
:10B918005FFA88F80836D045D5D1074B0020187053
:10B9280004E0D1F880301B6C98470120BDE8FC8703
:10B93800805F002034020020AA0C002030B543EAC2
:10B9480002229DF80C40CA8221250023049A0D7515
:10B958000B83092523464D754C83BDE8304000F024
:10B968009DB800BF70474A4A00232DE9F04713707D
:10B9780053709370D37005461A46E91801338978D5
:10B988000139C9B2022998BF0122062BF5D1012A33
:10B998007CD03F4991F802C00A784B7828460226A5
:10B9A80001F10A098778BFB18C1801322771D2B228
:10B9B800002406E0013409EB040A1AF801ACBA4580
:10B9C80003D05FFA84F8E045F4D3E04504D1CC18FD
:10B9D800877801332774DBB20136F6B20130082EBE
:10B9E800E0D12B4C012B2270637041D1207CE07098
:10B9F800FDF757FA2B78102B1BD022460AD8022BBA
:10BA08001BD003D89BB1012B1DD112E0042B16D0FB
:10BA1800052B0AE0402B12D004D8142B11D0202B70
:10BA280011D10AE0412B0CD0502B0CD109E0A375A1
:10BA380009E0174B02229A7505E0012302E003236F
:10BA480000E004239375124A937DD178114A012BA3
:10BA580005D803EB4103D05CFDF718FA0AE0032090
:10BA680000FB013102EB8102D2F8C030984701E0B7
:10BA78000023E370064A137802F10A019370002349
:10BA88000432985C58540133062BFAD1BDE8F0878C
:10BA9800AB0C0020C8970408FDF7F6B9C878012850
:10BAA80010B504D002284FF0010319D108E00C7832
:10BAB8008B814C7008240C708A600877022308E098
:10BAC8000A7F0D2A03D10020CB70087710BD0B2AFE
:10BAD80001D1CB7010BD0C2A04D1CB70032010BD4E
:10BAE800184610BD184610BD00EB421310B50024CF
:10BAF80083F8B24300EB42130324C3F8BC130821B4
:10BB0800C3F8C01383F8B8431146FDF780FFC0B2ED
:10BB180010BD38B500EB4314002584F8B2535C011E
:10BB28000519C5F8BC1300EB4311C1F8C02312B9BD
:10BB3800012285F8C923041900EB431294F8C913AC
:10BB4800002914BF0221002182F8B8131946FDF715
:10BB58005EFF002038BD38B500EB4314012584F89A
:10BB6800B2530225C4F8BC1384F8B853C4F8C023F0
:10BB78001946FDF74CFF002038BD38B500EB4315DA
:10BB8800002485F8B24300EB4315C5F8C02395F8A7
:10BB9800C923C5F8BC13A24214BF0222224685F865
:10BBA800B8231946FDF733FF204638BD38B500EBFA
:10BBB80043140125C4F8C02394F8C823C4F8BC135F
:10BBC800002A14BF0222002284F8B25384F8B82352
:10BBD8001946FDF71CFF002038BDF8B504461F467E
:10BBE8000E46154602201A460E49FDF757F904EB92
:10BBF8004713012283F8B22393F8C823C3F8BC6320
:10BC0800002A14BF0221002182F0010283F8B81330
:10BC1800C3F8C05383F8C82320463946FDF7F7FE1A
:10BC28000020F8BD86A1050838B500EB43150024AF
:10BC380085F8B24300EB4315C5F8C02395F8C8232F
:10BC4800C5F8BC13A24214BF0221214682F00102AA
:10BC580085F8B81385F8C8231946FDF7D8FE20469D
:10BC680038BD38B500EB4314012584F8B253254696
:10BC7800C4F8BC13C4F8C023002485F8B843194697
:10BC8800FDF7C5FE204638BD38B500EB4315002446
:10BC980085F8B24300EB4315C5F8BC13C5F8C023BB
:10BCA80085F8B8431946FDF7B2FE204638BD00BFF7
:10BCB80010B562F07F020A750622BDF80C404A757D
:10BCC800CB8240F2094203F47F43B3F5407F0CBFB7
:10BCD80013460023029A0B8323464C83BDE8104089
:10BCE800FFF7DCBE73B5BDF818601D4642F440731B
:10BCF80000F588728DE8440000220446FFF7D8FF5B
:10BD0800B8B994F81131032B13D194F81031023BD0
:10BD18009E42A8BF1E46B6B2034606E0E2180233AA
:10BD280092F8122105F8012B9BB2B342F6D30023F7
:10BD38002B707CBD73B500F5887316468DE84800F6
:10BD480000224FF4807304460D46FFF7B1FF002828
:10BD580045D194F8103185F8223094F8113185F8DE
:10BD6800233094F8132194F8123103EB0223AB84A7
:10BD780094F8143185F8263094F8153185F8273071
:10BD880094F8163185F8283094F81731082E85F87C
:10BD9800293024D994F8192194F8183103EB022397
:10BDA8006B8594F81B2194F81A3103EB0223AB85B9
:10BDB80094F81D2194F81C3103EB0223EB8594F8C9
:10BDC8001E3185F8303094F81F3185F8313094F8F9
:10BDD800203185F8323094F8213185F833307CBD34
:10BDE80010B500230524CA821A460B754C750B83BF
:10BDF8004B83BDE81040FFF751BE10B5002309245E
:10BE0800CA821A460B754C750B834B83BDE81040EC
:10BE1800FFF744BE10B50A83012400220C75CB82BB
:10BE28000B2413464C754A83BDE81040FFF736BE15
:10BE380030B54FEA431302240C75C31801244C751E
:10BE4800002412F0800F0A83CC824C8314BF83F83D
:10BE5800C84383F8C943002225461346BDE830404D
:10BE6800FFF71CBE2DE9F04F93461A7802705A78F6
:10BE780089B042709A780691D97802EB0122428003
:10BE88001A7902715979417199798171D979C17198
:10BE9800197A0172BDF84810092940F29480022AE3
:10BEA80000F293804B4A092192F800C0548881E03F
:10BEB8001A789B1889185A78042A89B27AD19E78F8
:10BEC80093F803A0069F09254FFA86F8BAF1020FE6
:10BED80005FB08726ED81D781F7900955D7901956C
:10BEE8009D790295DD7903951D7A022F049504D971
:10BEF800384B83F800C05C8067E04FEA4805059539
:10BF0800CDF81C800025814650E018781B180918C8
:10BF18005878052889B249D10798844511D00098E6
:10BF28009670107004205070019882F803A0507128
:10BF38000298177190710398D0710498B4461072E2
:10BF480016E0187993F8058000EB0820844230DC6D
:10BF580000989670107004205070019882F803A021
:10BF680050710298177190710398D07104981072EB
:10BF7800059893F8008040FA85F40BEBC4000BF8A1
:10BF880034805C7844709C788470DC78C47093F852
:10BF980005801C7904EB082484809C7984715C7981
:10BFA8001879013500EB0424A4B2EDB268B2B842A6
:10BFB800ABDB484642888A423FF67AAF054B002001
:10BFC8005880187002E0002000E0032009B0BDE8A6
:10BFD800F08F00BFC20C0020F7B54FF4007300F5D6
:10BFE800887701921546002206460C460097FFF70F
:10BFF8005FFE034633B113E0F11891F8101199541C
:10C00800013300E0074A99B2A942F5D304F134009C
:10C0180004F13E0104F150023B460095FFF722FF70
:10C02800FEBD00BFE65F002003780A88D3180B80A6
:10C038000378C018704700BF036823F0010303604A
:10C048000023036043608360C3600361212343616D
:10C058002C4B98421CD02C4B984220D02B4B98420A
:10C0680025D02B4B98422AD02A4B98422FD02A4BC6
:10C07800984233D0294B984237D0294B984204D163
:10C088004FF03D5243F8AC2C7047264B984203D1F1
:10C098003D2243F8082C7047234B984204D14FF4B3
:10C0A800746243F8202C7047204B984204D14FF417
:10C0B800741243F8382C70471D4B984204D14FF046
:10C0C800746243F8502C70471A4B984203D11A4AAD
:10C0D80043F8642C7047194B984203D1184A43F827
:10C0E8007C2C7047174B984203D1174A43F8942C7D
:10C0F8007047164B984204BF4FF03D5243F8AC2CA2
:10C10800704700BF10600240286002404060024053
:10C11800586002407060024088600240A06002409F
:10C12800B860024010640240286402404064024043
:10C1380058640240706402403D0000208864024058
:10C14800400F0020A064024000003D20B864024077
:10C158000268134B10B51340CC680A6822434C6937
:10C1680022438C692243CC6922430C6A22434C6ADD
:10C1780022438C6A22434C6B22438C6B2243134329
:10C18800036042690C6BCB6A22F007022343134316
:10C1980043610B6943604B6883608B68C36010BD63
:10C1A8003F801CF00023036043608360C360036129
:10C1B80043618361C361036243628362C362036351
:10C1C800436383637047036811B143F0010301E0DF
:10C1D80023F0010303607047036811B143F400437F
:10C1E80001E023F4004303607047036811B143F092
:10C1F800200301E023F0200303607047416070478B
:10C20800406880B27047036812B143F4002301E02C
:10C2180023F40023036001617047036811B143F4FC
:10C22800802301E023F48023036070470AB1016191
:10C238007047C16070470068C0F3C040704700682D
:10C2480000F001007047406900F0380070470A4A62
:10C258000A4B10B50A4CA04288BF13468A004CBF4F
:10C268005B681B6821F0F02121F0821119420CBF94
:10C278000020012010BD00BF0064024000600240A1
:10C288000F64024010B5084B084A094CA04288BF09
:10C29800134611F0005F21F0F02121F0821114BF44
:10C2A800D960996010BD00BF006002400064024080
:10C2B8000F6402400B0607D5436912B143F08003AF
:10C2C80001E023F080034361802909D001F01E01B9
:10C2D800036812B119430160704723EA0101016044
:10C2E8007047124B124A10B5124CA0428CBF14462C
:10C2F8001C4621F0F02323F0C3132BB1026802F08F
:10C308001E0202EAD12202E0426902F0800288009D
:10C318004CBF6368236821F0F02121F08210184097
:10C3280002D0101C18BF012010BD00BF00600240E1
:10C33800006402400F64024010B5084B084A094CDB
:10C34800A04288BF134611F0005F21F0F02121F0D0
:10C35800821114BFD960996010BD00BF006002400F
:10C36800006402400F640240044B00221A605A60C5
:10C378009A60DA60024A5A61704700BF003C014087
:10C38800FFFF7F00837910B5002B29D01A4B016875
:10C398001C68CA4314401C605C6822405A600279D9
:10C3A80002F1804202F59E3214682143116002684E
:10C3B8009C68D1430C409C60DC682140D96041797D
:10C3C800102906D1996811439960D9680A43DA603F
:10C3D80010BD01F1804303F59E3319680A4308E054
:10C3E8000379016803F1804303F59E331A6822EA52
:10C3F80001021A6010BD00BF003C014000230C225E
:10C4080003600371427183717047024B1A690243DA
:10C418001A617047003C0140034B5B6918420CBF2E
:10C4280000200120704700BF003C0140014B5861CB
:10C43800704700BF003C0140054B1A685B69034028
:10C4480004D010420CBF00200120704718467047E6
:10C45800003C0140014B5861704700BF003C01405F
:10C468004FF0204318B943F2DB021A6003E043F2AD
:10C47800D20243F820204FF02042411C6FF0704355
:10C4880042F8213002F5827242F82030704770B5C8
:10C4980084684568C368C16A026825431D43036907
:10C4A8001D4343691D4383691D43C3691D43036AD3
:10C4B8001D43436A1D43836A1D43036B0D431D439C
:10C4C8004FF02043082C43F8225005D153F822405E
:10C4D80044F0400443F82240436B9E691D6835438D
:10C4E8005E6845EA06159E6845EA0625DE6845EA5F
:10C4F80006451E695B6945EA0655541C45EA03650D
:10C508004FF02043B1F5804F43F8245010D1836B8E
:10C51800986919680143586841EA0011986841EA26
:10C52800002118695B6941EA005141EA036101E0B1
:10C538006FF07041014B43F8221070BD040100A058
:10C54800022242604FF480524262416B4FF4005223
:10C5580010B5826200230F22FF2403608360C3604A
:10C56800036143618361C3610362C36203630A6059
:10C578004A608C60CA600A614A618B61816B0A609B
:10C588004A608C60CA600A614A618B6110BD4FF0D5
:10C59800204321B153F8202042F0010203E053F870
:10C5A8002010024A0A4043F820207047FEFF0F007F
:10C5B80010280CBF064B074B4FF040024FF01801F4
:10C5C80019605A604FF0FC329A60DA60704700BF19
:10C5D800600000A0800000A030B5836844681C4358
:10C5E800C36844F008041C4303691C43436944EAD4
:10C5F8004324836944EA4334C36999685A6809043F
:10C6080041EA02211A68DB68114341EA0361036ABF
:10C618009A685D68120442EA05221D68DB682A43AD
:10C6280042EA03620368102B0CBF034B034B1C60E8
:10C638009960DA6030BD00BF600000A0800000A0F3
:10C6480010230360C269002343608360C3600361F1
:10C6580043618361FC23136053609360D360026A73
:10C66800136053609360D360704741B110280CBFCA
:10C67800074B084B1A6842F004021A6070471028EA
:10C688000CBF034A034A044B11680B401360704700
:10C69800600000A0800000A0FBFF0F0041B110283F
:10C6A8000CBF084B084B1A6842F040021A607047EA
:10C6B80010280CBF034A044A044B11680B4013604E
:10C6C800704700BF600000A0800000A0BFFF0F00FF
:10C6D800102802D1024B58697047024B58697047BD
:10C6E800600000A0800000A0054B18221A600022FC
:10C6F8005A604FF0FC329A60DA601A61704700BFE6
:10C70800A00000A00268436842F0100242EA4322F7
:10C71800836842EA4332144B10B51A60C2689168C4
:10C728005468090441EA04211468D268214341EAA3
:10C7380002629A60026991685468090441EA042116
:10C748001468D268214341EA0262DA60426991685A
:10C758005068090441EA00211068D268014341EA9F
:10C7680002621A6110BD00BFA00000A0C2680023C9
:10C77800036043608360FC23136053609360D3605D
:10C788000269136053609360D36042691360536019
:10C798009360D3607047054B18B11A6842F00402E1
:10C7A80002E01968024A0A401A607047A00000A017
:10C7B800FBFF0F0062B1102801D10E4B03E0B0F56A
:10C7C800807F03D10C4B5A68114311E00B4BFAE7F9
:10C7D800102804D1074B5A6822EA010108E0B0F595
:10C7E800807F0CBF044B054B5A686FEA010111406A
:10C7F80059607047600000A0800000A0A00000A061
:10C80800102801D1064B04E0B0F5807F0CBF054B22
:10C81800054B5B680B420CBF00200120704700BF2E
:10C82800600000A0800000A0A00000A0102804D193
:10C83800074B5A6822EA010108E0B0F5807F0CBF77
:10C84800044B054B5A686FEA010111405960704763
:10C85800600000A0800000A0A00000A0102801D166
:10C86800084B04E0B0F5807F0CBF074B074B5B68B3
:10C8780013EA010004D013EAD1010CBF0020012003
:10C88800704700BF600000A0800000A0A00000A0CA
:10C89800102804D1084B5A6822EAD10109E0B0F502
:10C8A800807F0CBF054B064B5A684FEAD10122EA3C
:10C8B80001015960704700BF600000A0800000A01F
:10C8C800A00000A008B52C4B984205D101200146D4
:10C8D80000F048FC012048E0284B984205D102208E
:10C8E800012100F03FFC02203FE0254B984205D192
:10C8F8000420012100F036FC042036E0214B984248
:10C9080005D10820012100F02DFC08202DE01E4B48
:10C91800984205D11020012100F024FC102024E0C9
:10C928001A4B984205D12020012100F01BFC202041
:10C938001BE0174B984205D14020012100F012FC62
:10C94800402012E0134B984205D18020012100F0CD
:10C9580009FC802009E0104B98420BD14FF48070FD
:10C96800012100F0FFFB4FF480700021BDE8084072
:10C9780000F0F8BB08BD00BF000002400004024000
:10C9880000080240000C024000100240001402405F
:10C9980000180240001C0240002002402DE9F04728
:10C9A8000023D1F800801A464FF0010C03270CFA37
:10C9B80002F404EA0805A5422ED1066817FA03F422
:10C9C800E443264006600E79D0F8009006FA03FA90
:10C9D800013E4AEA0909012EC0F8009014D8866879
:10C9E80091F8059026408660866809FA03F949EAB5
:10C9F80006068660466826EA050545608D7946681C
:10CA08009540ADB235434560C5682C40C460CC79CB
:10CA1800C5689C402C43C46001320233102AC6D139
:10CA2800BDE8F0874FF6FF7303600023037143717D
:10CA38008371C371704782B04FF480330193019BB7
:10CA48000B430193019BC361C161019BC361C3692E
:10CA58000193C369019302B07047036919420CBF7F
:10CA6800002001207047006980B27047436919426D
:10CA78000CBF002001207047406980B270470183D5
:10CA88007047418370470AB10183704741837047FB
:10CA98004161704743694B404361704701F00703A8
:10CAA800C908083130B59B0050F821500F249C402C
:10CAB80025EA040440F8214050F8214012FA03F313
:10CAC8001C4340F8214030BD08B5134B984207D1AC
:10CAD8004FF40010012100F069FB4FF4001014E03E
:10CAE8000E4B984207D14FF48000012100F05EFB05
:10CAF8004FF4800009E00A4B98420BD14FF4000034
:10CB0800012100F053FB4FF400000021BDE808406C
:10CB180000F04CBB08BD00BF005400400058004066
:10CB2800005C00407FB50446868868460D4600F0E4
:10CB38006DFA02992C482B6826F03F063604B1FBA3
:10CB4800F0F0360C80B20643A680228822F001025B
:10CB58001204120C2280254A93420AD85B00B1FBCA
:10CB6800F3F301309BB280B22084032B98BF0423D7
:10CB780021E0EE884BF6FF72964205D1032253431B
:10CB8800B1FBF3F39BB206E019225343B1FBF3F375
:10CB98009BB243F480431A054FF4967208BF43F0E2
:10CBA800010350434FF47A7290FBF2F0013080B2E7
:10CBB80043F400432084A38323886989AA889BB20D
:10CBC80043F001032380238823F4816323F00203C5
:10CBD8001B040A431B0C13439BB223802A89AB898D
:10CBE80013439BB223817FBD40420F00A086010002
:10CBF80041F288330360002383804BF6FF72038180
:10CC080043814FF48043C28083817047038819B100
:10CC18009BB243F0010303E023F001031B041B0C48
:10CC280003807047038819B19BB243F4807303E013
:10CC380023F480731B041B0C03807047038819B10D
:10CC48009BB243F4007303E023F400731B041B0C32
:10CC58000380704712B141F0010101E001F0FE01CB
:10CC680001827047038819B19BB243F4806303E0E3
:10CC780023F480631B041B0C0380704783899BB2D9
:10CC880001F0FE0123F0FE030B4383817047838983
:10CC980019B19BB243F0010303E023F001031B0425
:10CCA8001B0C83817047038819B19BB243F0400382
:10CCB80003E023F040031B041B0C03807047038828
:10CCC80029B16FEA43436FEA53439BB201E05B0427
:10CCD8005B0C03807047038819B99BB243F080034B
:10CCE80003E023F080031B041B0C03807047B1F59D
:10CCF800804F838B04D023F480431B041B0C02E079
:10CD08009BB243F4804383837047B1F5006F038877
:10CD180003D19BB243F4006303E023F400631B04D4
:10CD28001B0C03807047B1F5005F038803D19BB2E9
:10CD380043F4005303E023F400531B041B0C03804B
:10CD48007047038819B19BB243F0100303E023F046
:10CD580010031B041B0C0380704701827047008A74
:10CD6800C0B27047038819B19BB243F4805303E003
:10CD780023F480531B041B0C03807047B1F5006F2C
:10CD8800038803D19BB243F4006303E023F40063F8
:10CD98001B041B0C03807047038819B19BB243F036
:10CDA800200303E023F020031B041B0C03807047BF
:10CDB800008BC0F307207047838819B19BB243F4F6
:10CDC800006303E023F400631B041B0C838070479B
:10CDD800838819B19BB243F4805303E023F4805352
:10CDE8001B041B0C8380704782B0002301930190C1
:10CDF800019BCB180193019B188880B202B0704741
:10CE080083889BB20AB1194301E023EA01018180BA
:10CE18007047838A008B9BB243EA0040084020F0A9
:10CE28007F40431A584240EB03007047838A008BC7
:10CE38009BB243EA004020F07F40704782B0002355
:10CE4800009301930B0F01900093009B21F07F4109
:10CE580013B1019B143302E0019B090C18330193B1
:10CE6800019B1B6819420CBF0020012002B07047CB
:10CE7800C94389B2818270478388808A80B208401A
:10CE88009BB206D001F0E06113EA11410CBF00200B
:10CE980001207047C94389B2818270470A4B1A68DA
:10CEA80042F001021A6000229A60196821F0847128
:10CEB80021F48031196005495960196821F48021ED
:10CEC8001960DA60704700BF003802401030002453
:10CED800024B00221A701870704700BF02380240D7
:10CEE800034B1A6822F0F80242EAC0021A6070473F
:10CEF80000380240014B1860704700BF00004742ED
:10CF0800064B002201281A701A7002D0042804D196
:10CF180001E01870704705221A7070477038024097
:10CF2800014B1860704700BF800E4742014341EA39
:10CF3800821200995B08013B42EA016141EA034120
:10CF4800014B5960704700BF00380240014B186020
:10CF5800704700BF600047428001034B40EA0171FF
:10CF6800C3F88410704700BF00380240014B1860B6
:10CF7800704700BF68004742014B1860704700BF08
:10CF88004C004742034B9A6822F0EC6202430A4382
:10CF98009A60704700380240034B9A6822F0784242
:10CFA80002430A439A60704700380240034B9A686C
:10CFB80022F0030202439A60704700BF0038024023
:10CFC800024B986800F00C00704700BF0038024020
:10CFD800034B9A6822F0F00202439A60704700BF40
:10CFE80000380240034B9A6822F4E05202439A60E8
:10CFF800704700BF00380240034B9A6822F4604231
:10D0080042EAC0029A607047003802401E4B9A6894
:10D0180002F00C02042A10B503D0082A03D01B4BD7
:10D0280018E01B4B16E059685A6811F4800F5968CC
:10D0380014BF174B154B02F03F02B3FBF2F3124A31
:10D048005268C2F30142C1F3881101324B435200C6
:10D05800B3FBF2F30C4903608B680E4A0468C3F310
:10D068000313D35C34FA03F343608C68C4F382245B
:10D07800145D33FA04F484608968C1F34231525C68
:10D08800D340C36010BD00BF003802400024F40044
:10D0980000127A003C02002000F44073B3F5407F90
:10D0A800084B08D1996820F0704221F4F81122F455
:10D0B80040720A439A601A6F000542EA10501867D6
:10D0C800704700BF00380240014B1860704700BF2E
:10D0D8003C0E4742014B1860704700BF400E474264
:10D0E800014B1860704700BF5C014742044B1A6B44
:10D0F80009B1104301E022EA00001863704700BF3D
:10D1080000380240044B5A6B09B1104301E022EA8F
:10D1180000005863704700BF00380240044B9A6B08
:10D1280009B1104301E022EA00009863704700BF8C
:10D1380000380240044B1A6C09B1104301E022EA9E
:10D1480000001864704700BF00380240044B5A6C56
:10D1580009B1104301E022EA00005864704700BF9B
:10D1680000380240044B1A6909B1104301E022EA71
:10D1780000001861704700BF00380240044B5A692C
:10D1880009B1104301E022EA00005861704700BF6E
:10D1980000380240044B9A6909B1104301E022EAC1
:10D1A80000009861704700BF00380240044B1A6ABB
:10D1B80009B1104301E022EA00001862704700BF7D
:10D1C80000380240044B5A6A09B1104301E022EAD0
:10D1D80000005862704700BF00380240044B1A6DC7
:10D1E80009B1104301E022EA00001865704700BF4A
:10D1F80000380240044B5A6D09B1104301E022EA9D
:10D2080000005865704700BF00380240044B9A6D13
:10D2180009B1104301E022EA00009865704700BF99
:10D2280000380240044B1A6E09B1104301E022EAAB
:10D2380000001866704700BF00380240044B5A6E61
:10D2480009B1104301E022EA00005866704700BFA8
:10D2580000380240044B1A7809B1104301E022EA71
:10D2680000001870704700BF0D3802404309012BB9
:10D27800074A01D1136803E0022B0CBF136F536FE9
:10D2880000F01F0033FA00F000F00100704700BF03
:10D298000038024007B5002301933120FFF7E6FF6D
:10D2A800019B01330193019BB3F5A06F01D00028C6
:10D2B800F3D03120FFF7DAFF003018BF01200EBD90
:10D2C800024B5A6F42F080725A677047003802402A
:10D2D800034BDB6818420CBF00200120704700BFD9
:10D2E80000380240014B1870704700BF0E380240EA
:10D2F80008B5154B98420BD101214FF48050FFF728
:10D3080061FF4FF480500021BDE80840FFF75ABF85
:10D318000E4B984207D14FF480400121FFF746FF9A
:10D328004FF4804009E00A4B98420BD14FF400407B
:10D338000121FFF73BFF4FF400400021BDE8084002
:10D34800FFF734BF08BD00BF00300140003800407F
:10D35800003C00400B88028810B54C8823438C8819
:10D368002343CC8823430C8923434C8923438C894A
:10D378002343CC8902F44152234313439BB20380D5
:10D38800838B23F400631B041B0C83830B8A0382A7
:10D3980010BD838B23F47B6323F00F031B041B0C4A
:10D3A8008383022303848B68F0B5858B022BADB28F
:10D3B80038D0294A8E889468002E14BF0226012688
:10D3C800240203D5946824F400049460D2F88440BD
:10D3D800D2F884705268DFF884C002F03F02BCFBC8
:10D3E800F2F2C4F388145443C7F30272B4FBF2F4A4
:10D3F800CA88B2F5007F4FF00A0201D1240A02E080
:10D408007601B4FBF6F46243B2FBF3F305330A2268
:10D418009BB2B3FBF2F303F001021202C3F34F0312
:10D4280092B200E000229C1EA4B2FE2C28BF00226B
:10D43800CC8828BF0223134323439BB203840B8861
:10D448004A882B4343F4006313438A8813438A8929
:10D4580013439BB28383F0BD0038024000127A0068
:10D468000023038043808380C380038143818381B9
:10D47800C38107230382704700230222038043806D
:10D488008380C380826083817047038819B19BB20F
:10D4980043F0400303E023F040031B041B0C03800C
:10D4A8007047838B19B19BB243F4806303E023F484
:10D4B80080631B041B0C83837047038823F4006379
:10D4C8001B041B0C038003889BB20B43038070472B
:10D4D800B1F5804F038803D19BB243F4804303E046
:10D4E80023F480431B041B0C038070474FF6FF6333
:10D4F8009942038803D09BB243F4807303E023F47A
:10D5080080731B041B0C03807047838819B19BB27E
:10D5180043F0040303E023F004031B041B0C838083
:10D528007047838819B19BB243F0100303E023F0DE
:10D5380010031B041B0C83807047838B23F47B63CD
:10D5480023F00F031B041B0C8383022303840B8823
:10D55800828BB3F5007F10B592B205D0002B0CBFBB
:10D568004FF48073002301E04FF480734C8822430A
:10D578008C88898942F4006222430A4392B2134399
:10D58800838310BD808980B270478181704703888A
:10D5980019B19BB243F4005303E023F400531B0476
:10D5A8001B0C0380704703889BB243F480530380AD
:10D5B8007047012902D0008B80B27047808A80B200
:10D5C8007047008A80B2704783889BB20AB11943BA
:10D5D80001E023EA010181807047090901238B409A
:10D5E8009BB21AB1828892B2134303E0828892B246
:10D5F80022EA030383807047038919420CBF002085
:10D6080001207047C94389B20181704710B58488E9
:10D618000089012301F00F0280B213FA02F21040D0
:10D62800A4B205D009098B401C420CBF0020012080
:10D6380010BD01F00F0101238B40DB439BB2038136
:10D64800704700BF08B501214FF48040FFF7BAFDCD
:10D658004FF480400021BDE80840FFF7B3BD014BFF
:10D66800186070470038014001F0030289080A4B2E
:10D67800023130B5920053F821500F24944025EA26
:10D68800040443F8214053F8214010FA02F21443ED
:10D6980043F8214030BD00BF00380140014B1860FD
:10D6A800704700BFDC002742014B1860704700BF7D
:10D6B80000042742024B186AC0F30020704700BFDD
:10D6C8000038014030B5048C24F001042404240CF3
:10D6D8000484058B048CADB2A4B225F0F305154380
:10D6E80024F00A0445EA031544F00104ADB20C43E2
:10D6F8000583048430BD30B5048C24F01004240460
:10D70800240C0484048B058C24F44074ADB22405E5
:10D71800240D25F0A00544EA022445F0100544EA4A
:10D72800033445EA0115A4B2ADB20483058430BDC3
:10D7380008B5474B984205D101200146FFF742FD45
:10D7480001203DE0B0F1804F05D101200146FFF7EF
:10D758002DFD012076E03F4B984205D102200121A2
:10D76800FFF724FD02206DE03B4B984205D10420D1
:10D778000121FFF71BFD042064E0384B984205D1D6
:10D7880008200121FFF712FD08205BE0344B984286
:10D7980005D110200121FFF709FD102052E0314B7F
:10D7A800984205D120200121FFF700FD202049E003
:10D7B8002D4B984209D102200121FFF703FD0220D9
:10D7C8000021BDE80840FFF7FDBC284B984207D16F
:10D7D8004FF480300121FFF7F5FC4FF48030EFE77C
:10D7E800234B984207D14FF400300121FFF7EAFCA0
:10D7F8004FF40030E4E71F4B984207D14FF48020E4
:10D808000121FFF7DFFC4FF48020D9E71A4B98423B
:10D8180005D140200121FFF7C9FC402012E0174B39
:10D82800984205D180200121FFF7C0FC802009E043
:10D83800134B98420BD14FF480700121FFF7B6FCCF
:10D848004FF480700021BDE80840FFF7AFBC08BD69
:10D85800000001400004004000080040000C0040A7
:10D868000010004000140040000401400040014046
:10D87800004401400048014000180040001C0040DE
:10D88800002000401C4A038890429BB212D002F547
:10D89800806290420ED0B0F1804F0BD0A2F580325A
:10D8A800904207D002F58062904203D002F5806270
:10D8B800904203D14A8823F0700313430F4A9042E1
:10D8C80008D002F58062904204D023F440730A899C
:10D8D8009BB2134303804B68C3620B880385064BD6
:10D8E800984203D003F58063984201D18B7A03866E
:10D8F80001238382704700BF0000014000100040F0
:10D908004FF0FF3343600023038003814380837219
:10D918007047018582827047038823F070031B04D7
:10D928001B0C0B430380704741627047C16270470C
:10D93800406A7047008D80B27047038819B19BB266
:10D9480043F0020303E023F002031B041B0C0380D3
:10D958007047038819B19BB243F0040303E023F036
:10D9680004031B041B0C03807047038819B19BB286
:10D9780043F0800303E023F080031B041B0C0380A7
:10D988007047038823F008031B041B0C03800388DB
:10D998009BB20B4303807047038823F440731B0436
:10D9A8001B0C038003889BB20B43038070470388DA
:10D9B80019B19BB243F0010303E023F001031B04F8
:10D9C8001B0C03807047038C23F001031B041B0C02
:10D9D800038470B5038C8488028B0D884E8822F0EE
:10D9E80073021204120C2A438D8923F002031B04CC
:10D9F80035431B0CADB22B430E4DA842A4B203D045
:10DA080005F58065A8420ED1CD894E8A23F008031A
:10DA18002B438D8823F004032B430D8A354324F4CC
:10DA28004074ADB22C43848002838A6842630384C5
:10DA380070BD00BF00000140038C23F010031B04DD
:10DA48001B0C0384038C828830B5048B0D8824F466
:10DA5800E6442404240C23F0200344EA05241B0490
:10DA68008D891B0C43EA05134D8843EA0513134DB2
:10DA7800A84292B2A4B29BB203D005F58065A84231
:10DA880015D1CD8923F080039BB243EA05134FF6E5
:10DA9800BF751D408B8845EA03130D8A22F4406246
:10DAA80042EA85024D8A42EA85029BB292B282809E
:10DAB8008A6804838263038430BD00BF000001408C
:10DAC800038C23F480731B041B0C0384038C82884F
:10DAD80030B5848B0D8824F073042404240C23F4BB
:10DAE80000731B042C438D891B0C43EA05234D88C6
:10DAF80043EA0523124DA84292B29BB203D005F522
:10DB08008065A84215D1CD8923F400639BB243EA0E
:10DB180005234FF6FF351D408B8845EA03230D8A00
:10DB280022F4405242EA05124D8A42EA05129BB29B
:10DB380092B282808A688483C263038430BD00BF46
:10DB480000000140038C23F480531B041B0C038446
:10DB5800038C30B58488828B0D8822F4E642120447
:10DB6800120C23F4005342EA05221B048D891B0C76
:10DB780043EA05334D8843EA05330B4DA842A4B266
:10DB880092B29BB203D005F58065A84205D10D8AF3
:10DB980024F4804444EA8514A4B2848082838A6889
:10DBA8000264038430BD00BF0000014000230380ED
:10DBB8004380838083608381C3810382438270476B
:10DBC80030B5058C0124ADB28C4025EA040400F17F
:10DBD8001803048409B1082907D149084FF68F7042
:10DBE800CC582040C850C8580AE00439C1F34E0147
:10DBF80048F6FF70CC582040C8501202C85892B25C
:10DC08000243CA5030BD4163704781637047C163A6
:10DC1800704701647047038B23F070031B041B0CCF
:10DC28000B4303837047038B23F4E0431B041B0C53
:10DC380043EA01239BB203837047838B23F070036D
:10DC48001B041B0C0B4383837047838B23F4E04333
:10DC58001B041B0C43EA01239BB283837047038B8D
:10DC680023F008031B041B0C0B4303837047038B2F
:10DC780023F400631B041B0C43EA01239BB20383B8
:10DC88007047838B23F008031B041B0C0B4383830F
:10DC98007047838B23F400631B041B0C43EA0123A6
:10DCA8009BB283837047038B23F004031B041B0C74
:10DCB8000B4303837047038B23F480631B041B0C03
:10DCC80043EA01239BB203837047838B23F0040349
:10DCD8001B041B0C0B4383837047838B23F48063E3
:10DCE8001B041B0C43EA01239BB283837047038BFD
:10DCF80023F080031B041B0C0B4303837047038B27
:10DD080009025B0441EA53439BB203837047838B48
:10DD180023F080031B041B0C0B4383837047838B06
:10DD280009025B0441EA53439BB283837047038C27
:10DD380023F002031B041B0C0B4303847047038C62
:10DD480023F008031B041B0C0B4303847047038C4C
:10DD580023F020031B041B0C43EA01139BB203842A
:10DD68007047038C23F080031B041B0C43EA011348
:10DD78009BB203847047038C23F400731B041B0CB1
:10DD880043EA01239BB203847047038C23F40063A6
:10DD98001B041B0C43EA01239BB203847047038CCA
:10DDA80023F400531B041B0C43EA01339BB2038486
:10DDB800704710B5048C01238B40A4B224EA0303F6
:10DDC8000384038C12FA01F10B439BB2038410BD48
:10DDD80010B5048C04238B40A4B224EA0303038403
:10DDE800038C12FA01F10B439BB2038410BD00238C
:10DDF8000122038043808280C38003817047406B87
:10DE08007047806B7047C06B7047006C7047038B1E
:10DE180023F00C031B041B0C0383038B9BB20B43E3
:10DE280003837047038B23F440631B041B0C038399
:10DE3800038B9BB243EA01239BB203837047F8B577
:10DE48000C464988A288B4F800E0238905460029D1
:10DE58000CBF02270027012A14BF01260226BEF1A3
:10DE6800000F10D1FFF72EFC2846E188FFF7CFFFFF
:10DE78002846394632462389FFF73DFCE188284683
:10DE8800BDE8F840CEE7FFF736FC2846E188FFF703
:10DE9800C9FF2846394632462389FFF713FCE18833
:10DEA8002846BDE8F840B2E7838B23F00C031B0437
:10DEB8001B0C8383838B9BB20B4383837047838BB9
:10DEC80023F440631B041B0C8383838B9BB243EABC
:10DED80001239BB283837047F8B50D460B88AA8847
:10DEE800498804463BB92B89FFF7ECFBE9882046B3
:10DEF800BDE8F8408BE7042B07D12B89FFF7FBFB24
:10DF0800E9882046BDE8F8408CE7082BB5F808C03A
:10DF1800078C1DD127F480773F043F0C0784868B3C
:10DF2800038CB6B29BB226F0F30623F4206346EACC
:10DF38000C1C43EA01211FFA8CFC89B24CEA02024C
:10DF480041F4807182830184E988BDE8F840ABE739
:10DF580027F480573F043F0C0784868B038C26F4F4
:10DF6800407623F4005336055B04360D5B0C46EA15
:10DF7800022243EA013342EA0C329BB2E98892B2A8
:10DF880043F4805382830384BDE8F84097E74A88C6
:10DF98000B8813438A881343CA8813430A89134397
:10DFA8004A8913438A8913439BB2A0F844307047C7
:10DFB8000023038043808380C3800381438183815E
:10DFC8007047B0F8443029B16FEA43436FEA5343CE
:10DFD8009BB201E05B045B0CA0F844307047838877
:10DFE80019B19BB243F0040303E023F004031B04BC
:10DFF8001B0C83807047838819B19BB243F00103DF
:10E0080003E023F001031B041B0C83807047838902
:10E018009BB20AB1194301E023EA010181817047EB
:10E0280081827047038A19420CBF00200120704783
:10E03800C94389B201827047038A828911EA0300C1
:10E0480092B203D011420CBF002001207047C9438F
:10E0580089B2018270470A43A0F848207047838933
:10E068009BB20AB1194301E023EA0101818170479B
:10E07800838819B19BB243F0080303E023F0080337
:10E088001B041B0C83807047038923F007031B04C0
:10E098001B0C03817047038923F070031B041B0CBE
:10E0A8000B43038103899BB243F007030381704745
:10E0B80038B50D4611460122602D044602D1FFF7FE
:10E0C8001AFB01E0FFF7FEFA238923F070031B0413
:10E0D8001B0C1D43258123899BB243F00703238131
:10E0E80038BD038923F070031B041B0C0B43038109
:10E0F8007047838823F070031B041B0C838083887C
:10E108009BB20B4383807047038923F007031B04EA
:10E118001B0C038103899BB20B430381704703895E
:10E1280023F080031B041B0C038103899BB20B4360
:10E138000381704710B50489E4B20C43144344EAE0
:10E148000324A4B2048110BD10B50446FFF7F2FF02
:10E1580023899BB243F48043238110BD10B5044644
:10E16800FFF7E8FF238923F077031B041B0C43F018
:10E178007703238110BD70B50489068B058C26F4BE
:10E188004076ADB226F0030624F00704360425F0E5
:10E1980022052404360C1543240C46F4807645EAFF
:10E1A8000315214346F00106ADB2018106830584BB
:10E1B80070BD838819B19BB243F0800303E023F05C
:10E1C80080031B041B0C83807047A0F85010704715
:10E1D80008B5234B984205D110200121FEF7F2FF24
:10E1E800102037E01F4B984207D14FF4003001212F
:10E1F800FEF7DCFF4FF4003009E01B4B98420BD1CF
:10E208004FF480200121FEF7D1FF4FF48020002138
:10E21800BDE80840FEF7CABF144B984207D14FF437
:10E2280000200121FEF7C2FF4FF40020EFE7104B5A
:10E23800984207D14FF480100121FEF7B7FF4FF441
:10E248008010E4E70B4B984209D120200121FEF70A
:10E25800B9FF20200021BDE80840FEF7B3BF08BD84
:10E26800001001400044004000480040004C0040BD
:10E278000050004000140140038ACA889BB223F46E
:10E28800405330B513430D46038283890989AA8810
:10E2980023F4B0530A43698923F00C031B040A438F
:10E2A8001B0C92B213438381838AAA899BB223F4FD
:10E2B8004073134385B0838204466846FEF7A6FE82
:10E2C8001A4B9C4203D003F580639C4201D1039B07
:10E2D80000E0029BA28912B2002A4FF019012A68B5
:10E2E80001FB03F101DA520000E092006423B1FB64
:10E2F800F2F1B1FBF3F21201100903FB1011A0892E
:10E3080000B2002806DAC9003231B1FBF3F303F09A
:10E31800070305E009013231B1FBF3F303F00F0302
:10E328001A4392B2228105B030BD00BF00100140EF
:10E338004FF4165303600C2200238380C3800381AB
:10E348004281838170470B88028A10B54C88234329
:10E358008C88C988234392B20B4322F470629BB223
:10E368001343038210BD0023038043808380C3804E
:10E378007047838919B19BB243F4005303E023F437
:10E3880000531B041B0C83817047038B03F47F43EA
:10E398000383038B9BB20B4303837047838929B1A3
:10E3A8006FEA43436FEA53439BB201E05B045B0CA3
:10E3B80083817047838A19B19BB243F4006303E0F9
:10E3C80023F400631B041B0C83827047C905C90D25
:10E3D800818070478088C005C00D7047038A23F08C
:10E3E8000F031B041B0C0382038A9BB20B4303829B
:10E3F8007047838919B19BB243F0020303E023F00D
:10E4080002031B041B0C83817047838923F4006378
:10E418001B041B0C838183899BB20B438381704748
:10E42800038A23F020031B041B0C0382038A9BB27C
:10E438000B4303827047038A19B19BB243F48043AC
:10E4480003E023F480431B041B0C03827047838979
:10E458009BB243F0010383817047838A19B19BB251
:10E4680043F0080303E023F008031B041B0C83821A
:10E478007047038BDBB20383038B9BB243EA012310
:10E4880003837047838A19B19BB243F0200303E0EA
:10E4980023F020031B041B0C83827047838A19B165
:10E4A8009BB243F0100303E023F010031B041B0C82
:10E4B80083827047838A23F004031B041B0C838226
:10E4C800838A9BB20B4383827047838A19B19BB2BC
:10E4D80043F0020303E023F002031B041B0C8382B6
:10E4E8007047838A9BB20AB1194301E023EA01010C
:10E4F80081827047C1F3421310B501F01F01012456
:10E5080014FA01F1A34201D10C3004E0022B01D12D
:10E51800103000E0143003680AB1194301E023EA1F
:10E528000101016010BD038819420CBF00200120C1
:10E538007047C94389B201807047012210B501F0C4
:10E548001F03C1F342149A40012C01D1838903E0CF
:10E55800022C0CBF038A838A9BB21340028892B2B2
:10E5680043B1090A012313FA01F111420CBF00203B
:10E57800012010BD184610BD090A01238B40DB435A
:10E588009BB20380704700BF81F0004102E000BFEA
:10E5980083F0004330B54FEA41044FEA430594EA5B
:10E5A800050F08BF90EA020F1FBF54EA000C55EA96
:10E5B800020C7FEA645C7FEA655C00F0E2804FEA67
:10E5C8005454D4EB5555B8BF6D420CDD2C4480EA49
:10E5D800020281EA030382EA000083EA010180EA79
:10E5E800020281EA0303362D88BF30BD11F0004FC7
:10E5F8004FEA01314FF4801C4CEA113102D04042FD
:10E6080061EB410113F0004F4FEA03334CEA133337
:10E6180002D0524263EB430394EA050F00F0A7804F
:10E62800A4F10104D5F1200E0DDB02FA0EFC22FA4A
:10E6380005F2801841F1000103FA0EF2801843FA3E
:10E6480005F359410EE0A5F120050EF1200E012A2F
:10E6580003FA0EFC28BF4CF0020C43FA05F3C0186D
:10E6680051EBE37101F0004507D54FF0000EDCF1E6
:10E67800000C7EEB00006EEB0101B1F5801F1BD38F
:10E68800B1F5001F0CD349085FEA30004FEA3C0C93
:10E6980004F101044FEA445212F5800F80F09A8089
:10E6A800BCF1004F08BF5FEA500C50F1000041EB8D
:10E6B800045141EA050130BD5FEA4C0C404141EB91
:10E6C800010111F4801FA4F10104E9D191F0000FB8
:10E6D80004BF01460020B1FA81F308BF2033A3F13B
:10E6E8000B03B3F120020CDA0C3208DD02F1140C32
:10E6F800C2F10C0201FA0CF021FA02F10CE002F16D
:10E708001402D8BFC2F1200C01FA02F120FA0CFC65
:10E71800DCBF41EA0C019040E41AA2BF01EB0451AE
:10E72800294330BD6FEA04041F3C1CDA0C340EDCAC
:10E7380004F11404C4F1200220FA04F001FA02F3EF
:10E7480040EA030021FA04F345EA030130BDC4F1AD
:10E758000C04C4F1200220FA02F001FA04F340EAA2
:10E768000300294630BD21FA04F0294630BD94F053
:10E77800000F83F4801306BF81F480110134013D3A
:10E788004EE77FEA645C18BF7FEA655C29D094EAAB
:10E79800050F08BF90EA020F05D054EA000C04BF29
:10E7A8001946104630BD91EA030F1EBF0021002014
:10E7B80030BD5FEA545C05D14000494128BF41F0B3
:10E7C800004130BD14F580043CBF01F5801130BD17
:10E7D80001F0004545F0FE4141F470014FF00000A2
:10E7E80030BD7FEA645C1ABF194610467FEA655C53
:10E7F8001CBF0B46024650EA013406BF52EA0335F5
:10E8080091EA030F41F4002130BD00BF90F0000FE2
:10E8180004BF0021704730B54FF4806404F132041E
:10E828004FF000054FF0000150E700BF90F0000FD7
:10E8380004BF0021704730B54FF4806404F13204FE
:10E8480010F0004548BF40424FF000013EE700BFCE
:10E8580042004FEAE2014FEA31014FEA02701FBF5E
:10E8680012F07F4393F07F4F81F06051704792F030
:10E87800000F14BF93F07F4F704730B54FF46074AA
:10E8880001F0004521F0004120E700BF50EA0102F5
:10E8980008BF704730B54FF000050AE050EA0102A2
:10E8A80008BF704730B511F0004502D5404261EB12
:10E8B80041014FF4806404F132045FEA915C3FF453
:10E8C800DCAE4FF003025FEADC0C18BF03325FEAEC
:10E8D800DC0C18BF033202EBDC02C2F1200300FAA1
:10E8E80003FC20FA02F001FA03FE40EA0E0021FAC6
:10E8F80002F11444C1E600BF70B54FF0FF0C4CF4B0
:10E90800E06C1CEA11541DBF1CEA135594EA0C0F65
:10E9180095EA0C0F00F0DEF82C4481EA030621EAA0
:10E928004C5123EA4C5350EA013518BF52EA0335DB
:10E9380041F4801143F4801338D0A0FB02CE4FF08D
:10E948000005E1FB02E506F00042E0FB03E54FF0BD
:10E958000006E1FB03569CF0000F18BF4EF0010EB5
:10E96800A4F1FF04B6F5007F64F5407404D25FEAB1
:10E978004E0E6D4146EB060642EAC62141EA555164
:10E988004FEAC52040EA5E504FEACE2EB4F1FD0CA6
:10E9980088BFBCF5E06F1ED8BEF1004F08BF5FEA24
:10E9A800500E50F1000041EB045170BD06F00046D6
:10E9B80046EA010140EA020081EA0301B4EB5C0483
:10E9C800C2BFD4EB0C0541EA045170BD41F480117B
:10E9D8004FF0000E013C00F3AB8014F1360FDEBFA0
:10E9E800002001F0004170BDC4F10004203C35DA7C
:10E9F8000C341BDC04F11404C4F1200500FA05F3FF
:10EA080020FA04F001FA05F240EA020001F000429F
:10EA180021F0004110EBD37021FA04F642EB060115
:10EA28005EEA430E08BF20EAD37070BDC4F10C043F
:10EA3800C4F1200500FA04F320FA05F001FA04F203
:10EA480040EA020001F0004110EBD37041F10001EF
:10EA58005EEA430E08BF20EAD37070BDC4F12005FA
:10EA680000FA05F24EEA020E20FA04F301FA05F262
:10EA780043EA020321FA04F001F0004121FA04F20A
:10EA880020EA020000EBD3705EEA430E08BF20EADA
:10EA9800D37070BD94F0000F0FD101F00046400014
:10EAA80041EB010111F4801F08BF013CF7D041EA96
:10EAB800060195F0000F18BF704703F0004652009A
:10EAC80043EB030313F4801F08BF013DF7D043EA6B
:10EAD8000603704794EA0C0F0CEA135518BF95EA21
:10EAE8000C0F0CD050EA410618BF52EA4306D1D1A8
:10EAF80081EA030101F000414FF0000070BD50EAC7
:10EB0800410606BF1046194652EA430619D094EA50
:10EB18000C0F02D150EA013613D195EA0C0F05D13A
:10EB280052EA03361CBF104619460AD181EA03018E
:10EB380001F0004141F0FE4141F470014FF0000046
:10EB480070BD41F0FE4141F4780170BD70B54FF0E1
:10EB5800FF0C4CF4E06C1CEA11541DBF1CEA135561
:10EB680094EA0C0F95EA0C0F00F0A7F8A4EB050443
:10EB780081EA030E52EA03354FEA013100F088803A
:10EB88004FEA03334FF0805545EA131343EA126303
:10EB98004FEA022245EA111545EA10654FEA0026B8
:10EBA8000EF000419D4208BF964244F1FD0404F571
:10EBB800407402D25B084FEA3202B61A65EB0305CD
:10EBC8005B084FEA32024FF480104FF4002CB6EB8A
:10EBD800020E75EB030E22BFB61A754640EA0C000A
:10EBE8005B084FEA3202B6EB020E75EB030E22BF4A
:10EBF800B61A754640EA5C005B084FEA3202B6EB8B
:10EC0800020E75EB030E22BFB61A754640EA9C0049
:10EC18005B084FEA3202B6EB020E75EB030E22BF19
:10EC2800B61A754640EADC0055EA060E18D04FEAD7
:10EC3800051545EA16754FEA06164FEAC30343EA77
:10EC480052734FEAC2025FEA1C1CC0D111F4801F44
:10EC58000BD141EA00014FF000004FF0004CB6E73D
:10EC680011F4801F04BF01430020B4F1FD0C88BFDC
:10EC7800BCF5E06F3FF6AFAEB5EB030C04BFB6EBE7
:10EC8800020C5FEA500C50F1000041EB045170BDDA
:10EC98000EF0004E4EEA113114EB5C04C2BFD4EB07
:10ECA8000C0541EA045170BD41F480114FF0000E8B
:10ECB800013C90E645EA060E8DE60CEA135594EA07
:10ECC8000C0F08BF95EA0C0F3FF43BAF94EA0C0F0A
:10ECD8000AD150EA01347FF434AF95EA0C0F7FF47F
:10ECE80025AF104619462CE795EA0C0F06D152EAD3
:10ECF80003353FF4FDAE1046194622E750EA4106B7
:10ED080018BF52EA43067FF4C5AE50EA41047FF4C7
:10ED18000DAF52EA43057FF4EBAE12E74FF0FF3C2C
:10ED280006E000BF4FF0010C02E000BF4FF0010CFD
:10ED38004DF804CD4FEA410C7FEA6C5C4FEA430C76
:10ED480018BF7FEA6C5C1BD001B050EA410C0CBFC5
:10ED580052EA430C91EA030F02BF90EA020F002027
:10ED6800704710F1000F91EA030F58BF994208BF8E
:10ED780090422CBFD8176FEAE37040F0010070474B
:10ED88004FEA410C7FEA6C5C02D150EA013C07D1A2
:10ED98004FEA430C7FEA6C5CD6D152EA033CD3D0ED
:10EDA8005DF8040B704700BF8446104662468C46E7
:10EDB8001946634600E000BF01B5FFF7B7FF00281A
:10EDC80048BF10F1000F01BD4DF808EDFFF7F4FF43
:10EDD8000CBF012000205DF808FB00BF4DF808EDCE
:10EDE800FFF7EAFF34BF012000205DF808FB00BFF1
:10EDF8004DF808EDFFF7E0FF94BF012000205DF813
:10EE080008FB00BF4DF808EDFFF7CEFF94BF0120C7
:10EE180000205DF808FB00BF4DF808EDFFF7C4FFC0
:10EE280034BF012000205DF808FB00BF4FEA410213
:10EE380012F5001215D211D56FF47873B3EB625244
:10EE480012D94FEAC12343F0004343EA505311F06B
:10EE5800004F23FA02F018BF404270474FF00000FD
:10EE6800704750EA013005D111F0004008BF6FF03B
:10EE7800004070474FF00000704700BF4A0011D2B1
:10EE880012F5001211D20DD56FF47873B3EB6252FC
:10EE98000ED44FEAC12343F0004343EA505323FA08
:10EEA80002F070474FF00000704750EA013002D17D
:10EEB8004FF0FF3070474FF0000070474FEA4102B3
:10EEC800B2F1E04324BFB3F5001CDCF1FE5C0DD9C0
:10EED80001F0004C4FEAC0024CEA5070B2F1004F0A
:10EEE80040EB830008BF20F00100704711F0804F0D
:10EEF80021D113F13872BCBF01F00040704741F4D2
:10EF080080114FEA5252C2F11802C2F1200C10FAD5
:10EF18000CF320FA02F018BF40F001004FEAC123B9
:10EF28004FEAD32303FA0CFC40EA0C0023FA02F35D
:10EF38004FEA4303CCE77FEA625307D150EA013333
:10EF48001EBF4FF0FE4040F44000704701F0004003
:10EF580040F0FE4040F40000704700BF4BB942B992
:10EF6800002908BF002802D04FF0FF31084600F002
:10EF780037B882B0EC462DE9005000F01BF8DDF8F8
:10EF880004E002B00CBC7047F8B5144606460F46BC
:10EF98001D4600F027F804FB01F300FB0535A4FB30
:10EFA8000023EB18069CB21A67EB0303C4E900239D
:10EFB800F8BD00BFF8B5144606460F461D4600F0DA
:10EFC80075F900FB05F5A0FB042304FB0155EB18BC
:10EFD800069CB21A67EB0303C4E90023F8BD00BF1F
:10EFE800704700BF00292DE9F0071D46C0F29E803A
:10EFF8000024002DC0F2958007460D4616469C4613
:10F00800002B3ED18A4254D9B2FA82F343B1C3F1FC
:10F01800200620FA06F501FA03F19A4029439840A0
:10F02800160CB1FBF6F597B206FB15114FEA104C1A
:10F0380007FB05F34CEA01418B4209D9891805F110
:10F04800FF3C80F015818B4240F21281023D891805
:10F05800C3EB010CBCFBF6F306FB13C180B207FB44
:10F0680003F740EA0140874207D9591E821880F009
:10F078000581974240F20281023B43EA05420023A0
:10F0880003E08B420AD900231A461046194614B1E8
:10F09800404261EB4101BDE8F0077047B3FA83F3E2
:10F0A800002B40F087808C4501D38242ECD80122A6
:10F0B800EBE712B90123B3FBF2F2B2FA82F6002EA3
:10F0C8003AD1891A150C1FFA82FC0123B1FBF5F716
:10F0D80005FB17114FEA10480CFB07F648EA0141F7
:10F0E8008E4207D9891807F1FF3802D28E4200F202
:10F0F800DA804746891BB1FBF5F605FB161180B28D
:10F108000CFB06FC40EA0140844507D9711E8218B1
:10F1180080F0B080944540F2AD80023E46EA074256
:10F12800B3E7E443524263EB430365E7404261EBD4
:10F1380041014FF0FF345CE7B240C6F1200521FAE7
:10F1480005F320FA05F701FA06F9150CB3FBF5F8F3
:10F1580047EA09091FFA82FC05FB18374FEA1941EB
:10F168000CFB08F341EA0747B040BB420AD9BF1875
:10F1780008F1FF3180F09580BB4240F29280A8F1FF
:10F188000208BF18FE1AB6FBF5F305FB13611FFA58
:10F1980089F90CFB03F649EA01418E4206D95F1E44
:10F1A800891878D28E4276D9023B8918891B43EA9E
:10F1B80008438BE7C3F1200726FA07F80CFA03F295
:10F1C80048EA020C21FA07F105FA03FA4FEA1C494A
:10F1D80020FA07F5B1FBF9F845EA0A0509FB181703
:10F1E8002A0C1FFA8CFA0AFB08F142EA0747B942CF
:10F1F80006FA03F609D917EB0C0708F1FF324ED2CD
:10F20800B9424CD9A8F1020867447F1AB7FBF9F252
:10F2180009FB1271ADB20AFB02FA45EA01418A45BF
:10F2280007D9551E11EB0C0137D28A4535D9023A58
:10F23800614442EA08424FEA124C1FFA86F808FB7A
:10F248000CF7360C95B208FB05F806FB057505EBBF
:10F25800184506FB0CFCAF4288BF0CF5803CCAEB96
:10F2680001010CEB1546B14212D309D000230CE77B
:10F278006546EDE60E4646EA074206E70B46FCE61B
:10F288001FFA88F800FA03F308EB0545AB42EDD204
:10F29800013A0023F9E63B4688E72A46C9E7904643
:10F2A800B3E788466EE7023F891823E72DE9F00F98
:10F2B800144605460E46002B3FD18A424AD9B2FA77
:10F2C80082F343B1C3F1200025FA00F201FA03F6F4
:10F2D8009C4016439D40210CB6FBF1F22F0CA0B2C6
:10F2E80001FB126C00FB02F347EA0C46B34208D953
:10F2F800571E361980F0FF80B34240F2FC80023A74
:10F308003619F61AB6FBF1F301FB1361ADB200FB37
:10F3180003F045EA0141884207D95E1E091980F0C9
:10F32800EC80884240F2E980023B43EA0242002333
:10F3380010461946BDE8F00F70478B4243D8B3FA20
:10F3480083F4002C42D18B42234601D382423BD81E
:10F358000122EDE712B90123B3FBF2F4B4FA84F207
:10F36800002A40F08A80091B260CA7B20123B1FBB2
:10F37800F6F006FB10114FEA154C07FB00F24CEAB9
:10F3880001418A4207D9091900F1FF3C02D28A4299
:10F3980000F2D3806046C2EB010CBCFBF6F206FB20
:10F3A80012C1ADB207FB02F745EA0145AF4207D9E2
:10F3B800511E2C1980F0A380A74240F2A080023A87
:10F3C80042EA0042B4E700231A46B1E7C4F1200735
:10F3D80022FA07F603FA04F3334321FA07FA4FEA4D
:10F3E800134C01FA04FB20FA07F141EA0B0BBAFBB4
:10F3F800FCF70CFB17A61FFA83F84FEA1B4508FB1E
:10F4080007F945EA0645A94502FA04FA04D97A1E1D
:10F41800ED18C0F088801746C9EB0505B5FBFCF66A
:10F428000CFB16521FFA8BFB08FB06F84BEA02414D
:10F43800884503D9721EC91870D3164646EA074292
:10F44800170C1FFA8AFC0CFB07F695B24FEA1A4311
:10F458000CFB05FC03FB056505EB1C4503FB07F3EB
:10F46800AE4288BF03F58033C8EB010103EB1543B7
:10F47800994250D347D000235AE79440C2F120085C
:10F48800260C20FA08F721FA08F501FA02F9B5FB6B
:10F49800F6F847EA090906FB1855A7B24FEA194CCE
:10F4A8004CEA054C07FB08F3634500FA02F509D955
:10F4B8001CEB040C08F1FF323DD263453BD9A8F19F
:10F4C8000208A444C3EB0C02B2FBF6F306FB1320BC
:10F4D8001FFA89F907FB03F249EA00418A4206D973
:10F4E800581E091925D28A4223D9023B0919891ABB
:10F4F80043EA08433BE73A4603E7334615E70A463B
:10F5080042EA004214E71FFA8CF100FA04F001EB1A
:10F518000545A842AFD2013A002309E788458CD9AE
:10F52800023EC9188AE7A9457FF675AF023FED1874
:10F5380072E70346DBE79046C4E7023809192AE771
:10F54800002103E00A4B5B584350043109480A4B39
:10F5580042189A42F6D3094A02E0002342F8043BD3
:10F56800074B9A42F9D3F9F77DF900F00DF8704787
:10F57800ACA60508000000200C0B0020100B002092
:10F58800EC610020FEE70000844B854A2DE9F34139
:10F598004FF4FA661E60834BDFF874821A60824A61
:10F5A800824B1A60824B42F210721A60814B6424BB
:10F5B8001C60814B4FF0FF321A60804B00251D7094
:10F5C800012788F80070F7F7B9FEF6F7EBFE20463A
:10F5D800F7F74EFBF6F70CFF2046F7F749FBF7F76E
:10F5E80093FEF7F7E1FCF7F759FB2046F7F740FBE6
:10F5F800F9F720FA2046F7F73BFB4FF4FA50F7F7F4
:10F60800A3FA2046F7F734FBF6F724FE2046F7F76F
:10F618002FFB2846F7F76CFB6948F7F729FBF4F747
:10F628007FF92046F7F724FB664B03F110022946C1
:10F638008DE8240028465A681B68F4F777FB3046A3
:10F64800F7F716FB2846F4F7F1FD4FF6FF70F4F7CD
:10F6580003FE322003215C4A2B46F4F715FF96205F
:10F668008C215A4A2B46F4F70FFF9620584AA021BE
:10F678002B46F4F709FFB421564A2B469620F4F797
:10F6880003FF3046F7F7F4FADC21534A2B462846A5
:10F69800F4F7FAFE5148F7F7EBFA2046F7F7E8FADD
:10F6A800F6F7A0FB2046F7F7E3FA9FED4D0AF7F7C8
:10F6B80037FB2046F7F7DCFA4A4B4B4A00933946AA
:10F6C8004A4B4B48FBF782FC2046F7F7D1FAF5F78F
:10F6D800A5F92046F7F7CCFA1420F6F7F3F82846F0
:10F6E800F6F743F92046F7F7C3FAF6F7C5FA2046C6
:10F6F800F7F7BEFAF6F74EFE2046F7F7B9FAF6F72F
:10F70800C1FB08B188F80050F6F7C8FB08B1F9F753
:10F7180075F8384B00241C70F1F7A2FDF5F734F9A1
:10F7280008B9354802E0354B35481C70F1F7AFFD94
:10F73800344E354DF5F79CFDF8F797F9F8F7CAF907
:10F74800F7F7CEFFF7F702FF3746F6F7BDFB33783A
:10F7580033B1012B02D1F7F755FC01E0F7F77AFC3A
:10F7680000243C70F7F7B8FDF3F75CFBF8F7A4FF4B
:10F778002A8812B2012AE8D124484FF40051FDF733
:10F7880082F9F8F707FAF7F751FD20484FF40051CE
:10F798002246FDF778F92C80D7E700BF64400020A7
:10F7A800E06735008840002080C3C9013841002047
:10F7B8008C4000204C40002084400020684D0020F0
:10F7C80000127A00A8780108A59F0508BF9F0508C0
:10F7D800CB9F0508D79F0508E09F0508002D31013C
:10F7E8000000FA44C40100209840002024020020B0
:10F7F800983A00206C400020BC0D0020943A00206C
:10F80800A80F002090400020FC0B002000080240B8
:10F81800080D002010B4314C0180B1F5807F4460A0
:10F828008270C37052D00DD9B1F5806F39D017D915
:10F83800B1F5006F2ED0B1F5805F24D0FF2040B223
:10F8480010BC704720293AD014D9402930D08029DB
:10F85800F4D123494FF02012C26081600020EEE706
:10F86800B1F5007FEAD11F4B4FF00811C1608360EA
:10F878000020E4E71029E1D11B494FF00122C260C2
:10F8880081600020DBE7194B4FF00111C1608360F4
:10F898000020D4E7164A4FF00213C36082600020AC
:10F8A800CDE714494FF00412C26081600020C6E71A
:10F8B800114B4FF04011C16083600020BFE70F4A31
:10F8C8004FF08013C36082600020B8E70C4A4FF005
:10F8D8001013C36082600020B1E700BFC09E040817
:10F8E800FE8E0508CE8E0508BE900508C08E050858
:10F8F800C28E0508C68E05083E8F0508BE8F05080E
:10F90800DE8E05082DE9F00FB2B02E9030932E9BB5
:10F9180000882E9C5B68309FA4682D90451E03EBE1
:10F928004506BF08209328942C952F911F921E9668
:10F93800319700F03A814FEA900A4FEACA0B00F07B
:10F9480003002F99299003F1080504EB0B00CDF86B
:10F9580084A0CDF8A8B019951A921B9718961791FC
:10F968002B90179A189E13883380B2F802C0A6F815
:10F9780002C09488B480D788F78008361896219FEB
:10F98800199E0832179256F8041C56F8082C4FF0A6
:10F99800000A4FF0000B002F00F06982CDE904AB9C
:10F9A800CDE906ABCDE902ABCDE900AB289CBC465E
:10F9B800029BDDF80C902568C2FBC5394FF00008A2
:10F9C80048EA030ACB46CDE902AB049BDDF814B044
:10F9D800C1FBC53BCDF824B0CDF82080DDE908ABEC
:10F9E800C1EA02004AEA030ACDE904AB069BDDF846
:10F9F8001CB03268C0FBD53BCDF82CB0CDF82880C0
:10FA0800DDE90AABC2EA01074AEA030ACDE906AB17
:10FA18009DE80108C7FBD50BCDF834B0CDF8308090
:10FA2800DDE90CAB4AEA000A63680298CDE900AB4D
:10FA38000834DDF80CB0C1FBC30BCDF83CB0CDF8F1
:10FA48003880DDE90EAB4AEA000ACDE902AB7168FD
:10FA58000498DDF814B0C2FBC30BCDF844B0CDF860
:10FA68004080DDE910AB4AEA000ACDE904AB06980C
:10FA7800DDF81CB0C7FBD30BCDF84CB0CDF84880EF
:10FA8800DDE912ABC1EA02054AEA000ACDE906AB94
:10FA98009DE80108C5FBD30BCDF854B0CDF85080D4
:10FAA800DDE914AB08364AEA000ABCF1010CCDE9DD
:10FAB80000AB7FF47DAF2A9D19982B9B2E18299FA8
:10FAC800002F35D01868039F029BC2FBC037002463
:10FAD8001D971C94DDE91C4544EA0304CDE9024561
:10FAE800049B059DC1FBC035002723952297DDE9BE
:10FAF800224544EA0304CDE90445C1EA0203079D0F
:10FB0800069AC3FBD02525952497DDE9244544EAC8
:10FB180002043368C3EA0101CDE9064553465D4650
:10FB2800C1FBD03527952697DDE926AB4AEA030ABB
:10FB3800069A029C0499039D079FD30B059AE60B2E
:10FB4800C90B46EA454043EA474441EA424604F3C2
:10FB58000F0500F30F0C199BCCEA054706F30F00BD
:10FB68001A9D1B9E2F604FEADA3A08334AEA4B4B3C
:10FB78000BF30F04C0EA04426A600835711E19933A
:10FB88001A951B917FF4EDAE319A2F9E1E991F9BFB
:10FB9800DDF880B0D00037180D182F970BEB000A4E
:10FBA8001F181E951F97CDF880A0DDF8C0C01CF067
:10FBB800030BCDF820B000F086802D9BDDF8BC80CB
:10FBC800CDF808B05808DDF880A0DDF8A0B00690A0
:10FBD800CDF81080049A1E9E32F8025B069826F82B
:10FBE800025B0492BAF80270BBF80230BAF800203F
:10FBF800BBF800401E9617FB03F112FB04F6451EE6
:10FC08004FEAE17711EB06082B4605F0010047EBB8
:10FC1800E6790AF104020BF10401002D3BD0A8B1EA
:10FC2800B2F800C0BBF80470548848881CFB07F57C
:10FC380018EB050749EBE57614FB00F917EB090803
:10FC480046EBE97904320431013B24D00F88B2F83D
:10FC580000C0568848888C8895881CFB07FC18EBE0
:10FC68000C0816FB00F7D088CE8849EBEC7C15FB16
:10FC780004F518EB07084CEBE77918EB050710FBC0
:10FC880006FC49EBE57417EB0C0844EBEC790832F9
:10FC98000831023BDAD11F9A02994FEAD83545EA72
:10FCA800494404F30F0322F8023B4F1E0AF1020AEB
:10FCB8001F9202978ED1DDF880A0DDF820B00AEB04
:10FCC8004B0ACDF880A02C9E2E98B50840683FD0EE
:10FCD800209F47EA000212F0030F00F1080307F122
:10FCE800080214BF002101219F4298BF904294BF8F
:10FCF80000260126314277D097E8420001600121B1
:10FD08006C1EA942466004EA010419D044B192E885
:10FD18001200196002215C6008320833A9420FD032
:10FD280092E850001C605E60966802F1080BD26889
:10FD38009E600231DA601033A9420BF10802EFD15C
:10FD4800DDF880C0ED000CEB050B4019CDF880B054
:10FD58002C9C14F0030343D05A085400002A00F0E6
:10FD68008E80209D40EA050717F0030F209F14BFDF
:10FD780000250125011D3E1D012B94BF002505F01E
:10FD880001058F4298BFB04294BF002101210D4266
:10FD980075D039689200BF18A342016020971044BB
:10FDA800C4EB03011CD0209B013933F8024B0A46EF
:10FDB80020F8024B01F0010192B129B133F8021B7E
:10FDC800013A20F8021B0BD01C46014634F802CB3E
:10FDD80021F802CB5D88A31C4580881C023AF3D128
:10FDE80032B0BDE8F00F7047B7F800C0A0F800C007
:10FDF8007C884480BE888680691EFE880C46BA4688
:10FE080001F00101C680002C9AD089B1B2F800B087
:10FE1800A3F800B051885980B2F804C0A3F804C010
:10FE2800B2F806B00832A3F806B00833013C87D010
:10FE380016881E8051885980B2F804B0A3F804B01F
:10FE4800B2F806C0A3F806C016891E8103F1080B94
:10FE58005189ABF802109389ABF80430D689103277
:10FE6800023C0BF10803ABF80660E1D168E7289B78
:10FE7800CDE904ABCDE906ABCDE902AB1FE61946E7
:10FE880091E700BF2DE9F00F9CB006780F900F9C0A
:10FE980040880F9DA4686D681990B3FBF6FA471E59
:10FEA8004FEA5A0804EB4709AAEB480340460A946C
:10FEB8000D951A97CDF86C800C911492CDF82C9072
:10FEC8001193002800F0B5811746199A199CCDF8AE
:10FED80048809108CA00159104F00303A9181792E5
:10FEE800169310971891760075084FEA450C002D67
:10FEF80000F03B840B9FDDF8308047EA080010F0E3
:10FF0800030F14BF0021012108F10404381D012E3C
:10FF180094BF002101F00101804598BFA74294BF1A
:10FF28004FF000094FF0010911EA090F00F01D8494
:10FF3800BB46D8F8002001236F1EAB42CBF8002047
:10FF480007EA03072146024614D237B12468022380
:10FF58000431021DAB4204600CD20C46104654F822
:10FF6800047B40F8047B496802335160211D021D5F
:10FF7800AB42F2D3DDF83080DDF82CB04FEA4C0507
:10FF8800664508EB05020BEB0503CCEB06001DD01C
:10FF9800013832F802CB014623F802CB00F0010009
:10FFA800A1B128B132F8029B013923F8029B0DD088
:10FFB80014461F4634F8029B27F8029BB2F802A0A9
:10FFC800A21CA3F802A0BB1C0239F1D10C9ADDF8DF
:10FFD8003CC00B989CF80080710053180A9E0C9343
:10FFE800159BCDF84C80451806EB48020B950E92F0
:08FFF800002B00F0B18300248E
:020000040801F1
:100000000025CDE90445CDE9024507930D99134636
:100010000A9AB3F804A0B2F806B0CDF804A0B3F879
:1000200006A00E881588CDF820B0CDF824A0DDE913
:1000300002AB15FB06F51AEB050A4BEBE57BCDE9A8
:1000400002AB1F884888B2F802C0B3F80290B2F839
:1000500004808C88CDF81880DDE904AB16FB07F628
:100060001AEB060A4BEBE67BDDE902671CFB00F5A9
:10007000761910FB09F047EBE5771AEB000A4BEB1A
:10008000E07BCDE902ABDDF818B0DDF804C0B1F8D3
:100090000680099D1BFB04F016EB000A47EBE07B92
:1000A000DDE9026714FB0CF4361947EBE477089C92
:1000B00014FB08F00831083208331AEB000418FB6F
:1000C00005F84BEBE075079816EB080A47EBE87B61
:1000D0000138CDE90245CDE904AB079099D1179ECF
:1000E0000E9C0A9B1899A7199A190E97169F002F14
:1000F00073D00E9B31F8020B32F8024B33F8026BCF
:10010000DDE90289DDE904AB14FB00F47D1E10FB80
:1001100006F618EB040849EBE4791AEB060A4BEBF8
:10012000E67B2F4605F00100CDE90289CDE904AB5D
:10013000002D52D0002873D031F8024B32F8020B58
:1001400033F8025B10FB04F614FB05F0DDE9024511
:10015000DDE90489A41945EBE67518EB000849EBC5
:10016000E079013FCDE90245CDE9048935D0C246A9
:10017000CB46DDE902890D46144604972146284600
:100180001A4630F8026B31F8027B32F802CB6D88E8
:1001900064885B8817FB06F718EB070816FB0CF65C
:1001A00049EBE7791AEB060714FB05FA4BEBE67B04
:1001B00015FB03FC8C1C931C0499851C18EB0A0886
:1001C00049EBEA7917EB0C0A4BEBEC7B8A1ECDE985
:1001D00002890492D2D1CDE904AB029D039904981F
:1001E000DDF828A0059BEA0B109D42EA41481299D0
:1001F00008F30F09A5F80090DDF84C90C70B0AEB47
:100200008908281D4A1E47EA4346CDF8288006F390
:100210000F0410906C8012920AD00F9C267866E62C
:10022000DDE904AB0D4614460497DDE90289A5E734
:10023000149F1B9B07EB83061496119F002F00F061
:10024000A681DDF864B0DDF86480DDF834C04FEAE3
:100250009B09CDF81C904FEAC90908F0030A0CEB82
:10026000090BCDF82090CDF810A0CDF824B0DDF822
:100270003CC09CF8006075084FEA450C002D00F06A
:100280007E820C990B980B9F40EA010414F0030F37
:1002900014BF002201220C1D0430012E94BF002245
:1002A00002F00102814298BFA74294BF00230123BC
:1002B0001A4200F06482BA4601230F68691EAB42FD
:1002C000CAF80070024601EA0307214614D237B18A
:1002D00027680223211D021DAB4207600CD20C4689
:1002E000104654F8047B40F8047B4968023351609F
:1002F000211D021DAB42F2D3DDF83090DDF82C80D9
:100300004FEA4C05664509EB050208EB0503CCEB0B
:1003100006001DD0013832F802BB014623F802BBAB
:1003200000F00100A1B128B132F8025B013923F8D5
:10033000025B0DD014461F4634F802AB27F802AB1F
:10034000B2F802C0A21CA3F802C0BB1C0239F1D152
:10035000DDF82CA0DDF830B0079876000AEB060C2B
:100360000BEB0608CDF82CC0CDF83080002800F04B
:10037000F0810A9ADDF834805788B2F800A0DDF8E1
:1003800028909488B9F80690B8F8062084460D980D
:1003900041880588B8F8040017FB01F61AFB05F33D
:1003A000B3461BEB03014FEAE67714FB00F047EB83
:1003B000E3750F180A9B19FB02F145EBE0750CF190
:1003C000FF3617EB010AB14606F0010008F10802FA
:1003D00003F1080345EBE17B002E00F0858048B374
:1003E000DDF834C01E88BCF80840588851889788CA
:1003F0009D88B2F80680B3F806C016FB04F41AEB29
:10040000040A10FB01F14BEBE4761AEB010415FB37
:1004100007FB46EBE17014EB0B011CFB08F640EB0D
:10042000EB740832083311EB060A44EBE67BB9F1B2
:10043000010959D0CDE902ABCB46B3F80080B3F83F
:1004400008901688CDF8389018FB06F6DDE9028989
:100450005D88548898889188B2F806C0DF88B2F821
:1004600008A015FB04F418EB060810FB01F149EB9A
:10047000E67918EB040817FB0CF749EBE47918EB65
:10048000010849EBE17918EB070849EBE779CDE979
:100490000289DDF838905D89548998899189B2F88C
:1004A0000EC0DE8919FB0AF7DDE9028915FB04F4A9
:1004B00018EB070810FB01F149EBE77918EB04088A
:1004C00049EBE47916FB0CF618EB010449EBE175F6
:1004D00010321033A01945EBE671BBF1020BCDE9E8
:1004E0000201AAD182468B460DF1200898E8160039
:1004F0006318049D9DB332F802CB33F8026B16FBF0
:100500000CF4013D1AEB040A294605F001004BEBFF
:10051000E47B25B358B132F8028B33F8020B10FBA1
:1005200008F71AEB070A4BEBE77B691E17D0144656
:10053000184634F8025B30F8027B52885B8817FB60
:1005400005F81AEB08064BEBE87713FB02FBA21C3D
:10055000831C16EB0B0A47EBEB7B0239E7D10F9DAF
:10056000DDF8508095F800C00A9A119E4FEADA3300
:1005700043EA4B4404F30F0028F8020B02EB4C074C
:10058000711E0A97CDF8508011917FF470AE1A9EBB
:100590000F9CB508A06842D00A9F47EA000616F0F3
:1005A000030F07F1080200F1080314BF0021012125
:1005B0009F4298BF904294BF4FF0000A4FF0010A4B
:1005C00011EA0A0F7FD097E84200016001216C1EFA
:1005D000A942466004EA010419D044B192E812002D
:1005E000196002215C6008320833A9420FD092E8FA
:1005F00050001C605E60966802F10804D2689E603C
:100600000231DA601033A94204F10802EFD1DDF8BB
:1006100028A0ED000AEB05094019CDF82890DDF877
:1006200068A01AF003034AD05A085400002A00F0C8
:10063000A480DDF828B040EA0B0515F0030F14BFC5
:10064000002501250BF10406011D012B94BF002597
:1006500005F001058B4598BFB04294BF4FF0000CE8
:100660004FF0010C15EA0C0F00F08780DBF800104A
:1006700092009344A3420160CDF828B01044C4EB2B
:1006800003011CD00A9B013933F8024B0A4620F8BB
:10069000024B01F0010192B129B133F8021B013A7A
:1006A00020F8021B0BD01C46014634F802CB21F87F
:1006B00002CB5D88A31C4580881C023AF3D11CB094
:1006C000BDE8F00F7047B7F80090A0F800907C8864
:1006D0004480BE888680691EFE880C46B84601F0BC
:1006E0000101C680002C92D091B111881980B2F816
:1006F00002C0A3F802C0B2F804A0A3F804A0B2F8A4
:1007000006900832A3F806900833013C3FF47FAF0F
:1007100011881980B2F802C0A3F802C0B2F80490A0
:10072000A3F80490B2F806A0A3F806A016891E81CB
:1007300003F1080C5189ACF802109389ACF804302D
:10074000D6891032023C0CF10803ACF80660DFD108
:100750005DE70D9A0A9B4FF0000A4FF0000BC8E6C8
:1007600000260027CDE904670A9A0D99CDE90267B2
:10077000BCE430460B9B0C9A0EE4194682E73046E7
:100780000B9B0C9AC6E500BF00B553EC102B42F250
:10079000FB1223F00043C3F6E972934285B026DDD5
:1007A0004FF6FF72C7F6EF7293420BDD51EC100B60
:1007B00002460B46FDF7F0FE02460B4643EC102BBB
:1007C00005B000BD684600F0BFFB00F00300012843
:1007D0009DED000B9DED021B1AD0022810D0F8B938
:1007E00000F0D2FE53EC102B10461946E4E79FEDC3
:1007F000101B00F0C9FE53EC102B10461946DBE726
:1008000000F0C2FE53EC102B104603F10041D3E779
:1008100001F0F6FB53EC102B104603F10041CBE73F
:10082000012001F0EDFB53EC102B10461946C3E7F5
:1008300000000000000000002DE9F04759EC108B8B
:10084000C9F30A56A6F57E74073C132C4D46CA46DA
:10085000474626DC002C4FDB4FF6FF76C0F20F0632
:1008600046FA04F606EA090555EA080517D044A336
:10087000D3E9002351EC100BFDF790FE002200237A
:10088000FEF7CEFA00284AD0B9F1000F6EDB2AEA53
:10089000060A4FF000085346424643EC102BBDE8D1
:1008A000F087332C0CDDB4F5806FF8D151EC100BD0
:1008B0003A460B46FDF772FE41EC100BBDE8F0879F
:1008C000A6F58265033D4FF0FF3323FA05F515EADF
:1008D000080FE4D02AA3D3E9002351EC100BFDF755
:1008E0005DFE00220023FEF79BFAC0B1B9F1000FB4
:1008F0001CDB28EA050813E021A3D3E9002351EC0F
:10090000100BFDF74BFE00220023FEF789FA38B1E9
:10091000B9F1000F1BDB4FF00008C24600E0CA46E9
:100920005346424643EC102BBDE8F087142C09D007
:10093000C6F5866303334FF0010808FA03F818EB95
:100940000708D6D30AF1010A28EA0508E8E729F0E2
:10095000004848EA07084FF0000AD045CBF6F07A85
:1009600008BFCA4618BF4FF00008D9E74FF48013FC
:1009700043FA04F409EB040A89E700BFAFF30080EF
:100980009C7500883CE4377E00B553EC102B42F296
:10099000FB1223F00043C3F6E972934285B027DDD2
:1009A0004FF6FF72C7F6EF7293420BDD51EC100B5E
:1009B00002460B46FDF7F0FD02460B4643EC102BBA
:1009C00005B000BD684600F0BFFA00F00300012842
:1009D0009DED000B9DED021B1DD0022812D008BB1F
:1009E000012001F00DFB53EC102B10461946E3E7F4
:1009F00000209FED111B01F003FB53EC102B104660
:100A00001946D9E7012001F0FBFA53EC102B1046F0
:100A100003F10041D0E700F0B7FD53EC102B104676
:100A20001946C9E700F0B0FD53EC102B104603F156
:100A30000041C1E7AFF300800000000000000000AB
:100A400000F0E6B8D0B52DED048BB0EE408AF0EEA4
:100A5000608A3C4C8AB000F0DBF994F90030B0EECB
:100A6000409AF0EE609A013335D0B0EE480AF0EECD
:100A7000680A01F04FFD00282DD051EC180B002220
:100A80000023FEF7B9F930B32F4B247801930023EC
:100A900008938DED028B8DED048B002C23D0002765
:100AA0000026CFF6F07751EC180B00220023CDE999
:100AB0000667FEF78DF9002825D002239C4200939B
:100AC00036D0684601F05EFD002831D0089B002B2F
:100AD00027D19DED069BB0EE490AF0EE690A0AB0F7
:100AE000BDEC048BD0BD4FF6FF774FF06046CCF2E3
:100AF000EF7751EC180B00220023CDE90667FEF7D3
:100B000067F90028D9D10123022C009315D068463B
:100B100001F038FD88B10D4801F036FD8DED060B72
:100B2000D4E701F0EFFF089B9DED069B0360D2E741
:100B300001F0E8FF22230360C8E701F0E3FF21236F
:100B40000360E8E74C020020ACA1050810A40508EA
:100B500010B52DED048BB0EE408AF0EE608A294C82
:100B60008AB000F02DFC94F90030B0EE409AF0EE1F
:100B7000609A01332BD0B0EE480AF0EE680A01F01B
:100B8000C9FC20B351EC180B00220023FEF72AF910
:100B9000E8B11D4B247801930123009300230893AF
:100BA0008DED048B8DED028BCCB10020002102462F
:100BB0000B46FDF7CFFF022CCDE9060115D101F060
:100BC000A1FF21230360089BABB99DED069BB0EE0E
:100BD000490AF0EE690A0AB0BDEC048B10BD002290
:100BE000002343EC172B8DED067B684601F0CAFC11
:100BF0000028E8D1E3E701F085FF089B9DED069B07
:100C00000360E4E74C020020B4A1050800000000E6
:100C1000F8B5B0EE407AF0EE607A53EC112B544206
:100C200010461D46002125F00047044353EC102BCD
:100C300047EAD474C7F6F0718C4216463DD8544248
:100C4000344323F0004242EAD4748C4235D805F193
:100C5000404101F5801101434FD0AC1704F002046C
:100C6000164344EAD37435D0384341D00021C7F647
:100C7000F0718F424FD00021C7F6F0718A4237D011
:100C8000D21B12153C2A42DC002D7DDB53EC112BCC
:100C900051EC170BFDF75EFF41EC100B01F030FC3F
:100CA00001F06AFA51EC100B012C68D0022C57D0DD
:100CB000002C48D141EC170B07E051EC170B53EC1B
:100CC000112BFDF76BFC41EC170BB0EE470AF0EE71
:100CD000670AF8BD032CC7D801A151F824F000BF62
:100CE000CB0C0108CB0C0108090D0108030D01080C
:100CF000002B25DB9FED307BE7E7BDE8F84001F0F6
:100D00003BBA9FED2F7BE0E79FED2F7BDDE72AA12C
:100D1000D1E90001C8E7BA423CD0032CABD801A10D
:100D200051F824F03B0D0108350D0108090D0108AB
:100D3000030D01089FED267BC7E79FED277BC4E7E6
:100D40009FED277BC1E730A3D3E90023FDF724FC07
:100D50001DA3D3E90023FDF71FFC41EC170BB4E7FB
:100D600029A3D3E90023FDF717FC02460B4616A181
:100D7000D1E90001FDF710FC41EC170BA5E701F1EB
:100D8000004141EC170BA0E73C32BFF67FAF0020DB
:100D9000002189E7032CABD8DFE804F00B0805023B
:100DA0009FED117B91E79FED127B8EE79FED127B0C
:100DB0008BE79FED137B88E7182D4454FB21F93F07
:100DC000182D4454FB2109C0182D4454FB2109401F
:100DD0000000000000000080000000000000000093
:100DE000182D4454FB21F9BFD221337F7CD902C096
:100DF000D221337F7CD90240182D4454FB21E9BF16
:100E0000182D4454FB21E93F075C143326A6A13C6E
:100E10002DE9F84F55EC104BB5F5801F2F4622DA1F
:100E200025F00043234368D0002D2046294670DB7F
:100E300000230022C4F25033FDF762FD4FF6FF732A
:100E40000F46C7F6EF739F4204460D466FF035021A
:100E500010DD2046294622462B46FDF79FFB41EC3C
:100E6000100BBDE8F88F4FF6FF73C7F6EF73002243
:100E70009F42EEDC3B15A3F57E73073B9A18D60F15
:100E8000901927F07F47C6F57E76FDF7D3FC07362D
:100E900027F4700747EA065545EC104B8046894613
:100EA00001F00AFC4046494621A3D3E9002355EC52
:100EB000104BFDF725FD20A3D3E9002382468B4686
:100EC00040464946FDF71CFD1DA3D3E90023064615
:100ED0000F4620462946FDF713FD02460B463046D5
:100EE0003946FDF75BFB02460B4650465946FDF777
:100EF00055FB41EC100BBDE8F88F00210020CCF22F
:100F0000503100220023FDF725FE41EC100BBDE817
:100F1000F88F22462B46FDF73FFB00220023FDF70A
:100F200019FE41EC100BBDE8F88F00BFAFF3008055
:100F300000609F501344D33F362BF111F3FE593D0F
:100F40000EE526157BCBDB3F2DE9F04F53EC102B44
:100F500042F2FB1223F00044C3F6E97294428FB0D0
:100F60001E46074640F3AA804DF67B13C4F20203E7
:100F70009C422ADC002E51EC100BDDA3D3E90023A8
:100F800040F3CA81FDF708FB42F2FB13C3F6F97385
:100F90009C428046894600F0AA80D7A3D3E900236B
:100FA000FDF7FAFA0D4604462B462246C7E90045EE
:100FB00040464946FDF7F0FACFA3D3E90023FDF7F9
:100FC000EBFA0125C7E9020181E042F2FB13C4F20A
:100FD00039139C4240F3AA804FF6FF73C7F6EF73B4
:100FE0009C4278DC4FEA245AAAF5826AAAF1060AE2
:100FF00051EC100BA4EB0A5319461D460446FDF7AD
:1010000019FFFDF717FC8046894642464B462046AD
:101010002946CDE90889FDF7BFFA00230022C4F272
:101020007013FDF76DFC0D460446FDF703FFFDF759
:1010300001FC804689462046294642464B46CDE97A
:101040000A89FDF7A9FA00230022C4F27013FDF704
:1010500057FC002204460D460023CDE90C45FDF760
:10106000B7FE002800F07B8140464946002200235D
:10107000FDF7AEFE03240AAD013C40B175E9020163
:1010800000220023FDF7A4FE013C0028F6D12346F0
:10109000022400949E4C08A839465246019400F060
:1010A000ABFB002E054612DA7A68FB6802F10042BB
:1010B00003F100437A60FB60454208E00022002310
:1010C00043EC172B87ED000B80ED027B00252846B3
:1010D0000FB0BDE8F08F51EC100B02460B46FDF748
:1010E0005BFA0025C7E90201C7E90001EFE77AA32F
:1010F000D3E90023FDF750FA79A3D3E90023804612
:101100008946FDF749FA0D4604462B462246C7E9B3
:10111000004540464946FDF73FFA71A3D3E9002355
:10112000FDF73AFA0125C7E90201D0E701F0E8F935
:1011300059EC108B6CA3D3E9002340464946FDF7D8
:10114000DFFB00230022C3F6E073FDF727FAFDF76B
:1011500071FE0546FDF76EFB65A3D3E90023CDE9DB
:101160000201FDF7CDFB02460B4640464946FDF71E
:1011700013FA61A3D3E9002382468B46DDE902011D
:10118000FDF7BEFB1F2DCDE90401504659462BDC6F
:101190006A1E604B53F82230A34225D0DDE90423B8
:1011A000FDF7FAF902460B46C7E900238146884657
:1011B0004A46434650465946FDF7EEF9DDE9042319
:1011C000FDF7EAF9002E02460B46C7E90223BFF6F7
:1011D0007EAF08F1004301F10041C7F800907B6049
:1011E000B860F9606D4272E7DDE90423FDF7D4F9D8
:1011F00088462415C8F30A53E31A102B8146C7E921
:101200000001D5DD34A3D3E90023DDE90201FDF7B8
:1012100077FB8046894642464B4650465946FDF785
:10122000BBF9CDE90601DDE9062350465946FDF735
:10123000B3F942464B46FDF7AFF929A3D3E90023A2
:1012400080468946DDE90201FDF75AFB42464B46DE
:10125000FDF7A2F9CDE90401DDE90423DDE906018A
:10126000FDF79AF98846C8F30A53E41A312C8146EF
:10127000C7E9000140F3958021A3D3E90023DDE90C
:101280000201FDF73DFB8046894642464B46DDE9BB
:101290000601FDF781F982468B4652465B46DDE941
:1012A0000601FDF779F942464B46FDF775F916A39D
:1012B000D3E9002380468946DDE90201FDF720FBE2
:1012C00042464B46FDF768F9CDE9040150465946C0
:1012D00064E700BFAFF300800000601A61B4D03D46
:1012E0007370032E8A19A33B83C8C96D305FE43F36
:1012F00000004054FB21F93F3163621A61B4D03DD4
:101300000000002E8A19A33BC14920259A837B390E
:101310003CA20508BCA10508FDF740F942F2FB1309
:10132000C3F6F9739C42804689461AD01EA3D3E9BE
:101330000023FDF733F90D4604462B462246C7E944
:10134000004540464946FDF727F917A3D3E9002396
:10135000FDF724F94FF0FF35C7E90201B7E6032492
:1013600095E613A3D3E90023FDF718F912A3D3E9F7
:10137000002380468946FDF711F90D4604462B46A9
:101380002246C7E9004540464946FDF705F90AA34C
:10139000D3E90023FDF702F94FF0FF35C7E9020159
:1013A00095E6DDE906AB03E73163621A61B4D03D2F
:1013B0000000601A61B4D03D7370032E8A19A33BFC
:1013C0002DE9F84353EC102B00242546C7F6F074A2
:1013D000C7F6F0751C40AC422DED028BB0EE408A92
:1013E000F0EE608A1946104600F0AB80002B7FDDDE
:1013F0001A1500F08980A2F57E7721F07F4323F44F
:101400007003073FD20743F4801366D5C20F4FF035
:10141000000C02EB43037F104200654616204FF498
:1014200000116C18D60F9C424FEA420202DC65188C
:101430001B1B8C444908013806EB4303F1D12026DD
:1014400080464FF0004107E043D0D40F49085200D6
:10145000013E04EB43031BD0AB4208EB0104F3DD78
:1014600004F00049B9F1004F04EB01082BD0A94664
:101470009442C5EB0303C4EB020288BF013B401852
:10148000D40F49085200013E4D4604EB4303E3D11B
:101490001A4327D146084FEA6C0101F17E511CF036
:1014A000010F01F5C00118BF46F0004601EB0753DC
:1014B000324643EC182BB0EE480AF0EE680ABDEC59
:1014C000028BBDE8F883B8F1000FD0DB05F101090C
:1014D000CEE79442C4D91D46B7E7C20F02EB4303DF
:1014E000400093E7431C39D000F001031818D1E7FE
:1014F00023F000441443DED0002B36D11A46C10A33
:10150000153A40050029FAD011F4801329D1490079
:101510000133CC02FBD5C3F10105C3F1200420FA4D
:1015200004F4521921439840A2F57E7721F07F43BD
:1015300023F47003073FD20743F480133FF566AFEF
:10154000CBE751EC100BFDF7DBF902460B4651ECF3
:10155000180BFDF723F841EC180BACE70CF1010C6C
:1015600099E7202401250023D9E751EC100B0B4605
:10157000FDF712F802460B46FDF7ECFA41EC180BAA
:1015800099E700BF000000002DE9F04F5BEC10ABC5
:101590002DED028BB0EE418AF0EE618A2BF0004413
:1015A000B4F1795F85B071DA50465946FDF742FCD7
:1015B000002800F0FD8052465B4650465946FDF734
:1015C0009FF981A3D3E9002306460F46FDF798F95A
:1015D0007FA3D3E90023FCF7E1FF32463B46FDF74A
:1015E0008FF97DA3D3E90023FCF7D6FF32463B46B3
:1015F000FDF786F97AA3D3E90023FCF7CFFF324643
:101600003B46FDF77DF978A3D3E90023FCF7C4FF3F
:1016100032463B46FDF774F975A3D3E90023FCF786
:10162000BDFF32463B46FDF76BF9804689460023F5
:101630000022C3F6E07330463946FDF761F94246B1
:10164000CDE900014B4630463946FDF759F953ECD8
:10165000182B04460D4650465946FDF751F90246EF
:101660000B4620462946FCF797FF02460B46DDE96C
:101670000001FCF791FF0B4600210246C3F6F07112
:101680000020FCF789FF41EC100B83E052465B46DB
:1016900050465946FDF734F94BA3D3E900230646DB
:1016A0000F46FDF72DF94AA3D3E90023FCF776FF97
:1016B00032463B46FDF724F947A3D3E90023FCF764
:1016C0006BFF32463B46FDF71BF945A3D3E90023E8
:1016D000FCF764FF32463B46FDF712F942A3D3E91B
:1016E0000023FCF759FF32463B46FDF709F940A3BA
:1016F000D3E90023FCF752FF3B463246FDF700F9E1
:1017000043F23233C3F6D3739C42804689468EDD62
:101710000023C3F6E9739C4241DC0021A4F50013C9
:1017200000220020C3F6F07114461D46FCF734FF7A
:10173000CDE9020100230022C3F6E07330463946AA
:10174000FDF7DEF822462B46FCF726FF4246CDE9A0
:1017500000014B4630463946FDF7D2F853EC182BC2
:1017600004460D4650465946FDF7CAF802460B4658
:1017700020462946FCF710FF02460B46DDE9000132
:10178000FCF70AFF02460B46DDE90201FCF704FF05
:1017900041EC100B05B0BDEC028BBDE8F08F9FED66
:1017A000067B00258DED027B0024C3F6D275C1E7D0
:1017B0009FED030BEEE700BF000000000000E73FD5
:1017C000000000000000F03FD43888BEE9FAA8BD50
:1017D000C4B1B4BD9EEE213EAD529C804F7E923E80
:1017E0009015CB19A001FA3E7751C1166CC1563F36
:1017F0004C5555555555A53F2DE9F04F4AF6AB25AB
:10180000ADF51B7DD41EC2F6AA2585FB0465E41741
:10181000A49F114E0690C4EBA50424EAE47456F884
:1018200027600A941F46E34303EB43037C1E02EB4D
:10183000C30314EB0608099602940891079321D478
:101840000A9EA599351B08F101080CAE4FEA8808DD
:10185000002401EB85090BE044A3050859F80400B6
:10186000FCF7E8FF043401354445E6E9020109D0FC
:10187000002DF3DA04340020002101354445E6E967
:101880000201F5D1099C002C2CDB099C5EAE06EB15
:10189000C4060DF5B87ABB460096029D002DC0F235
:1018A00054820EA9069D01EBCB064FF000084FF0C5
:1018B0000009002476E90223F5E80201FDF720F88B
:1018C00002460B4640464946FCF768FE0134BC42DE
:1018D00080468946EED1EAE90289009DAA450BF1CE
:1018E000010BDAD1099E731E9B0086AC9AAD04EB06
:1018F0008604ED180B9300960C940D95009C009EA9
:10190000E4009AAD2B19002E049453E93C892EDD96
:1019100004995EAC059485AE651800230022C3F6D9
:10192000706340464946FCF7EBFFFDF783FAFCF78E
:1019300081FF00230022C4F2701382468B46FCF71D
:10194000DFFF02460B4640464946FCF725FEFDF701
:1019500071FA044646F8044F75E9020152465B46A7
:10196000FCF71CFE059CA54280468946D5D149EC72
:10197000108B079800F010FE55EC104B00224FF032
:101980007F5320462946FCF7BBFF41EC100BFEF7C6
:1019900053FF002351EC100B0022C4F22003FCF78C
:1019A000AFFF02460B4620462946FCF7F5FD0D46E3
:1019B0000446FDF73FFA0646FCF73CFF02460B469D
:1019C00020462946FCF7E8FD079D002D8046894604
:1019D00040F3C180009C9AAD621E05EB8202079C19
:1019E00052F8503CC4F1180043FA00F101FA00F03B
:1019F0001B1AC4F11700761842F8503C43FA00F560
:101A0000002D30DD009C0136002C40F3B18186AA08
:101A100002EB840000244FF6FF7352F8041BC0F25F
:101A2000FF035B1A14B9C1F1807311B142F8043C91
:101A300001248242EFD10799002911DD012900F02C
:101A40006D8102290CD1009A9AA9531E01EB8303E0
:101A500053F8502C22F07F4222F4400243F8502CDD
:101A6000022D00F082804046494600220023FDF707
:101A7000AFF9002800F09C80009C601E099C844205
:101A80000EDC009C86A901EB84030C9C002253F819
:101A9000041DA34242EA0102F9D1002A40F07082FB
:101AA0000D9C54F8503C002B40F068820B9D86AE94
:101AB0007219012352F8041D01330029FAD0009C49
:101AC000E31804F1010A9A45059341DC0A9E029D40
:101AD00004EB060BA59C05EB0A0304EB8B0B049CA3
:101AE000013B0EAD5EAE05EBC305361900950496BD
:101AF0005BF8040FFCF79EFE009D029EE5E90201E3
:101B0000002E00954FF000084FF0000917DB0AEB9C
:101B100007060EA9069D01EBC606002476E90223FE
:101B2000F5E80201FCF7ECFE02460B46404649464A
:101B3000FCF734FD0134BC4280468946EED1049C5A
:101B4000059DE4E902890AF1010AAA450494CFDD62
:101B5000059E0096D2E640F0EF80009D9AA901EB29
:101B6000850353F8545CED154AE7002142464B4685
:101B70000020C3F6F071FCF70FFD80468946002C6B
:101B80003FF471AF07989FED8E0B00F005FD4046C6
:101B900053EC102B4946FCF7FFFC80468946404633
:101BA000494600220023FDF713F900287FF464AFB3
:101BB00005960495002840F0FC81079C49EC108BA9
:101BC000604200F0E9FC57EC106B002330463946C8
:101BD0000022C4F27013FDF719F9002800F0F78114
:101BE00000230022C3F6706330463946FCF788FEB6
:101BF000FDF720F9FCF71EFE00230022C4F270134B
